:020000040800F2
:1000000000C00020D14D0108714E0108B937010828
:10001000714E0108714E0108714E01080000000088
:10002000000000000000000000000000714E010808
:10003000714E010800000000714E01082FA6000853
:10004000714E0108714E0108714E0108714E010890
:10005000714E0108714E0108B1E30008AFE30008DA
:10006000714E0108714E0108714E0108714E010870
:10007000714E0108714E0108C5E30008714E010878
:100080005D890008714E0108714E0108714E01082A
:10009000714E0108714E0108714E0108ADE3000870
:1000A000714E010829D40008714E010839D40008A6
:1000B00019D4000809D40008F9D30008956700088E
:1000C000996700088D67000891670008714E010864
:1000D000714E0108BDE30008B3E30008714E01084A
:1000E0003DA60008714E0108714E0108714E0108CD
:1000F000714E0108714E0108714E0108714E0108E0
:10010000714E0108714E0108714E0108714E0108CF
:10011000714E0108714E0108714E0108714E0108BF
:10012000714E0108714E0108714E0108714E0108AF
:1001300000000000000000000000000000000000BF
:1001400000000000000000000000000000000000AF
:10015000000000000000000000000000000000009F
:10016000000000000000000000000000000000008F
:10017000000000000000000000000000000000007F
:10018000000000000000000000000000000000006F
:10019000000000000000000000000000000000005F
:1001A000000000000000000000000000000000004F
:1001B000000000000000000000000000000000003F
:1001C000000000000000000000000000000000002F
:1001D000000000000000000000000000000000001F
:0401E0005FF8E0F1F3
:1001E8002DE9F04F684B694F9FB03B6000237B605F
:1001F80010F0DAFE18B910F0F9FE09F04DF809F020
:10020800F7F8634A634D1378634E43F001031370A4
:1002180000230693079308934FF4E01309932B6880
:10022800B07B43F480332B60AB6943F01003AB61C0
:100238002B6803F400330793069B01330693079B4F
:100248001BB9069BB3F5A06FF2D12B68514913F483
:10025800003301D0022315E00A6842F001020A6067
:1002680006932B6803F002030793069B013306935A
:10027800079B1BB9069BB3F5A06FF2D12B689A07B1
:1002880039D501230893454B45491A6842F01002B5
:100298001A601A6822F003021A601A6842F0020211
:1002A8001A606B686B606B686B606B6843F48063A3
:1002B8006B603C4B1A68043B22F070425A603A4A21
:1002C8001160696821F47C116960596841F0004146
:1002D8005960D96821F40041D9609B681B0449BF63
:1002E800324B4FF4E01313604FF480130993089BCB
:1002F800012B01D117E0FEE7022B18D168B1099B49
:10030800B3F5801F02D14FF4A01305E0099BB3F5A4
:10031800E01F02D14FF40013099309996B680B434E
:1003280043F4803302E06B6843F460136B602B681E
:1003380043F080732B602968164B8C01FBD55968F4
:1003480021F003015960596841F0020159606B6856
:10035800104903F00C03082BF9D14B68DFF854B0AF
:1003680003F00C03042B03D0082B03D00C4B29E01B
:10037800136827E04B684868C3F38343C00303F15D
:10038800020319D40A4A1CE0878A0008D800002012
:1003980058310020001002400811002000200240BF
:1003A80000127A000410014038000020001BB7003A
:1003B80000093D0060000020496812688C0348BFAE
:1003C80052085343CBF800306B68DFF87082C3F3F0
:1003D800031343441A7EDBF800301EACD340CBF83D
:1003E80000307F4A7F4BDFF858A2D360AB69029296
:1003F80043F00103AB616B6A4FF00009BB606B6AA5
:10040800794843F080736B62AB6943F01C03AB61BE
:100418004FF6FF7324F82C3D21468DF84E900FF0CF
:1004280043FE504621460FF03FFE704821460FF02C
:100438003BFE6F4920464B6843F000734B600FF05A
:1004480071F9139B6B49A646B3FBF1F36A49029A0B
:100458000B606A4B4FF47A71C3F80090DBF80030F8
:10046800DFF8E0C1B3FBF1F36549013B4B60F023D2
:1004780082F823300723C1F808900B60B36808F1AD
:10048800280BCCF80030BBE80F00AEE80F009BE863
:100498000300AB698EE8030043F00803AB61AB6966
:1004A800042243F00803AB61AB6943F02003AB615E
:1004B8000823CAF810301023CAF81030E246514B0E
:1004C8001A6109F1040154F80900214409F10809E5
:1004D8000FF0EAFDB9F1180FF3D164200AF099F88A
:1004E800A0224948002116F0D0FDEB69002243F014
:1004F8000703EB61AB6943F4006343F00C03AB61A2
:10050800424B4FF0000B03F10C0102F801B001322D
:100518000E2AF5D1FF229A76DA761A775A773C4B6B
:100528003C4A59461A603C483022DAF8005016F026
:10053800ACFD5946C5F380190423384ADFF8D8E0E2
:10054800885C0C224A4302F80E00B9F1000F08D16A
:100558001E3801289FBFFF2003F1FF3302F80E0069
:10056800DBB201310429E8D12D4A2E481370737982
:100578002D4A264913702D4A3A62C03202602C4A2D
:10058800A80602EBC302527848BF01224A62002241
:1005980040F2DC50274921F812000132082AF7D12D
:1005A8000CA800211C22029316F06FFD15F4007BA5
:1005B80005F4006A029B47D0AA040BD4BAF1000FD5
:1005C8000AD01D4A96F88601A2F10C01012808BF3D
:1005D8000A4602E0194A00E0174A0292129435E0EE
:1005E80000ED00E00005FA05000801400010014098
:1005F8000000014040420F00801F0020841F00209F
:1006080010E000E000140140CC1F0020D8000020BA
:100618007C2A0020FC120020802A002071C90108D1
:10062800BD100020E8200020400900201C110020F7
:1006380010BF010828100020689601085C96010880
:10064800000C0140542D0020CDF808B00E2B03D02B
:1006580003F0EF03082B02D101238DF8423001206B
:1006680009F078FD18B14088003018BF0120C5F3A3
:1006780040038DF83630C5F3403300F001008DF8A3
:100688003030C5F3C0338DF835008DF838908DF8CB
:100698003330BAF1000F07D096F886A10AF1FF3E71
:1006A800DEF1000A4AEB0E0AC5F300438DF8393033
:1006B8007B6A1BF1000B18BF4FF0010B003318BF0A
:1006C80001238DF83B30C5F300538DF83C30B6F864
:1006D8004A31B6F84801ADF84030B6F8563105F061
:1006E8000101C5F3C002ADF83E30C5F38043ED0407
:1006F800ADF8460048BFB9488DF8373048BFB0F864
:100708005001B6F8543148BFADF84600B3F5FA7F4A
:10071800ADF8443084BF0023ADF8463096F8D631A2
:10072800AF4887F82830002387F8293043709DF8B0
:1007380042308DF834A0002B8DF831108DF832201E
:100748008DF83AB00CBF0023022301B902B101337E
:1007580008EB8308D8F840304FF00009A3F1020AEB
:100768001A3303934FF6FF733AF802BF9B4500F024
:1007780081819DF835205FFA8BF31AB19A1E012A00
:1007880040F274819DF8382032B196491A0189588F
:10079800954A914200F06A819DF8392032B1914919
:1007A8001A018958904A914200F060819DF83620DC
:1007B80052B18C4A8D4802EB03125168814203D131
:1007C8001289102A00F052819DF8332052B1854ACF
:1007D800864802EB03125168814203D11289022A2A
:1007E80000F044819DF8342052B17E4A804802EBE3
:1007F80003125168814203D11289022A00F036811E
:10080800129A7AB1774D116805EB0315686888422A
:1008180008D129899088884200F02881D2888A42A4
:1008280000F024814FEA1B2BBBF1020F02D19DF887
:10083800302004E0BBF1010F04D19DF83120002ADB
:1008480000F01481674A9DF83C004FEA031802EB58
:100858000805114630B19DF8420018B9043B032B36
:1008680040F2EC80BBF1010F5FFA8BF344D1614E8B
:100878004144FF2391F80DE086F8703086F8713016
:10088800486801F1080309890027ADF84C100221D6
:100898008DF84F1086F8747013A9C6F880508DF83B
:1008A8004EE00592049386F82C7037637763B7633C
:1008B800F76686F8727086F873700FF0F5FB049B84
:1008C800059A997852F808003A4607F094FE2846A7
:1008D80039465A460DF0C2FC474BC6F88C70C6F82C
:1008E8008430464B2846C6F8883006F1840106F164
:1008F80088020DF0FBFCB9E0022B4AD15FFA89F2BD
:100908001C2101FB02FC3B4A002602EB0C07354A7E
:100918004FF0010B02EB080191F80DE001F108021C
:100928004868098987F87590ADF84C1087F87660A3
:1009380013A987F87E6087F874B0C7F88050CDF89F
:1009480014C08DF84EE004928DF84F300FF0ACFBD8
:10095800244B049A53F808009178324607F04BFE6E
:10096800284631465A460DF079FC254A214BDDF8D8
:1009780014C0C7F8842003EB0C01224A8431C7F85D
:100988008820C7F88C6028460A1D0DF0AFFCD944B2
:100998006CE0032B50D19DF83730164E1A4F3BB1FF
:1009A80096F82A80284608214FF6FF72002337E080
:1009B800BDF8442096F82A80B2F5FA7FBDF8463093
:1009C80028D912492846B1FBF2F2082192B207F061
:1009D80067FE0F4B47F8280027E000BF08110020EA
:1009E8000101002030B9010800040040000801405E
:1009F800000C0140D80000206D8000084D810008DF
:100A08003986000843800008981F002000127A00E9
:100A18006D8100086A492846B1FBF2F2012192B2C1
:100A280007F03EFE674B47F82800C36096F82A3067
:100A3800013386F82A3019E0042B17D1BDF83E207F
:100A48005F4B614E93FBF2F22846BDF8403001211E
:100A580092B296F8297007F023FE96F8293006EB33
:100A680087070133C7F8540186F82930039B9A4554
:100A78007FF478AE544E554B96F82920002586F819
:100A88007421534A1D7017789846A7F11702022A55
:100A98001AD8336A0021585903EB050913F044F9B1
:100AA80010B1736A7BBB27E04A4B05EB030E99E84C
:100AB8000F008EE80F0098F8003010350133C02D74
:100AC80088F80030E5D1ECE7434B13F837C003EB67
:100AD800C703D3F8049088F800C0B9F1000FE0D03C
:100AE8006545DEDA3B4A2B0103EB020E4B440FCB84
:100AF80001358EE80F00F3E7384B1A68994612F46F
:100B0800805F26D11FE0364B364A13F8370003EBD7
:100B1800C7035D681070002DEED000238342EBDA26
:100B2800C3EBC3016A18D2F80090DFF8C4C00133E0
:100B380041F80C9001EB0C0E9188AEF804109279F4
:100B48008EF80620EAE707F0EF03082B264B25D19D
:100B580026E098F80030012BF5D9244D05EB031356
:100B680003F1100810354545EDD055F8100C4FF03D
:100B78007C5112F045FF4FF07C5145F8100C55F8A8
:100B8800140C12F03DFF4FF07C5145F8140C55F849
:100B98000C0C12F035FF45F80C0CE3E70E2F08D1CA
:100BA8001A78182F42F010021A7023D109F0A0FF0A
:100BB80020E01A78192F22F010021A70F5E700BF0A
:100BC80040420F005D810008D8000020C81F0020A7
:100BD800400900207C08002010BF0108542D002087
:100BE800A4A4010874200020FC1800208408002018
:100BF8007520002009F060FFD9F80030BC4F580379
:100C08005EBFBC4B01221A70BB4A4FF48058137860
:100C18004FF0020B43F00403137014238DF84E3089
:100C2800BB69214643F00403ADF84C808DF84FB002
:100C3800B248BB610FF038FAB14AB24B00201A60D3
:100C480009F000FDB04BB14D93E80300BB6984E89F
:100C5800030043F00803BB61139814A90FF024FAAA
:100C6800FB69284643F48043FB613B69214643F412
:100C780080433B6118238DF84E304FF42043ADF884
:100C88004C3003238DF84F304FF0040A0FF00CFA64
:100C98004FF48043284621464FF01009ADF84C30F8
:100CA8008DF84EA00FF000FA28462146ADF84C808A
:100CB8008DF84E900FF0F8F93A69072342F4804214
:100CC8003A613A69012022F480423A61904A1188D7
:100CD80001F4415141F4457141F003011180918BB8
:100CE80021F4006101FA09F121FA09F191831382D3
:100CF800118889B241F040011180C5F81080DFF8F1
:100D08002C820FF0EBFBD8F80040824D04F400432E
:100D180003934A4604F4006328460021049316F01E
:100D2800B4F94FF6FF728DF82EB014F002044FF0AC
:100D3800000BADF82C208DF82FB00DD01EA921F88E
:100D48004C9D6E480EF092FE0124072385F800A002
:100D580085F801B0AC70EB70039B73B102231EA938
:100D680021F84C3D65480EF081FE0123E2182B71F5
:100D7800AB7107236C71EB71D4B2049B7BB1022376
:100D88001EA921F84C3D61480EF070FE092301228E
:100D98002B73AA73631C07226C73EA73DCB27B683B
:100DA8005D4843F440437B607B694FF0000943F0A2
:100DB80001037B61BB69DFF860A143F40073BB6189
:100DC8000EF038FC554B012C1393554B13A9149373
:100DD80094BF4B46802318934FF4807319934FF4B4
:100DE80080631A9320231B9350464FF400531694A4
:100DF8001C93CDF85490CDF85C90CDF874900EF01B
:100E0800FBFBDAF80030474A43F00103CAF8003028
:100E18005368012C23F4702394BF0021012123F48B
:100E2800807343EA0123536091683F4B013C0B40B8
:100E380043F4602343F002039360D36AE4B223F4DB
:100E4800700343EA0454D462012305EB0902917844
:100E580000297DD015F80900591C0928C9B2D27893
:100E6800DFF8C0E011D9A0F10A04DEF80CA004EB09
:100E780044044FF0070C0CFA04FC2AEA0C0CA240BC
:100E88004CEA0202CEF80C200EE0DEF8104000EB2F
:100E9800400C4FF0070A0AFA0CFA24EA0A0402FA8C
:100EA8000CF22243CEF81020062B1E4C0ED8013B24
:100EB800626B03EB83034FF01F0E0EFA03FE22EA68
:100EC8000E0200FA03F31343636340E00C2B2FD8A0
:100ED800073B226B03EB83034FF01F0E0EFA03FE52
:100EE80022EA0E0200FA03F3134323632FE000BF44
:100EF80000100240A80D00205831002000080140D1
:100F080095A4000868310020AC960108000C014047
:100F180000380040DC2A0020080002404C24014030
:100F2800EC2A002000240140FDF7F1FF542D002099
:100F3800A3F10D02D4F82CC002EB82021F239340C8
:100F48002CEA030E00FA02F34EEA0303E3620B46AF
:100F580009F10409B9F1100F7FF477AFAF4B9A6824
:100F680042F480729A609A6842F001029A609A6824
:100F780042F008029A609968A84A0907FBD4936866
:100F880043F004039360A54B9A6812F00409FAD160
:100F9800A34D9A68B5F85C0142F4A0029A60002853
:100FA80041F08782B5F95E31002B41F08282B5F9B4
:100FB8006031002B41F07D82D8F800309B031FD5AB
:100FC800C82009F026FBAE200FF0F3F908B10FF0A6
:100FD800F5F9944C86F87501C82009F01AFB924B74
:100FE80000210C222046C6F8783116F04EF802236C
:100FF800E3700CF034FC09F0E5FA8C4B0344A36071
:1010080095F86B31B5F864410493894B95F863A161
:101018001B6895F86C81B3F85630B5F80CB0059399
:10102800EB7B844D00210C228348039316F02DF8A6
:1010380014222846002116F028F8804A002313704D
:10104800C6F87C3105F092FC30B37D4BB4F5807F57
:101058002B607C4B6B607C4BEB607C4B2B617C4B3F
:1010680001D1002216E0BB2C01D9012212E0612C2B
:1010780001D902220EE0292C01D903220AE0132CFF
:1010880001D9042206E0092C01D9052202E0002C2E
:10109800E7D006221A7062E06E4B93F8825125B9A8
:1010A80005F022FC002800F070836B4B00221A80A8
:1010B8000DB905F0C3FBB4F5807F00F06B83BB2C42
:1010C80000F26A83612C00F26983292C00F268839C
:1010D800132C00F26783092C00F26683002C14BFDE
:1010E800062500255D4A1920138823F040031B04B8
:1010F8001B0C1380138823F038031B041B0C43F0CC
:101108003003138013889BB243F04003138096F892
:10111800801105F083FB012009F070FA29461A2096
:1011280005F07CFB012009F069FA13A805F0F8FA2C
:101138009DF94E30484A013300F0208313889BB252
:10114800002B40F020833B4B454A64201A60454AF7
:101158005A60454ADA603D4A1A6109F05AFA012391
:10116800424A434D2B70136843F001031360002378
:10117800404ABAF1090F00F2B180DFE80AF005AF82
:101188000505818105819AA51370C6F87C3105F0A3
:10119800EDFB002875D006210A4613AB682010F035
:1011A8005FFC9DF8511001F001029DF84F1001F00D
:1011B80001014B0043EA82019DF84D2002F0010332
:1011C8000B430AD05BB2012B01D1002302E0022BB2
:1011D8000ED1012386F8813111E00BAB68200C2178
:1011E800012210F03DFC9DF82C3013F00F0303D1C1
:1011F800052009F07BFA02E0042BEAD1E5E70E4B63
:101208001D4A1A601D4A5A6096F88121002A0CBFAF
:101218006F226E221A720323F0E200BF00240140FD
:10122800081100204829002092120020404B4C0051
:1012380038100020EC200020202D00200021002064
:10124800A9640008B56300083564000890C1793DB9
:1012580000000020D8000020442D00200038004065
:101268004962000829670008A1660008F8180020EC
:101278005C0000208331002019650008F563000830
:10128800137096F8826136B1C44B00221A8036B9C1
:1012980005F0D4FA03E005F027FB58B1F4E7C04B9A
:1012A800C04A64201A60C04A5A6009F0B2F907239C
:1012B800A4E2137005F06EFA38B1B94BBB4A1A6054
:1012C800BB4A5A60082399E21370B54BB94A1A60B1
:1012D800B94A5A6000221A7209238FE2BAF1010F43
:1012E8003FF652AF1370B8F1040F00F2BF81DFE888
:1012F80018F00500C801680005008A010A2009F0F5
:1013080088F97720A02101220BAB10F0A9FB002857
:1013180057D01E210122772010F0E2FB4FF42F60F6
:1013280009F06CF90026A6F160010025C9B2022275
:1013380013AB77208DF84C508DF84D5010F090FB82
:101348009DF84D309DF84C2043EA02229B4B03F553
:10135800C27172520236102EE5D1B3F89221294695
:1013680002F00F0E02F47F42A3F892212B460126C9
:10137800924D21F001002844B0F88401002818BFDC
:10138800002611F0010F03D0C0B24340082002E04C
:1013980083EA1023FAE713F4004F18BF83F4C0530D
:1013A80001384FEA4303F6D101311029E0D142EA6E
:1013B8000E02A5F8922126B9C3F303339E4500F027
:1013C80024827E4B93F89431002B41F09280BB69C4
:1013D8007B4E43F01003BB6102234FF400558DF898
:1013E8004F303046102313A98DF84E30ADF84C50CD
:1013F8000EF05AFE4FF48043ADF82C3030460423EB
:101408000BA98DF82E300EF04FFE6E4B35611A6821
:101418001AB10F2009F06AF901E06B4A1A606B4BA8
:1014280001275A69002522F470625A615A6913A883
:1014380042F400725A614FF48043139308238DF8E5
:1014480051308DF850508DF852700EF0DFFA282385
:101458000DEB03004FF003088DF828308DF8298034
:101468008DF82A508DF82B7010F078FF142009F0B1
:10147800D0F87720D0213A460BAB10F0F1FA0028CB
:1014880000F0B2809DF82C304C4D552B85F8AF31CB
:10149800A5F8B88140F0A880D1213A460BAB772057
:1014A80010F0DEFA9DF82C30772003F00F021B09AC
:1014B80085F8B02185F8B131162213ABAA2110F0B6
:1014C800CFFA9DF84C209DF84D3043EA0223A5F849
:1014D80098319DF84E209DF84F3043EA0223A5F835
:1014E8009A319DF850209DF8513043EA0223A5F81F
:1014F8009C319DF852209DF8533043EA0223A5F809
:101508009E319DF854209DF8553043EA0223A5F8F2
:10151800A0319DF856209DF8573043EA0223A5F8DC
:10152800A2319DF858209DF8593043EA0223A5F8C6
:10153800A4319DF85A209DF85B3043EA0223A5F8B0
:10154800A6319DF85C209DF85D3043EA0223A5F89A
:10155800A8319DF85E209DF85F3043EA0223A5F884
:10156800AA319DF860209DF8613043EA022341F2D8
:101578007072A5F8AC31164B85F894711A8046F64E
:1015880078125A80134A5A60134A9A60134ADA60EA
:10159800134A1A61134A5A6100F0ABBF442D002068
:1015A800202D002039620008C5660008296200085D
:1015B800CD650008BDF20008D9F20008D800002067
:1015C80000100140841F0020016200080000014053
:1015D800700600208D6200088163000869620008B7
:1015E8003563000825610008944A136823F4804392
:1015F8001360934B934A1968914204BF00221A6002
:101608004FF400537361904D95F8BC61002E40F083
:101618000E81142008F0FDFF05F2BD137620D021BD
:10162800012210F01DFA95F8BD31582B29D105F586
:10163800E07388211822762010F012FA31227620E1
:10164800F42110F04DFA0123804A85F8BC31804B13
:101658009A60804A1E805A6045F6D8125A807E4A9F
:10166800DA607E4A1A617E4A5A61E0E0B8F1010FF9
:1016780007D07C4B7C4A83F80280136843F004034C
:101688001360794D2B689E0702D5784B1B689847E5
:10169800039BE4B26C4E764A4BB32B684CB940F2CC
:1016A800596113F0020F40F2712318BF0B467D21D8
:1016B80008E09C0759BF4FF47A7319464FF4FA6350
:1016C8004FF47A719B4505DBBBF57A6FA8BF4FF4E1
:1016D8007A6B00E09B464B1E5B44B3FBF1F3013B86
:1016E800DBB203FB011186F88031116005E09DF83B
:1016F8000C30C2F800B086F880315E4FB8463B68BF
:101708009847049C5C4F0023022C3B7004D0032CA8
:1017180019D0002C40F08E8000221EAB03F82C2D2F
:10172800C6F8DC211E200A21012210F099F950B1D7
:101738009DF84C30482B06D1504B514A1A60514AFB
:101748005A600223BEE04FF0000A1EAB03F82CAD2E
:101758000C205146012210F083F9002800F0CD86B4
:101768009DF84C30482B06D1444B474A1A60474AEB
:101778005A600323A6E0504600F0BFBE9DF94C30E6
:1017880001337FF4DBAC0023138005F003F8394BF9
:1017980060B92BE00025A5E40125A3E40225A1E416
:1017A80003259FE404259DE405259BE4384ABB2CCA
:1017B8001A60384A5A60384ADA60384A1A61384B2F
:1017C80001D901220EE0612C01D902220AE0292C5C
:1017D80001D9032206E0132C01D9042202E0092CC6
:1017E80002D905225A70BAE40622FBE72D4A1A608C
:1017F8002D4A5A602D4A9A600823B1E41A4A6B7040
:10180800136843F0020313606DE542F21072104B47
:101818004FF003081A805A80254A5A60254A9A6070
:10182800254ADA60254A1A61254A5A6121E74FF0AC
:1018380004081EE7012C4BD91C4663E7000401404D
:10184800841F002001620008D800002021610008E0
:1018580070060020236100085F620008E962000842
:10186800BD5E00085C000020F8180020202D002034
:10187800B82D0020EC200020803100204C060020EC
:101888001501010885FD000885FE0008F9FD00081E
:1018980029660008916500086D65000890C1793DCA
:1018A80000000020C1F20008E1F20008BFF20008C1
:1018B80055620008D96200084B620008C962000836
:1018C800015D00081C4AD3702B6843F008032B60A5
:1018D8001A4C94F858310BB1194A137094F85931CD
:1018E8000BB1184A137094F85A3103B13B702B6846
:1018F800DFF85CA013F0080F2CD0BDF914204FF0CE
:10190800640B92FBFBF73846049212F025F8049A10
:1019180003900BFB172000B212F01EF80A4912F0D0
:101928006FF8039B0146184611F062FF074912F051
:1019380067F8CAF8000010E05C00002008110020D9
:1019480000210020833100208988883C0000204144
:101958007C1F00200023CAF80030B74A0A271378F2
:1019680043F002031370B54B10225A6108221A6122
:10197800DFF8C8A21920DAF80C30013F83F0100311
:10198800CAF80C30DAF80C3083F00803CAF80C30C7
:1019980008F03FFE012008F055FE192008F039FE36
:1019A800002008F04FFE17F0FF07E1D108231027A9
:1019B800CAF81030CAF810702B68180709D5A04B60
:1019C800CAF814701B6898479E4B0122CAF8107019
:1019D8001A709D4B9D4F1B68187B11F0BDFF9C49E9
:1019E80012F00EF807F034FB8246388811F0B4FF85
:1019F800514612F005F815F055FD964B18803888B9
:101A080011F0AAFF0146944812F0AEF8934912F07B
:101A1800ABF8934B8E491860D8F8100011F0F0FF1E
:101A2800904911F0EDFF904F904BFF2118601B2259
:101A3800384615F02AFB00223A702A688C4B01219F
:101A480012F0020F19701FBF79700321197002215B
:101A580018BFB970510748BF1978384641BF4D1CA7
:101A68001D7003257D5412F00A0F0CD01A7804213A
:101A7800B954511CC9B205257D54D11C02321970C4
:101A8800D2B20621B9547B4D29688F0641BF1A7816
:101A9800571C1F70072748BF87540A0608D51A78AD
:101AA80009278754971C01321F70D2B20A2787541E
:101AB8006779082F01D00E2F08D11A7802F1010E8C
:101AC80083F800E04FF00B0E00F802E01A7811F4EA
:101AD800803F4FF00C0C00F802C002F1010E1CBF51
:101AE800DFF88CC102325FFA8EFE83F800E01FBF78
:101AF8008CF800205C4A4FF00E0C02F80EC04A0722
:101B080048BF1A784FF0120C41BF02F1010E83F85A
:101B180000E04FF0100E00F802E01A7811F4806F20
:101B280002F1010E5FFA8EFE83F800E000F802C0B1
:101B38000ED094F818C2BCF1000F09D0DFF830C1FC
:101B480002328CF80020484A4FF0130C02F80EC0FD
:101B58001A7811F4007F4FF0140C00F802C002F15B
:101B6800010E1CBFDFF808C102325FFA8EFE83F84F
:101B780000E01FBF8CF800203B4A4FF0150C02F81C
:101B88000EC0182F13D11A784FF0160E00F802E085
:101B980002F1010E5FFA8EFE4FF0170C00F80EC02E
:101BA80002F1030E0232D2B283F800E087540A032E
:101BB80041BF1A78571C1F70192748BF8754CF0593
:101BC80041BF1A78511C19701A2348BF8354002149
:101BD8009822294815F059FA0DF00BFC274A284B92
:101BE800B4F852111A60274BB4F8980119802649A5
:101BF80000230B808B7025490A6081B2244A22F8A1
:101C080013100133122BF9D12B68D9045CBFB4F837
:101C18009E1111801B0740F1F28094F89231062B37
:101C280000F2E780DFE803F004363D6883A2A200F3
:101C380045F2F05230E000BF58310020000C01405E
:101C48004C0600206406002094210020200000207B
:101C580035FA8E3CB02100200AE81C4100401C46A1
:101C680088070020BD37863501100020902100200C
:101C780000100020542D0020D829002092120020A6
:101C8800DC0E0020E00E0020C42F00204C31002084
:101C9800902D002042F6F8227E4B1A800DF032FC7F
:101CA800A6E042F6F8227B4B1A8011F055FE7A49DD
:101CB80011F0A6FE794911F099FD12F08DF8002374
:101CC800774A42F823000133122BF9D1754A764935
:101CD80040201160754A137008F016FB002800F0C8
:101CE800888001234FF0070A90F9000040218DE811
:101CF80008046F4A6F4B76E042F6F822654B4020A5
:101D08001A806D4A674B1A60684B10221A7008F0E7
:101D1800FBFA00286DD001234FF0000890F900006D
:101D280040218DE80801654A4FF4E1335BE042F653
:101D3800F822584B40201A80614A5A4B1A605B4B74
:101D480008221A7008F0E0FA002852D001234FF058
:101D5800000C90F9000040218DE80810594A4FF412
:101D6800E13308F0AFF9C6F8E0013EE042F6F821A9
:101D7800484A062B11804D494FF00C02DFF884C108
:101D8800DFF884E1504F514C51480A700ED00023BF
:101D98008CF800308EF800303B701B2323704D4BBD
:101DA800027005221A704FF4E1340BE000218CF820
:101DB80000108EF80010397002702121454A2170F8
:101DC800454C1370454A374B40201A6008F09CFA7E
:101DD80078B101234FF0000E90F900008DE808401B
:101DE80023463F4A402108F06DF9003018BF012012
:101DF80028B9082007F01EFA3A4A2A4B1A602B68BD
:101E08002A4A13F4804F1FBF08211170364825490C
:101E180018BF086042F20101194099B144F62060E8
:101E28001C499F04088041BF082111702F481D4993
:101E380048BF0860DC0741BF0C2111702C481949C4
:101E480048BF086011781806A1F10401517040F1EB
:101E58009280284F284CC6F8E47100263146152296
:101E68002648DFF8A88066706660A660053F15F012
:101E78000CF93046C8F800700AF0FBFF204B02202E
:101E88001B68E36008F040FA002841D1802007F081
:101E9800D1F968E0E8070020CDCCCC3F0000B04481
:101EA8005C3000203400002079340108742A0020B6
:101EB8001D360108A0860100653401087135010846
:101EC8005134010825350108B0290020D329002004
:101ED80047310020D429002090D00300C3F2000825
:101EE800E9F20008D5340108A9340108C53401080D
:101EF800B5340108FC120020A4070020C00200200D
:101F0800782D002048310020B1290020C407002086
:101F180046796378C5490C2202FB03125278B24213
:101F280004D00133DBB2042BF4D900236370D8F852
:101F3800003062781B7890F90000002B4FF00C03FA
:101F480003FB021314BF0326012600225B780096C8
:101F58000192022108F0B6F8B54B1860002895D018
:101F680001200AF086FFB34B1868B34B00F5C57221
:101F78001A600BF025F82B6813AE13F4007F65D0B8
:101F8800AE4AAF4C029B102723609369AD4843F0DB
:101F980001039361029B0AA91B888DF82A70ADF88A
:101FA800283002238DF82B300EF07EF82368A548E0
:101FB8005B880AA9ADF8283004238DF82A300EF082
:101FC80073F8D4F800E00F219EF808304FF00108AC
:101FD80003F0030203F0FC0303F1804303F58033AD
:101FE80098689200914020EA01019960996808FA7E
:101FF80002F20A439A60DEF80430934A4FF0000A6E
:102008005361304613938DF850A08DF851708DF8B8
:1020180052800DF0FBFC23680BA85B7A8DF82EA08C
:102028008DF82C3003238DF82D308DF82F8010F08B
:1020380095F9864B864A1B683C3B1360854A1368B2
:102048003B431360844B4FF0FF321A60834B844A42
:10205800844C1360844A803313602B680027D903AB
:10206800277040F1B5800EF0A5FB40F22A3CDFF85E
:102078002CB2DFF8C8A14FF001086246584639462D
:10208800CDF808C084F8008014F0FFFFDAF81830A3
:10209800764843F00403CAF818304023ADF82830D6
:1020A80018238DF82B300AA903238DF82A300DF058
:1020B800DDFCDAF81C306E4943F00203CAF81C3024
:1020C8006C4B6D4C1B68AAF6947AB3FBF1F321882C
:1020D800013B21F45C710904090C21809BB21D218C
:1020E800A1852385A4F81480238C23F001031B0405
:1020F8001B0C2384238CA088218B23F0020321F05E
:10210800730109041B04090C1B0C41F0600180B227
:1021180043EA0803A0802183A7862384238B23F026
:1021280008031B041B0C43F008032383B4F8443052
:102138006FEA43436FEA53439BB2A4F84430DAF89A
:10214800A83F43EA0803CAF8A83F50460DF072FAC0
:102158004A4BDDF808C01393802318934FF480731B
:10216800CDF850B019934FF0100B4FF40053504670
:1021780031461C9317971A971B971D97CDF854B0A3
:10218800CDF858C00DF038FAA3890BA89BB243F4D8
:102198000073A381DAF8003043F00203CAF8003074
:1021A8008DF82CB08DF82D808DF82E708DF82F803D
:1021B80010F0D4F8324B1A68324B43F8292009F151
:1021C8000109B9F1200FF5D10DF090FE0DF08EFE4A
:1021D8002B685A0540F193802B4C2C4BD4F828855A
:1021E8000420C3F8008008F08FF80421C4F82C05F7
:1021F80008F066F8264B84F830050820C3F80080FC
:1022080008F082F8234B0821186008F059F8224F8B
:1022180084F83105002138462C2214F036FF8E232D
:102228007B704FF07C0AE0233AE000BF2497010856
:102238004429002038100020300F002000100240F0
:10224800A0070020000C014000040140782D002068
:102258009C070020F8180020581000203013002098
:10226800481F0020A90D00208829002000080140EF
:1022780000366E0160000020000400403404004075
:10228800B4960108AA0D0020D8000020EC18002000
:10229800441900209019002014190020D5020020AC
:1022A8004FF07D09FB7087F800A087F82B90964FB8
:1022B8002C220021384614F0E8FE8A237B70102077
:1022C800A023FB7087F800A087F82B90C4F834850A
:1022D80008F01AF81021C4F8380507F0F1FF84F85F
:1022E8003C052020C4F8408508F00EF82021C4F8E9
:1022F800440507F0E5FF84F848050BF087F9834AA1
:1023080000241388322023F040031B041B0C138085
:1023180013884FF4805723F038031B041B0C1380D9
:1023280013889BB243F0400313809F238DF82C3011
:102338008DF82D408DF82E408DF82F4008F069F962
:102348008DF84D40724C0422676130460BA910F09D
:1023580049F827619DF84E209DF84D30120242EA57
:1023680003429DF84F301A436A4B9A426A4B17D082
:1023780008D86A498A420CD001F51A4102318A42CA
:1023880009D01CE066498A4205D001318A4207D04B
:1023980015E0202200E080221A804FF4807202E0CB
:1023A8004FF480721A805A809A88198812029A60AB
:1023B8004A43DA605B4A012182F8491504E00022A9
:1023C8001A805A809A60DA60DC68FCB1240CA04656
:1023D8004FF00009A14512DA09EB04077F10380411
:1023E800314610220DF096FF002356F823200132C3
:1023F8005BD10133042BF8D1B8463C46EAE70AF032
:1024080091FF484B4FEA0842C3F84C252B68464ACF
:1024180013F4002318BF0123137008F0D3F8434BBB
:102428001860434B5A791946052A02BF414B4FF4AD
:10243800C8721A80404B4FF47A721A803F4BC822F8
:102448001A803F4A137843F0080313703D4A137803
:1024580023F00203137040F602032A6813406BB19D
:1024680039483A4B18603A4B03201870394B012011
:10247800187039480023038038480380930341BF0C
:10248800374B04221A71DA7844BF42F00102DA703D
:102498008B6801222B60334B1A70334A137863F030
:1024A8007F0313701FB0BDE8F08F07F101092746BD
:1024B800A3E72E4B00221A7000B211F04DFA2C49F6
:1024C80011F09EFA1390B5F95E0111F045FA28490A
:1024D80011F096FA1490B5F9600111F03DFA24490B
:1024E80011F08EFA2349159013A806F0BBFDFEF7EC
:1024F80063BD4FF00208FFF7BCB8012C7FF6E8A9CE
:1025080000243870FFF708B9491900200038004046
:10251800000C014018BA20001000002015202000EF
:102528001740EF00D8000020B42D00202C0E00200A
:10253800081100205C2100207A3100207831002029
:10254800FC1800208231002084120020E4180020AA
:102558004819002054000020D00F0020D20F00207E
:1025680048290020A80D0020583100203C000020F8
:1025780035FA8E3CB82A0020924A2DE9F04F1368AC
:10258800914C03F59C43914E20332360336889B006
:1025980013F4804F059205D111F0DAF810B92379B8
:1025A8000133237163792BB103F1FF38864B83F82C
:1025B8000580DFE09846864B5FFA88F51F78DFF8DC
:1025C8003092AF4231D9D9F80030072D98BF595D04
:1025D800804B88BF29461B687D489847032D1ED825
:1025E800D9F8002005F10E0302EB83039988DA88F5
:1025F800A8B14FF47A73401A5843531A90FBF3F07A
:1026080040F6C90300F57A70984205DC40F2EE23E3
:102618009842B8BF184601E040F6CA0080B204EB01
:102628004505E88008F10108C5E794F8048003250A
:10263800B8FBF5F50F2384F82A3094F82B3005EB16
:102648004505019394F82C30C5EB08050393D9F898
:102658000030DFF8A4A10293EBB204930025BD4239
:1026680055DA5D4B4FEA450933F815B0019B53B96C
:1026780011F06EF828B1039B002B08BF4FF0000B38
:1026880001E0DDF804B0029B988A584502D8D88A40
:1026980058450ED2E8B211F031F8032D8346DFBF5A
:1026A80094F82AE00120A8402EEA0000D8BF84F858
:1026B8002A0011F04DF818B1484829F800B022E076
:1026C800049B94F876002AF813B030B9B8F1020FD9
:1026D80015D93D4B012083F87600BAF80000BAF806
:1026E80002300344BAF8040003443D489BB229F879
:1026F80000301BB2032093FBF0F39BB200E05B4673
:10270800364829F8003001350AF1060AA7E794F897
:102718002A203448A2F10F014A424A4184F8902005
:10272800314B6AB1314A1268520109D40268D9683A
:102738009A60521AC82A1DD9012283F8212019E06B
:1027480002689868DA605B68121A9A4288BF264B5A
:102758004FF0000184F82B1088BF83F82110002562
:10276800BD4207DAE8B210F0C9FF1C4B23F8150088
:102778000135F5E73368DD0405D51C4B1B68D80720
:1027880001D410F043FA059B1F68194B1A68907A18
:10279800A0B31249137B013831F810001BB1C0F502
:1027A8003B60083080B200B2A0F57A70B0F57A7F4D
:1027B800A8BF4FF47A7020EAE07011F0CDF80D4907
:1027C80051E000BF60310020300E0020542D002061
:1027D800742A002034000020360E0020902D00209E
:1027E800A80E0020782D0020C42F0020FC0F002008
:1027F8004C31002000007A445E0E00203368190432
:102808003AD5D4F89430934DFB1A002B34DB07F5F6
:102818009C432033C5F894308F4BD27A59798F4B2B
:1028280033F8113095F898109BB293FBF2F301310D
:1028380001F00F0285F898202A4482F8993003465F
:10284800874A825C0130134410289BB2F8D11BB22E
:1028580093FBF0F000B26428A8BF642020EAE0707F
:1028680011F07AF87F4911F07FF97F4911F0C8F823
:1028780011F0B2FA7D4B188033687D4D13F4807FD8
:1028880000F00F817B4BDFF8F0919F4205D999F852
:10289800022012B9012289F8022099F80220002AA0
:1028A80000F0FF80744A95F8008092F82170C8F310
:1028B80080087A1E57425741704A002F9246116885
:1028C80018BF4FF0000BC1F38063019308BF4FF0AE
:1028D800030B99F82020052A00F2DD80DFE802F0DA
:1028E800034E537988A5B8F1000F3AD0D4F8AC005C
:1028F800B4F8B01007F0A5FD012809D16049614A74
:1029080009681268C988642000FB0122C9F81020F0
:10291800019B6BB15A4A126812794AB110F062FDF4
:10292800032289F820204FF47A72C9F81C20D0E7D6
:10293800002F40F0B080534AD9F8101010684E4A62
:1029480088420AD9029210F04DFD029A032182F8BA
:10295800201040F6B831D161BBE7012182F8201080
:10296800B7E7019B4FF4806013B106F053FC01E018
:1029780006F03FFC0022C9F810208CE0002F49D156
:1029880010F030FDA5E727B1052289F820200120A5
:1029980000E03846B8F1000F0CD0D4F8AC204FF066
:1029A800020BD189384A11805180918034490968D5
:1029B8004988D180334A1168D9F81420914202D845
:1029C800B8F1000F64D147F23052C9F81C20032235
:1029D80021E02A7842F002022A7010F017F9294AF9
:1029E800D9F81C1012680A44C9F81820042212E009
:1029F800244A9FB11168D9F8182091424BD9234A2B
:102A080012781AB9DAF80020D30744D42A7822F0C9
:102A180002022A70052289F820205AE71268D9F89C
:102A28001C100A44C9F8182035E01549154A0968E8
:102A38001268C988642000FB01224FF48060C9F83D
:102A48001020002289F8202089F8032006F0D1FB05
:102A58003FE700BF300E0020DC2A0020EC2A0020CF
:102A6800C90E00200000C84200C07F445C1000204E
:102A780082310020404B4C00C42F0020FC0F002066
:102A8800E82F0020782D0020902D00200C00002039
:102A980000287FF41EAFBBF1000F02D0584607F0A4
:102AA800EBFD924F07F5C570B7F8521107F0C9FC56
:102AB8000197834668B910F087FC8D4B0022C3F854
:102AC80000B0C3F804B0C3F808B08A4B1A605A6063
:102AD8009A602B785F0736D53368D80633D5864B8E
:102AE8001B78D9062FD4854B1B789BB1019B93F893
:102AF800E231BBF1000F15D17BB1814B1A68D4F8D4
:102B0800B4309B1A002B08DA10F080F87D4B83F85C
:102B1800B8B018E0BBF1000F0DD1102007F0ACFDE4
:102B280001230EE03BB1764A4FF47A71126801FB3B
:102B38000323C4F8B43094F8B83023B107F088FD03
:102B4800002384F8B830019B93F8E0A193F8E111D1
:102B5800B3F89AE1B3F89CC1002318466A4F80087D
:102B680037F9132001337245C4BF60F07F00C0B24B
:102B78006245B8BF40F04000042BB946EED194F846
:102B8800B930604A834205D192F8BA30F92B04D89B
:102B9800013300E0002382F8BA30584B84F8B900BA
:102BA8001A785A4F9846E2B93B68DA0708D5BBF15C
:102BB800000F16D12B78DB0713D50FF079FE10E044
:102BC8002B7858070DD54F4B93F82B304BB1504B02
:102BD800DB7833B911B110F019F802E0BBF1000F3E
:102BE800F9D094F8BA30474A142BDFF840B140F0D6
:102BF800AF8098F800301AF1000A18BF4FF0010AA8
:102C08006BB392F8B9305F2B11D12B7803F0040322
:102C180003F0FF0113B10FF0F9FF08E00B20039157
:102C2800029207F029FD029A039982F8BA10BAF1C4
:102C3800000F14D094F8B9307D2B10D12B7803F005
:102C4800040303F0FF0213B10FF0E0FF07E00B20CD
:102C5800029207F011FD2B4B029A83F8BA202B78C9
:102C680003F0040303F0FF01002B71D194F8B9308D
:102C7800244A572B15D1274B4FF47A721A803368A0
:102C8800190601D50AF0ECF9234B1B685A0742BF15
:102C9800224A0A21118013F0080359D1204A1380CF
:102CA80056E03068400716D55A2B14D11D4B1878BA
:102CB80020B119701C4B01221A7049E092F8BB3000
:102CC80083F0010382F8BB300BB10C2000E00D202B
:102CD80007F0D2FC3CE05D2B00F01F855B2B00F079
:102CE8001E855E2B24D1032000F01ABD0811002098
:102CF80018220020CC220020FC1800200C00002004
:102D0800782D0020300E0020902D0020FC0F002090
:102D1800C42F00207A310020F818002078310020D4
:102D2800F8100020892100208A2100203810002076
:102D3800562B01D106F02AFD98F80030002B00F040
:102D4800058594F8B9306F2B40F0FA840FF0B0FD88
:102D58003368580732D594F8BB30A3B12B7859079C
:102D680011D5019BB9F90620B3F89A319A420ADDC8
:102D78003B6813F0010301BFAC4A32211180AC4A11
:102D880008BF82F8BB303B68DA030AD5A94B1A782A
:102D98002AB9A94A127812B9A44A3221118001220B
:102DA8000BE0A54A13784BB12B7803F0040303F02A
:102DB800FF011BB9A14B117001221A70DBF80090BA
:102DC80000233B6009F17B0809F1CB0A98F8002041
:102DD80098F8013018F8010C9A420BD2414607F0D6
:102DE800FBFA38B118F8022C012303FA02F23B6807
:102DF80013433B6008F10408D045E7D1904B1B789A
:102E080053B1904B904F1A68984612F0020FDFF8B2
:102E1800509240F03A8332E309F1CA0709F58978FC
:102E28003A787B7817F8010C9A4225D2394607F090
:102E3800D3FA08B397F804E00C21BB7801FB0E41E4
:102E4800824A013B03EB43031344D1F8C02097F8AF
:102E580003909A4276480FD0C1F8C030002390F80A
:102E6800EC20C1F8C430012303FA0EF322EA03036D
:102E780081F8BC9080F8EC3006374745D0D1744BC8
:102E8800DFF8E0A1D3F80080724B4FF0000B1B680D
:102E9800029394F82B300393DAF80030002B00F0FB
:102EA800E58293F80090B9F1000F00F0DF82DAF8BC
:102EB800042002998A1A002A0CDB01F5FA72CAF872
:102EC800042094F8EC10012202FA0BF221EA020223
:102ED80084F8EC20039A002A00F0C8821AF8042C1F
:102EE80059780432D2B2002940F081825A4931F926
:102EF80012105A4AB2F8982102F1C800814201DD45
:102F08009F7814E0C83A914202DA99784F420EE06D
:102F180094F8EC20012303FA0BF322EA030384F864
:102F2800EC30029B03F5FA73CAF804309EE294F879
:102F3800EC3043FA0BF3DB0700F19882002FCCBF8B
:102F48000220012007F0BAFB09F1FF32384B132A9F
:102F580000F28482DFE812F01400230032004400FB
:102F680061008800ED005201B701EC011B028202EA
:102F7800440055008800ED005201BF00240189017A
:102F880098F8001040460F44FA2FA8BFFA2727EAFE
:102F9800E77788F8007007F005FA01201EE098F836
:102FA800011040460F44642FA8BF642727EAE7773B
:102FB80088F8017007F0F6F902200FE098F803107E
:102FC80040460F44642FA8BF642727EAE77788F8AC
:102FD8000370D3F8F01007F09DF903203946D3E1C8
:102FE80098F805100D2039446429A8BF642121EA06
:102FF800E17188F8051007F0D1FAB9F10D0F00F06A
:103008002D8298F804100E2039446429A8BF642141
:1030180021EAE17188F80410B6E198F80610052055
:10302800394481F3080188F80610ADE170210020C9
:10303800300E002088210020892100208A210020CC
:1030480084310020FC0F0020F81800201C9B010888
:1030580060100020782D0020902D002008110020FD
:10306800C0190020F00E0020D3F8F4301A78022A94
:1030780022D13846049310F06FFCA94910F074FD72
:10308800049B596A059310F0B3FB0021049010F0DB
:1030980055FE059B48B9049AA249104610F06CFEEB
:1030A800049A059B10B19F4A00E000225A620F2043
:1030B800114607F05FFA0AE099780F203944C829C9
:1030C800A8BFC82121EAE171997007F067FAB9F140
:1030D8000F0F00F0C381944BD3F8F49099F80030A7
:1030E800022B1AD1384610F037FC8D4910F03CFD00
:1030F800D9F8201010F07CFB0021074610F01EFEC6
:1031080030B93846874910F037FE10B1854F00E0D6
:103118000027C9F82070122059E199F801101220EF
:103128003944C829A8BFC82121EAE17189F80110EA
:103138002AE1D3F8F4301A78022A22D138460493C7
:1031480010F00AFC774910F00FFD049B196B0593EA
:1031580010F04EFB0021049010F0F0FD059B48B9DB
:10316800049A7049104610F007FE049A059B10B1A6
:103178006C4A00E000221A631020114607F0FAF9A1
:103188000AE0197B10203944C829A8BFC82121EAC0
:10319800E171197307F002FAB9F1100F00F05E81BE
:1031A800614BD3F8F49099F80030022B1AD13846C5
:1031B80010F0D2FB5B4910F0D7FCD9F82C1010F0B6
:1031C80017FB0021074610F0B9FD30B938465549BC
:1031D80010F0D2FD10B1534F00E00027C9F82C7051
:1031E8001320F4E099F80B1013203944C829A8BF1C
:1031F800C82121EAE17189F80B10C5E0D3F8F43051
:103208001A78022A22D13846049310F0A5FB4749C0
:1032180010F0AAFC049BD96B059310F0E9FA002181
:10322800049010F08BFD059B48B9049A3D4910465F
:1032380010F0A2FD049A059B10B13A4A00E0002262
:10324800DA631120114607F095F90AE0997D1120FB
:103258003944C829A8BFC82121EAE171997507F046
:103268009DF9B9F1110F00F0F9802F4BD3F8F490C4
:1032780099F80030022B1AD1384610F06DFB2B4913
:1032880010F072FCD9F8381010F0B2FA0021074695
:1032980010F054FD30B93846224910F06DFD10B1D8
:1032A800204F00E00027C9F8387014208FE099F803
:1032B800151014203944C829A8BFC82121EAE17192
:1032C80089F8151060E0D3F8F49099F80030022BD3
:1032D8001AD1384610F040FB114910F045FCD9F8D6
:1032E800281010F085FA0021074610F027FD30B9A4
:1032F80038460C4910F040FD10B10A4F00E0002795
:10330800C9F82870092062E099F8031009203944A7
:10331800C829A8BFC82121EAE17189F8031033E060
:10332800000020410000C842300E002000007A440E
:10333800D3F8F49099F80030022B1AD1384610F0DF
:103348000BFBB44910F010FCD9F8341010F050FA07
:103358000021074610F0F2FC30B93846AD4910F0AC
:103368000BFD10B1AB4F00E00027C9F834700A20FC
:103378002DE099F80D100A203944C829A8BFC821A2
:1033880021EAE17189F80D1007F008F966E0D3F831
:10339800F49099F80030022B1DD1384610F0DCFA71
:1033A8009D4910F0E1FBD9F8401010F021FA0021F6
:1033B800074610F0C3FC30B93846964910F0DCFCDB
:1033C80010B1944F00E00027C9F840700B2039462F
:1033D80007F0D0F842E099F817100B203944C829B3
:1033E800A8BFC82121EAE17189F81710CCE70129A3
:1033F80034D19878894B33F91230B3F5617F05DB06
:1034080040F633029342A8BF134601E04FF46173BC
:10341800B9F10C0F22D14FF4966292FBF0F0A3F5AC
:10342800617393FBF0F37E4ADFB21378BB4215D089
:10343800042F34BF3B4602231370019A09FB032370
:10344800784A03F2B27313600DF08BFD4846394693
:1034580007F0A4F8781CC0B207F030F994F8EC2013
:10346800012303FA0BF3134384F8EC300BF1010B3F
:10347800BBF1040F0AF10C0A7FF40EADC1E4336806
:10348800D80510D5684BDB786BB13B6899070AD52E
:10349800B9F8003013F0010A0AD10FF095FF0120A6
:1034A80005F0B8FE04E0012005F0A3FE012300E0CA
:1034B8000023D8F8002052070DD563B1012005F08C
:1034C80098FEB9F800309B0708D40FF07DFF022062
:1034D80005F0A0FE02E0022005F08BFEB9F80030EE
:1034E800524A13F0030F4FF0100114BF51611161DC
:1034F8003A6812F00A0F27D0D8F80020D00609D56C
:1035080059070AD4042005F085FE494B1B88A4F806
:10351800F83002E0042005F06CFED8F800309A0676
:1035280007D5B9F800305B0606D4402005F072FED6
:1035380002E0402005F05DFED8F80030580642BF92
:103548003B4B1B88A4F8FA303B68990609D4D8F895
:1035580000301A0540F1B0804FF4807005F05AFE33
:10356800AEE0344B1B789B076ED5334B1B78042B8E
:103578006AD9D8F8003013F4007A0FD0B9F80030BF
:10358800DF063AD4102005F045FE202005F031FE74
:103598002A48011D09F0CEFC02232AE0B9F8007080
:1035A80007F01007BFB22FB1102005F022FE012747
:1035B80084F8FCA0D8F80030580512D5D4F80031AA
:1035C8001F495A89B1F90030002BB8BF5B429342BA
:1035D80007DAB1F90230002BB8BF5B429342C0F260
:1035E8000781B9F80030990608D5202005F001FEBA
:1035F800002384F8FC30012700E0002794F8043108
:103608009BBB0E2007F038F80E4B012283F80421EB
:103618002BE000BF0000C84200007A44902D002033
:10362800002D002060100020C42F0020000C014055
:10363800F8100020FC180020021900206810002053
:1036480000110020300E0020B9F8003003F03003DC
:10365800002B3FF47CAF102005F0CBFD202005F0B7
:10366800C8FD002384F8FC3002E0002F3FF46FAF60
:10367800002214466B4B002023F814006A4B191DD6
:1036880003F10A0721F814000021D151174478608A
:10369800B96023F8140003F132075A33D151D150DD
:1036A800174413447860B960586099601432002C4C
:1036B8007FF44DAF0124DDE74FF4807005F099FDEC
:1036C8005A4B5A791C46082A01D00E2A02D14020AA
:1036D80005F08FFD33685A0540F1A08094F8183240
:1036E8001BB92B7813F0040F03E0D8F8003013F45B
:1036F800002F0BD04E4B00221A703C200BF04AFFD3
:10370800002800F08B800EF02FFBF6E709F07EFF13
:1037180009B0BDE8F04F0BF06CBE012000E00220BC
:103728005FFA80F8019A08F1FF3382F8B03705F0A4
:10373800B3FD05F05DFE404606F0C0FFFFF708BB8D
:10374800BAF1000F02D07E2B3FF400AB94F8B930E9
:10375800972B05D1374B4FF4C8721A80FFF7F8BA88
:10376800A72B06D1344A137843F004031370FFF7EC
:10377800EFBA0022BB2B079201D1022303E0B72B3B
:1037880004D14FF6FE73ADF81E3009E0BE2B01D10F
:10379800022303E0BD2B1AD14FF6FE73ADF81C309F
:1037A800DBF80030BDF81C10B3F858200A44A3F821
:1037B8005820BDF81E10B3F85A200A44A3F85A201E
:1037C80005F0E4FF002384F8BA30FFF7C1BA792B7B
:1037D80004D11A4AD37823F0010306E07A2B7FF448
:1037E800B7AA164AD37843F00103D370FFF7B0BAEB
:1037F800B9F800309B063FF501AF202005F00AFD1F
:103808000F4B10481A685B68011D4360026009F09D
:1038180091FB0D4B012783F8FC70EFE609B0BDE87A
:10382800F08F00BF7C310020360F002008110020E7
:10383800792A00205C210020FC180020482900205B
:103848000419002070100020300E0020B54B2DE91F
:10385800F04FB3F90610B44B85B01F6801937A890D
:1038680091420EDBB1F5FA6FFC79BFBF8B1A634347
:10387800A2F5FA6493FBF4F4ACBFC4F164046434B5
:1038880000E06424A94BAA4AB3F898B193F96231CD
:1038980012689BB2029215460393002240F2E6306A
:1038A800A04B4FEA420C33F912E0CBEB0E0303F2C4
:1038B800F316864203D8002BB8BF5B4201E04FF4F1
:1038C800FA73022A2ED0029E96F811611EB1B342F5
:1038D800CCBF9B1B0023642093FBF0F8954E6FF040
:1038E800630A36F818900AFB083A08F1010836F915
:1038F80018600FFA89F8C8EB060606FB0AF696FB6D
:10390800F0F68D484E4420F80C60BE1836796420D5
:1039180073438A4E93FBF6F364339BB2634393FB82
:10392800F0F02CE0029890F812611EB1B342CCBFBF
:103938009B1B0023642093FBF0F0DFF82C926FF0C0
:10394800630808FB003A39F91060013039F91000B2
:10395800002BA0EB060000FB0AFA9AFBF8FA039882
:10396800C6EB0A0A0AFB00FA7348B8BF5B42A0F824
:1039780004A0B8794343714893FBF0F064306B7846
:103988004FF06408434393FBF8F36D4E022AB35497
:10399800EB7A6C4E00FB03F393FBF8F3B3546B7DA7
:1039A800654E00FB03F090FBF8F0674B9854674BAB
:1039B8000ED1DE4583F802800DDB5C4CB4F89A2109
:1039C800914214DBB1F5FA6FA8BF4FF4FA610FE02A
:1039D800DE459C5404DA36F80C305B4226F80C308D
:1039E8000132032A05F101057FF458AFE5E71146D6
:1039F800891A4FF47A735943C2F5FA62B1FBF2F1AE
:103A0800642391FBF3F2DFF874E16FF063073EF88B
:103A1800120007FB021101323EF9122007B2D21B35
:103A2800514391FBF3F30344F380494B424D1B8808
:103A38005F063BD5474A484B10881B88181A00B2C6
:103A48000FF08AFF45490FF0DBFF074605F000FB42
:103A58008046384605F089FA0746B5F902000FF0A6
:103A68007BFF8146B5F900000FF076FF414682469C
:103A78000FF0C6FF3946834648460FF0C1FF01469E
:103A880058460FF0B3FE10F081F9414628804846A9
:103A98000FF0B6FF3946804650460FF0B1FF014699
:103AA80040460FF0A5FE10F071F968802C4D2B6888
:103AB800980740F19E8045F207212A4B2A4F1A6841
:103AC8007B69D31A8B4240F394807A610CF03CF9FD
:103AD800264BDFF8AC901A789846032AB9F80030DC
:103AE80050D10A2B58D90023282088F8003006F036
:103AF80090FD0CF029F91E4B18880CF00FF91D4B9E
:103B08001A68D37890FBF3F0013008281A4BA8BF45
:103B180008201870537980B243433B831379584384
:103B2800788339E0902D00206010002008110020D3
:103B380038100020661F0020001100200CFEFFFF37
:103B480094220020C60F0020AC220020F82100207B
:103B5800C01900202A0F0020F810002035FA8E3CEA
:103B6800542D002060310020B80F00204819002093
:103B7800F42A0020E4180020540000204E1F0020E2
:103B8800E81800200A2B07D803239C4A88F800303D
:103B9800002313703B837B8398F80030984A012BED
:103BA8000CD002D3022B1BD023E03A8BB9F800309B
:103BB8009A421EDD012388F800300FE0B9F80010A2
:103BC8007B8B8B4202DD022313700FE08D4B1B8B26
:103BD8000133994202DD002313700AE0082006E051
:103BE8007B8BB9F8002001339A42E3DC072006F00A
:103BF80043FD2D68290577D5834B824F1A68FB69E9
:103C0800C3EB020845F2072398456DDD7F4BB6F9F3
:103C180006B0D3F800904FF47A7099F80A30FA6138
:103C2800012B98FBF0F8B4F85211ABF57A7B784E7B
:103C380003D042D3022B20D041E0764B396A5A7B1D
:103C4800754B4FF0080E33F8122091FBFEF392B239
:103C5800C91A8B183B6293FBFEF3BA8440F6E44220
:103C68009BB25343B9F80820C2EB13335843B9F950
:103C7800063090FBF3F0306021E0684BB9F808A0FB
:103C88001B78C6F800A05A0719D5654806F0D9FB75
:103C980020B915F0100F18BF4FF0000B0BFB0BF3FA
:103CA800322293FBF2F3B9F906205B445A434FF4EE
:103CB8007A7392FBF3F3534400E0002333603368D4
:103CC800D7E90A0103FB08F84FF47A7398FBF3F875
:103CD80010EB080041EBE8710023C7E90A01514ADB
:103CE80010F09AF8504B1860504E3368DB0427D513
:103CF8002F0622D54E4B1B789D071ED54D4B1878A5
:103D080004281AD900224C4B0521D718951C4FF0CE
:103D18000A0E122AD154E9B287F801E004D0B0EBB8
:103D2800510F2A46EFD800E014215A18322002F821
:103D3800010CFF225A540F2000E00A2006F09CFCD8
:103D48003E4D2A68002A51D03D4B3E4F18683968CD
:103D5800984681424AD83C4BDFF8F8901978526867
:103D6800E1B94FF0010A83F800A0B9F80030D35C3C
:103D780023B3504606F066FC344B83F800A00FF0DE
:103D8800F3FCB9F80030CBB92B681B78053B5345D9
:103D980014D806F017FC2E4B18600FE04FF0000AFD
:103DA80083F800A0B9F80030D35C3BB1504606F068
:103DB80049FC264B83F800A00FF0D6FC2B68B9F815
:103DC80000205B6823499B5CFE2B02D100230B80FB
:103DD8000CE0FF2B02D106F03BFC07E0D8F800000E
:103DE8000A2505FB030301323B600A800B4D2B7843
:103DF800580733D5184B08225A616DE0540000204B
:103E080048190020B80F002060310020E418002075
:103E1800F0180020DC2A0020EC2A00208231002043
:103E280092120020407E0500F4180020FC0F0020AC
:103E3800FC180020021900202C2D0020941F0020BF
:103E4800782D00208C1F0020881F00205031002072
:103E5800702F0020901F0020000C01403268D1070D
:103E68005CBF43F001032B70984B1B781F075EBFA4
:103E78002B7823F001032B70D60248BF2B78944A85
:103E880044BF23F001032B70924B1B6813F0040FFF
:103E980002D09149098851B99049098809B1980710
:103EA80005D48F4B1B88003318BF012333B102237D
:103EB80013702B7823F001032B7004E02978C907CD
:103EC80058BF0223137006F07DFB864B1B68C01A8F
:103ED800002801DB0FF048FC09F098FB824B1E78A4
:103EE8009846002E00F0AB80804E3368002B00F01F
:103EF800F186306806F03CFC002800F0EB867B4B2E
:103F08007B4C186806F031FC092801D03F2850D1B5
:103F18004FF0000A5746D4F80090764DB9F1000FDB
:103F280005D0754829684A4613F0FCF810B9AA4626
:103F380007B92F46714B10359D42EFD3C7B1D7F85B
:103F480000E0DAF800C023681EF803501CF80300EC
:103F5800A8420DD15A1C684938B92D2B05D8644D93
:103F68002A602025CD54885402E0CD542260EAE727
:103F780023680BB1574511D061480DF0E5FF57454F
:103F880007D857F8100B0DF0DFFF09200DF0D4FF0C
:103F9800F5E75C480DF0D8FF4FF000092368994514
:103FA800A7D2554B13F809000DF0C6FF09F1010916
:103FB800F4E72368002B40F07286042840F0B086AE
:103FC8004D480AF0AFFC00F085BED9F80000DFF8D4
:103FD80044A106F0CDFB40B3DAF8000006F0C5FBBB
:103FE800DBF80030024693F84810002935D1242820
:103FF80040F09280012283F84820DBF80030DFF897
:1040080010A193F84820062ADFD193F8490000F060
:1040180013FF8146002800F0AA803B6898790DF0CC
:10402800E0FE3B68002283F84820374B93F8353090
:10403800002B40F022864C36982E00F04B86334BEE
:10404800F21892F84A100129F5D1314FF3583A6025
:10405800304ABB4613609146B7E7012904D14D2881
:1040680014BF00220222C6E7022904D13C2814BF4B
:1040780000220322BFE703290CD140284FF000019A
:1040880002D983F84810B8E758711971D971987135
:104098000422B0E7042906D1997983F849004A40F7
:1040A8009A710522A7E70529A7D158791979884275
:1040B800987906D950409871481C18710B441A72A7
:1040C8009BE790420CBF0622002294E7FC180020D0
:1040D80050310020F8180020783100205C210020A1
:1040E8007A31002054310020843100201C2D00201A
:1040F800842900207CA20108542900204CA401082E
:1041080037BD01083CBD0108B80F0020D8290020A0
:10411800A0190020A41900202B78B74958073FF5AB
:104128006CAF232ADAF8003014D1012088F8000097
:10413800B24803910360B24802920363B1480DF09C
:1041480003FFB1480DF000FF0399029A0B7843F082
:1041580002030B70AD4B1B681B78934201BFAC4A3E
:10416800AC4B1A60AC4A04BFAC4BDA6045E7DAF8EE
:10417800002092F849304A2B00F038815CD8332B64
:1041880000F0A18421D8292B00F03B8409D8252BE5
:1041980000F01284272B00F01684232B40F0BC85F6
:1041A8003FE22D2B00F03E8407D82B2B40F0B4853E
:1041B8000DF0FAFD607100F05BBD2F2B00F00B8550
:1041C800312B00F01D8500F0A7BD3E2B00F00481C7
:1041D8001DD8372B00F0C78404D8352B00F05A823D
:1041E80000F09ABD392B00F0FB833C2B40F09485FE
:1041F800DFF82C92D9F800A00DF0D6FD8AF800005F
:10420800D9F80030187807F0A9F800F031BD432B31
:1042180000F0868406D8412B40F07E854FF00009D7
:1042280000F056BC442B00F01F85482B40F07485E5
:1042380009F0B6F800F01CBDD02B00F0368368D822
:10424800CA2B00F0F5801CD84E2B00F00E8410D835
:104258004C2B40F061850DF0A7FD84F8D8010DF0D6
:10426800A3FD84F8D9010DF0A9FDA4F8DA0100F046
:10427800FFBCC82B00F08380C92B00F0378300F007
:104288004BBDCD2B00F01C8304D8CC2B00F02A8228
:1042980000F042BDCE2B00F01C83CF2B40F03C85B4
:1042A8000DF08CFD6FF4AF6283189BB2C62B98BFDC
:1042B800A4F898010DF082FDA4F844010DF07EFDEC
:1042C800A4F846010DF07AFDA4F848010DF076FD3A
:1042D800A4F8DA010DF068FD84F8EF010DF064FD33
:1042E8000DF062FD84F8F0010DF05EFD84F88701A1
:1042F8000DF05AFD84F894010DF056FD484BD3F8A3
:1043080000900DF05BFD00EB80004000A9F856001E
:1043180066E3D62B00F04E820AD8D22B19D0C0F013
:104328000C83D32B25D0D42B00F04F8200F0F4BCA3
:10433800EF2B41D005D8D82B40F0EE844FF0000980
:1043480002E1F22B00F08982FA2B00F0CB8200F018
:10435800E3BC2B78590700F18B840DF025FD02286A
:1043680084F8B00740F2A7822E4B002283F8B027CA
:10437800A1E20DF023FD2C4B188000F079BC92F8D7
:1043880005904FEA5909B9F1120F03D90BF0FEF85D
:1043980000F06EBC4FF0000ACA4507D20DF00EFDC2
:1043A800224B23F81A000AF1010AF5E7144B0122FF
:1043B80083F8342000F05CBCDFF86490D9F800A0E2
:1043C8000DF0FCFCAAF85A00D9F800900DF0F6FCA4
:1043D800A9F8580000F04CBC0DF0E6FC84F8E201A6
:1043E8000DF0E2FC84F8E10100F042BC0DF0E6FCBF
:1043F800A08100F03DBC00BF823100201C2D0020B0
:10440800B80F00206CBD01083CBD01087C2A0020C3
:10441800EFBEADDEF04F00200400FA0500ED00E02D
:104428003810002008110020280F0020902D0020AF
:10443800D64B1A689A461278022A6AD1DAF80030FE
:1044480009F1080B02930DF0AFFC0FF081FAD04987
:104458000FF08AFB029B43F82B00DAF800B00DF04E
:10446800A3FC09F10A030BEB830B0FF071FAC9499E
:104478000FF07AFBDAF80030CBF8040002930DF065
:1044880093FC0FF065FAC4490FF06EFB09F10E0BAF
:10449800029B09F10109B9F1030F43F82B00CDD1B3
:1044A800B9F1070FDAF800B01AD10DF07DFC0FF062
:1044B8004FFAB7490FF058FBCBF84400DAF800B0D0
:1044C8000DF072FC0FF044FAB1490FF04DFBCBF838
:1044D8004800DAF800B00DF067FC8BF84C0012E0E9
:1044E8000DF062FCCB448BF80100DAF800B00DF057
:1044F8005BFCCB448BF80B00DAF800B00DF054FCF1
:10450800CB448BF8150009F10109B9F10A0FC7D19D
:10451800AEE3DAF800B00DF047FCCB448BF80100AD
:10452800DAF800B00DF040FCCB448BF80B00DAF859
:1045380000B00DF039FCCB4409F10109B9F10A0FBB
:104548008BF81500E5D193E3DFF840A209F1080BD9
:10455800DAF8003002930DF031FC0FF0F9F98E49CA
:104568000FF002FB029B43F82B00DAF800B00DF0C5
:1045780025FC09F10A030BEB830B0FF0E9F98649D7
:104588000FF0F2FADAF80030CBF8040002930DF0DD
:1045980015FC0FF0DDF980490FF0E6FA09F10E0B72
:1045A800029B09F10109B9F1030F43F82B00CBD1A4
:1045B800B9F1070FDAF800B01AD10DF0FFFB0FF0D0
:1045C800C7F975490FF0D0FACBF84400DAF800B013
:1045D8000DF0F4FB0FF0BCF96F490FF0C5FACBF8FA
:1045E8004800DAF800B00DF0E9FB8BF84C0012E057
:1045F8000DF0E4FBCB448BF80100DAF800B00DF0C5
:10460800DDFBCB448BF80B00DAF800B00DF0D6FBDD
:10461800CB448BF8150009F10109B9F10A0FC7D18C
:1046280026E30DF0C1FB132883463FF6AFAEDFF853
:104638005CA1DAF800900DF0B7FB002357490C2273
:1046480002FB0312117A814220D1137809EB8B09FE
:1046580089F879300DF0A8FB89F87A000DF0A4FBF1
:1046680089F87B000DF0A0FB4D4A4E4B89F87C0081
:104678001A60DAF800004C4B00211860793005F018
:10468800CFFE4A4B80F001001870F1E201331C2B79
:10469800D4D17BE60DF088FB0B2882463FF676AE38
:1046A8003A4BD3F800900DF07FFB03283FF66EAE2F
:1046B800062303FB0A9989F8CE000DF075FB89F8EB
:1046C800C9000DF071FB89F8CA000DF06DFB89F87F
:1046D800CB000DF069FB89F8CC000DF065FB89F87B
:1046E800CD00C5E25379092B7FF650AE019BD3F874
:1046F80000900DF059FB019B89F80000D3F8009059
:104708000DF052FB89F801000DF04EFB019B642867
:104718001B68A8BF642018710DF046FB019B642834
:104728001B68A8BF642058710DF03EFB019BFF2851
:104738001B68A8BFFF2098710DF036FB019B642809
:10474800D3F8009028BF642089F807000DF02CFBEF
:10475800019B89F80200D3F800900DF025FB019B1E
:1047680089F80300D3F800900DF028FB3B68A9F8FE
:104778000A005B790A2B40F27B820D4BD3F800903C
:104788000DF012FB89F8080072E200BF3810002013
:10479800000020410000C84200007A44889B0108BC
:1047A8004C120020200F0020240F00200C000020B5
:1047B800601000200DF002FBCB4B23F8190009F123
:1047C8000109B9F1080FF5D152E253790F2B7FF4A3
:1047D800DDAD0DF0E9FA072881463FF6D7ADDFF8E1
:1047E80034A3DAF800B00DF0E9FA0E2303FB09F957
:1047F800CB44ABF81901DAF800B00DF0DFFACB447E
:10480800ABF81B01DAF800B00DF0D8FACB44ABF8DE
:104818001D01DAF800B00DF0C7FACB448BF81F0180
:10482800DAF800B00DF0C0FACB448BF82001DAF8C2
:1048380000B00DF0B9FACB448BF82101DAF800B0DA
:104848000DF0B2FACB448BF82201DAF800A00DF093
:10485800BFFAD144C9F823010AE20DF0A5FA0F28DE
:1048680081463FF693AD0DF09FFAC9EBC909A14403
:1048780089F8D4000DF098FA89F8D5000DF094FA6B
:1048880089F8D6000DF090FA89F8D7000DF08CFA67
:1048980089F8D8000DF088FA89F8D9000DF084FA63
:1048A80089F8DA0006F024F9E2E12B785B0700F1D9
:1048B800DF810CF09BFB04F0EFFC04F099FDD7E1DD
:1048C8002B78580700F1D481884B4FF4C8721A80AE
:1048D800CEE12B78590700F1CB81854A137843F054
:1048E800040328E02B785A07E5D515E20DF05CFAA9
:1048F8007F4B1A7810B142F0020201E022F0020266
:104908001A700DF051FA7B4BDFF80C9218700DF00D
:104918005FFAC9F800000DF05BFAC9F804000DF061
:104928004DFA754B18800DF049FA744B744A18808B
:10493800137843F0020313709AE10DF035FA0290F0
:104948000DF046FA83460DF043FA82460DF040FA20
:1049580081460DF033FA0DF031FA0DF025FA029B7D
:10496800A3B9684B1020C3F800B0C3F804A004F042
:1049780040FC5F4A137843F001031370B9F1000F4C
:1049880000F07681604BC3F8009071E1102B40F085
:104998006F815E4BC3F800B0C3F804A0B9F1000FF3
:1049A80002D0594BC3F800905848594B0222011DB8
:1049B8001A7008F0BFFA5BE1A0600DF009FAA3686D
:1049C8001843A06054E10DF0F9F9A4F85C010DF06A
:1049D800F5F9A4F85E010DF0F1F9A4F8600147E1DA
:1049E8000DF0E2F984F87C010DF0DEF984F880011D
:1049F8000DF0DAF984F87F010DF0D6F984F8810119
:104A080036E10DF0DBF9A4F882010DF0D7F9A4F82E
:104A180084010DF0C9F984F886010DF0CFF9A4F8E6
:104A2800880125E10DF0C0F984F892010DF0C6F96E
:104A3800A4F89C010DF0C2F9A4F898010DF0BEF994
:104A4800A4F89A010DF0B0F9DAF8003084F893016F
:104A58005B79082B40F20C810DF0B0F9A4F89E01A7
:104A68000DF0ACF9A4F8A00102E192F80590032337
:104A7800B9FBF3F9B9F1120F3FF688ACDFF89CA047
:104A88004FF0000BCB4580F0F3800DF08DF98AF8DC
:104A9800A2010DF093F940F2ED23984205DD40F6AE
:104AA800CA039842A8BF184601E040F2EE20A0F2DF
:104AB800EE20192390FBF3F00BF1010B8AF8A30108
:104AC8000AF1020ADEE70DF06FF984F89401CFE0ED
:104AD8000DF06AF904EB090309F10109B9F1080FAE
:104AE80083F88A01F4D1C3E0022D00205C21002064
:104AF800FC1800200219002000190020FE180020D0
:104B08006610002068100020781000207010002027
:104B18002C0F002038100020041900200811002054
:104B28000DF042F9C4F8089060710DF051F9A368CE
:104B38001843A0600DF038F984F892010DF03EF9A1
:104B4800A4F85C010DF03AF9A4F85E010DF036F90D
:104B5800A4F860010DF032F9A4F882010DF02EF9E5
:104B6800A4F8840184E053794FF0070AB3FBFAF202
:104B7800C2EBC2029A1A12F0FF0F7FF407ACB3FB24
:104B8800FAFA0AF1FF3A5FFA8AFABAF1FF0F6FD020
:104B98000DF00AF95FFA80FB4FFA8BF005F0DAFAAC
:104BA800814600283FF4F2AB80F800B00DF006F91A
:104BB800A9F802000DF0F8F889F804000DF0F4F8EF
:104BC80089F805000DF0F0F889F807000DF0ECF809
:104BD80089F80600D5E7DFF85C9209F1400A0DF084
:104BE800EDF8A9F8A8020DF0DFF889F8AA020DF08F
:104BF800DBF809F1040989F8A702D145EFD137E0BC
:104C08000DF0D2F81F2881463FF6C0AB3B685B79B0
:104C1800082B7FF4BBAB0DF0D1F809F18A0904EB3E
:104C2800890A00F03F00AAF802000DF0C7F8BAF8A8
:104C38000230800100F4FE501843AAF802000DF07B
:104C4800B3F8000104F829000DF0AEF814F8293083
:104C580000F00F00184304F829000DF0A5F88AF8B1
:104C680001000BF0A7FD03E05F4B012283F835201C
:104C780000200DF0E5F8FFF7D0B95C4B985905F026
:104C88006EFD18B9322005F0C4FCF6E705F0F0FE19
:104C980004F0D8FA564A574BDA60FFF7CCB90C281B
:104CA80040D00A2847D1544D54480DF04DF92846B4
:104CB800232112F020FA08B1401B20602368002B42
:104CC8005CD14D4800213022236012F0DEF998F8BB
:104CD800003053BB4A4B1B689B0614D5494B4249CD
:104CE8001B688A6B9A1A002A0DDB474A1278042A35
:104CF80009D903F5123303F5F873444A8B63D36873
:104D080083F01003D360424B9B68002B69D0414865
:104D180005B0BDE8F04F18470AF038FCFFF77DB939
:104D28000C2804D13C480DF00FF93C480DE07F28D1
:104D380012D1FFF7DEB80D28B5D07F2809D12E4A49
:104D4800013B002136482360D1540DF0FDF8FFF7F0
:104D5800D0B82F2B3FF6CDA8A0F12002D2B25E2A00
:104D68003FF6C7A813B920283FF4C3A85A1C2260ED
:104D7800214AD0540DF0E0F8FFF7BBB85A1EA95CE1
:104D8800202901D113469AE71B4A00212360D154F8
:104D9800244B254DD3F800A0D5F800B0DFF8589083
:104DA800584612F0B6F9074659463A46484612F0B0
:104DB800B9F91E4A28B919F8073053445B785B07DC
:104DC80003D010359542E7D306E0954204D2781C0B
:104DD800EB684844984702E015480DF0B5F8002301
:104DE8006FE705B0BDE8F08FB80F0020D829002084
:104DF8000400FA0500ED00E054290020ADCA0108BE
:104E0800F81800206031002002190020000C014031
:104E1800EC200020F40F002041BD01083CBD010832
:104E280068BD0108680000207CA201084CA40108A4
:104E38004CBD0108081100202DE9F0474B28A0B00F
:104E4800044600F03B8600F2B480302800F0C686A5
:104E580051D8222800F0868423D8032800F06081E6
:104E680014D8012800F05081022840F0228704203D
:104E78000CF0E6FF43200CF0B4FF4C200CF0B1FF1F
:104E880046200CF0AEFF4C2000F04CBE042800F089
:104E98005181052840F00D871A200CF0D1FF00241D
:104EA80059E1282800F0D88515D8242800F0BF85B6
:104EB800262840F0FE86B44C06200CF0C1FFB4F85A
:104EC8005C010CF0C0FFB4F85E010CF0BCFFB4F854
:104ED800600100F0A9BD2C2800F0D1852E2800F033
:104EE8004C862A2840F0E58601200CF0A9FFA64B45
:104EF800587900F017BE3D2800F016831ED83628D2
:104F080000F021860BD8322800F00686342840F0BD
:104F1800D08648200CF094FF002500F045BC3A28C4
:104F280000F0B5823B2800F01684382840F0C1868E
:104F380004200CF085FF944C00F07FBD452800F05C
:104F4800A58627D8402800F0F085422840F0B18691
:104F58008D4C10200CF074FF60790CF042FFA068B3
:104F68000CF07AFF94F892010CF03BFFB4F85C0166
:104F78000CF069FFB4F85E010CF065FFB4F860014D
:104F88000CF061FFB4F882010CF05DFFB4F8840105
:104F980000F04ABD472800F05786C0F044864928EB
:104FA80040F0878602200CF04BFF774B988900F081
:104FB8003BBD702800F0EB8258D8692800F0478282
:104FC8002AD8652800F0FA8015D84D2800F0858584
:104FD800642840F06E8607200CF032FFE7200CF0C2
:104FE80000FF694B58790CF0FCFE00200CF0F9FE2C
:104FF800042000F05ABE672800F0AC8100F21A8243
:1050080012200CF01DFF614B00241B88B3F5806F44
:105018008CBF0825012580E16C2800F02B8217D869
:105028006A2800F087846B2840F0438605200CF03E
:1050380007FF574B18880CF006FF564B18880CF0E2
:1050480002FF554B93F86E0000F0010000F06ABDB6
:105058006E28514D00F0228200F2718206200CF079
:10506800EFFEE86D0CF0F8FE4C4B0EE2782800F0ED
:105078007E8119D8742800F0B8830BD8722800F004
:105088001984732840F0158608200CF0D9FE0124F5
:1050980000F049BC762800F06D8400F2EB832F20E5
:1050A8000CF0CEFE3E4C4EE3A42800F0898414D8C0
:1050B8007B2800F0EE82A02840F0FB850C200CF045
:1050C800BFFE384B18680CF0C7FE374B18680CF059
:1050D800C3FE364B186800F0E8BDF12800F0838164
:1050E800FE2800F09484F02840F0E3852A4C042040
:1050F8000CF0A6FE236CB3F85A000CF0A4FE236C47
:10510800B3F8580000F090BC03200CF099FE002082
:105118000CF067FE20460CF064FE0D2000F002BD86
:105128000CF08EFE01200CF05CFE0A200CF059FEFB
:1051380000F044BC06200CF083FE31200CF051FE38
:1051480030200CF04EFE33200CF04BFE52200CF0B9
:1051580048FE00F068BC164B185D01340CF041FEA7
:105168000B2CF8D10024134B185D01340CF039FED8
:10517800082CF8D10024104B185D01340CF031FED6
:10518800072CF8D100F093BD081100202000002062
:105198007619002078190020F80F0020F010002060
:1051A800579B0108E8F7FF1FECF7FF1FF0F7FF1FF9
:1051B80068BA010874BA010849BA0108CA4C0B2038
:1051C8000CF03EFE20880CF03EFE608880B20CF0A9
:1051D8003AFEC64B1B68C3F3C000C3F380028000CD
:1051E80040EA4200C3F340021043C3F3401240EACE
:1051F800C20003F0100318430CF025FEBC4B1A88BC
:10520800636802F0080103F4475949EA010903F405
:10521800804149EA010903F4004149EA010903F41C
:10522800803149EA010903F4003149EA010903F42C
:10523800802149EA010903F4002149EA010903F43C
:10524800801149EA010903F0007349EA0303DFF812
:10525800D49212F0010F99F8009018BF4FF002088D
:10526800C9F3800908BF4FF0000843EA090312F0A8
:10527800020F43EA080314BF4FF0040C4FF0000C70
:1052880012F0040F43EA0C0C14BF4FF0100E4FF04D
:10529800000E12F0400F14BF202700274CEA0E0E14
:1052A80012F0100F14BF4FF4007600264EEA0707DD
:1052B80012F0200F14BF4FF4806500253E4312F40E
:1052C800807F14BF4FF400600020354312F4007F44
:1052D80014BF4FF400110021284312F4806F41EAF3
:1052E800000114BF4FF080630023002019430346D8
:1052F800247AA3420AD27F4A9D5C012202FA05F56C
:105308000D421CBF9A4010430133F2E70CF0A4FD94
:10531800794B93F8B00700F005BC784B33F91400CB
:10532800013490FBF5F080B20CF08DFD032CF4D124
:105338006D4CA08C0CF087FDE08C0CF084FD208D6A
:105348000CF081FD608D0CF07EFDA08D0CF07BFDD6
:10535800E08D69E310200CF073FD0024684B185DA4
:1053680001340CF03EFD102CF8D100F0A0BC7020E8
:105378000CF066FD00260E2474435B4D01362B6C41
:105388002344B3F819010CF05EFD2B6C2344B3F8E9
:105398001B010CF058FD2B6C2344B3F81D010CF0D5
:1053A80052FD2B6C234493F81F010CF01AFD2B6C53
:1053B800234493F820010CF014FD2B6C234493F83C
:1053C80021010CF00EFD2B6C234493F822010CF004
:1053D80008FD2B6C1C44D4F823010CF03DFD082E6D
:1053E800C9D100F064BC70200CF02AFD424C04F1D5
:1053F800700594F8D4000CF0F4FC94F8D5000CF087
:10540800F0FC94F8D6000CF0ECFC94F8D7000CF003
:10541800E8FC94F8D8000CF0E4FC94F8D9000CF0FF
:10542800E0FC073494F8D3000CF0DBFCAC42E0D18C
:1054380000F03DBC10200CF003FD0024314B185D3A
:1054480001340CF0CEFC102CF8D100F030BC2E4DFD
:1054580000242878400000F0FE000CF0F1FC2B78C6
:105468009C4280F02484294B33F814000CF0EBFCA8
:105478000134F4E7264C06200CF0E2FC20880CF0FE
:10548800E2FC60880CF0DFFC224B1888CCE2042098
:105498000CF0D6FC144B186E00F007BC07200CF07B
:1054A800CFFC1D4B1888FF28A8BFFF20C0B20CF006
:1054B80098FC1A4B186880F3100080B20CF0C3FCFB
:1054C800B5F864000CF0BFFC0B4B93F88721144B24
:1054D800186822B10A23584380F3100001E000F352
:1054E8000F0080B2A0E200BFF80F0020F8180020DB
:1054F800C01900200110002008110020EA10002027
:10550800281000203C100020742A0020902D002034
:105518004C2D0020F8100020E8180020F418002076
:10552800F018002082310020BF4C02200CF088FCCB
:1055380094F8E2010CF055FC94F8E101F2E20B203A
:105548000CF07EFCAB6E002618780CF04AFCAB6EB3
:1055580058780CF046FCAB6EB44C334418790136DD
:105568000CF03FFC032EF6D1A36ED8790CF039FC71
:10557800A36E98780CF035FCA36ED8780CF031FC4B
:10558800A36E58890CF05FFCA36E187ACAE2A74C88
:105598001E200CF055FC236C00251B78022B65D1CE
:1055A800236C05F1080253F82200A1490EF028FAED
:1055B80011F078FF80F30800C0B20CF012FC236CE5
:1055C8009C4903EB8503D86A0EF01AFA11F06AFFBA
:1055D80080F30800C0B20CF004FC236C05F10E0245
:1055E80053F8220094490EF00BFA11F05BFF80F398
:1055F8000800C0B201350CF0F4FB032DD0D1072D03
:10560800236C21D1586C8A490EF0FAF911F04AFF3F
:1056180080F30800C0B20CF0E4FB236C8449986C5A
:105628000EF0EEF911F03EFF80F30800C0B20CF066
:10563800D8FB236C93F84C000EF08AF911F032FF76
:1056480080F30800C0B20BE02B4458780CF0C9FB7B
:10565800236C2B44D87A0CF0C4FB236C2B44587D64
:1056680001350CF0BEFB0A2DC9D120E3236C2B4475
:1056780058780CF0B6FB236C2B44D87A0CF0B1FBAD
:10568800236C2B44587D01350CF0ABFB0A2DEDD172
:105698000DE33C200CF0D4FB0024644D04F1080217
:1056A8002B6C654953F822000EF0AAF911F0FAFEA6
:1056B80080B20CF0C8FB2B6C5F4903EB8403D86AFB
:1056C8000EF09EF911F0EEFE80B20CF0BCFB2B6CD4
:1056D80004F10E0253F8220057490EF091F911F027
:1056E800E1FE013480B20CF0AEFB032CD5D1072CBF
:1056F8002B6C16D1586C50490EF082F911F0D2FE7D
:1057080080B20CF0A0FB2B6C4B49986C0EF078F92A
:1057180011F0C8FE80B20CF096FB2B6C93F84C008D
:105728000BE0234458780CF08EFB2B6C2344D87A7A
:105738000CF089FB2B6C2344587D01340CF083FB5F
:105748000A2CD4D1B3E214F8010F002800F0AF827C
:105758000CF047FBF7E701200CF072FB334B1B6C96
:105768001878DFE150200CF06BFB00252F4B0C2143
:105778001C6C324B04EB850494F87920013501FB4D
:10578800023393F838000CF02CFB94F87A000CF0F4
:1057980028FB94F87B000CF024FB94F87C000CF0B8
:1057A80020FB142DE2D182E2204B1C6C062303FB64
:1057B800054494F8CE000CF014FB94F8C9000CF0E2
:1057C80010FB94F8CA000CF00CFB94F8CB000CF01A
:1057D80008FB94F8CC000CF004FB013594F8CD00DC
:1057E8000CF0FFFA0C2DDFD161E24FF00008012622
:1057F80000270E4B1A7A974233DA0933FA5C0024F1
:105808000C2363430D4D05F13001595C914207D1DA
:105818002B44586B11F07DFC82468EB9B14611E0DD
:1058280001341C2CECD11AE008110020F80F0020DC
:10583800000020410000C84200007A44589B01083B
:1058480080440CE0D1450ADA0C2303FB04535B6B5C
:1058580013F809000CF0C5FA09F10109F2E701375C
:10586800C7E7002E00F023825FFA88F00CF0E8FA10
:105878000026BDE7CC4D0024287A0CF0E1FA2B7AFB
:105888009C4280F01482C94B0021E65C0C2202FB8A
:1058980001F3C74800F13007DA5DB24205D103448D
:1058A80093F838000CF09DFA02E001311C29EDD183
:1058B8000134E4E7BF4C16200CF0C2FAB4F89801A2
:1058C8000CF0C1FAB4F844010CF0BDFAB4F8460182
:1058D8000CF0B9FAB4F848010CF0B5FAB4F8DA01EA
:1058E8000CF0B1FA94F8EF010CF07BFA00200CF000
:1058F80078FA94F8F0010CF074FA94F887010CF037
:1059080070FA94F894010CF06CFA00200CF069FA23
:10591800A54B0A201B6CB3F9563093FBF0F080B20C
:105928000CF091FA89E0E0B201340CF05AFA092C33
:10593800F9D1BCE110200CF083FA9F4B9F4C1878EA
:1059480000F002000CF04DFA9D4B18780CF049FA63
:1059580020680CF081FA60680CF07EFA994B188880
:105968000CF071FA984B18880CF06DFA8E4BB3F85E
:105978006C0059E00CF018FA074612200CF060FA97
:10598800894C17B9266F656F05E0102F19BF0025E0
:105998002E46A66FE56F38460CF023FA30460CF019
:1059A8005BFA28460CF058FAD4F880000CF054FA48
:1059B80000200CF048FA00200CF045FA0020B1E075
:1059C800794D002495F884002E4680000130C0B23D
:1059D8000CF036FA95F884000CF003FA96F8843047
:1059E8009C4280F06481794D285D0CF0FAF905F14C
:1059F8001003185D0CF0F5F905F12003185D30353A
:105A08000CF0EFF9285D0CF0ECF90134E6E708201A
:105A18000CF016FA00200CF016FA00200CF013FA1D
:105A280000200CF010FA00200CF00DFA3FE10420E1
:105A38000CF006FA5F4B986837E194F87C010CF09B
:105A4800D0F994F880010CF0CCF994F87F010CF0AF
:105A5800C8F994F8810165E0564C07200CF0F0F97C
:105A6800B4F882010CF0EFF9B4F884010CF0EBF90A
:105A780094F886010CF0B5F9B4F88801D4E74D4CD8
:105A88000C200CF0DDF994F892010CF0AAF9B4F8A6
:105A98009C010CF0D8F9B4F898010CF0D4F9B4F8DA
:105AA8009A010CF0D0F994F893010CF09AF9B4F833
:105AB8009E010CF0C8F9B4F8A001B5E73D4C0420EC
:105AC8000CF0BEF994F8D8010CF08BF994F8D901D0
:105AD8000CF087F9B4F8DA01A6E73D4C3D4D207883
:105AE800002600EB4000C0B20CF0AAF9237802357A
:105AF8009E4280F0DC8015F8020C0CF072F915F863
:105B0800010C013600EB800000EB800000F2EE2073
:105B180080B20CF098F9E9E701200CF091F9254BD7
:105B280093F894010CF05DF9C1E008200CF088F9B5
:105B38000024204B234493F88A0101340CF051F9D6
:105B4800082CF6D1B3E0184B1A4C93F8C50004F1B1
:105B58002005C0EBC000C0B20CF072F994F8F60151
:105B680000231D4AD25C904200F0A5800C33302BF4
:105B7800F7D10834AC42F1D199E040200CF060F93B
:105B88000C4C04F14005B4F8A8020CF05CF994F848
:105B9800AA020CF026F9043494F8A7020CF021F9B3
:105BA800AC42F0D183E000BFF80F002001100020C4
:105BB800589B010808110020FC1800200419002037
:105BC8000219002000190020FE1800207D10002076
:105BD800742A0020AA120020802A0020E0200CF05D
:105BE8002FF9424C04F18005B4F82A02043400F07D
:105BF8003F000CF028F9B4F82602C0F386100CF028
:105C080022F994F8240200090CF0EBF894F8240225
:105C180000F00F000CF0E5F894F825020CF0E1F81C
:105C2800AC42E1D143E0324C0D200CF009F90AF006
:105C38003DFB0CF0D6F820880CF00EF9E0680CF06B
:105C48000BF907F0B5FA30E00CF0C2F805468420ED
:105C58000CF0F6F828460CF0FFF8254BDC6805F147
:105C68008003A3428CBF641B802407F05BFB28469B
:105C7800224669460AF04EFB05460024AC4216DA75
:105C88001DF804000CF0ADF80134F7E713200CF010
:105C9800D7F80024174B185D01340CF0A2F80B2C30
:105CA800F8D100200CF0D8F800200CF0D5F801202D
:105CB80018E0002016E00CF094F8B4F8F8010CF0A5
:105CC800C2F894F8FA010CF08CF894F8FB010CF087
:105CD80088F894F8FD010CF084F894F8FC010CF0B5
:105CE80080F846E720B0BDE8F08700BF0811002023
:105CF8001000002068BA01086B4B6C4A2DE9F04F80
:105D08005E8914684FEA062AB4EB0A0A9C884FF0A9
:105D180000054FEA04481C894FF0000BA4FB0A67F2
:105D280065EB0B0B04FB0B77F40944EA476418EBAB
:105D380004065C884FF000094FEAE7154FEAC438BB
:105D4800DC8849EB050787B0CDE90467A4FB0A673F
:105D580004FB0B77340A44EA076418EB04064FEA9D
:105D680027259C894FF0000949EB0507CDE9006715
:105D7800AAFB046704FB0B77F40D44EA472414F5E7
:105D8800FA664FEAE75545F10007B6F5FA6F77F17D
:105D98000003CDE90267964666DADDE90489A4FBCB
:105DA800046704FB05F34FF0050C07EB4307A6FB5C
:105DB8000C230CFB07335F104FEA3206B8EB0608DA
:105DC8004FEA920646EA837669EB07099F10DDE9F8
:105DD8000023921B63EB0703CDE90023DDE902678B
:105DE800334A4FF0FF33964277EB0303CDE904893A
:105DF80027DA40F6AC520023A4185D4104FB05F3F2
:105E0800A4FB04456FF0060205EB4305664202FB5E
:105E18000566A4FB0223334418EB020649EB03078B
:105E2800CDE904670B26A4FB062306FB0533DDE951
:105E380000455B104FEA3202A41A65EB0305CDE971
:105E48000045DDE902450AFB0BF3AAFB0AAB0BEBA5
:105E5800430B4FEADA7242EA4B02A41A4FEAEB7399
:105E680065EB0305CDE90245DEF80440009B019D82
:105E7800A4FB032304FB05334FEA525848EAC3281E
:105E88004FEA6359DDE90423B8EB020269EB030327
:105E98009946D30B43EA494300B1036009B1029B19
:105EA8000B6007B0BDE8F08F5C020020C010002036
:105EB80024FAFFFF2DE9F04FDFF8589285B0074626
:105EC800D9F808000E460DF047FD8E4C8046208814
:105ED8000DF03EFD4FF05C51054640460DF090FD3B
:105EE8004FF06451824628460DF08AFD014650461F
:105EF8000DF07CFC4FF06251824640460DF080FD6B
:105F08004FF06A51804628460DF07AFD014640461A
:105F18000DF06CFC0546B4F902000DF01DFD0146BC
:105F280028460DF06DFD5146054650460DF068FDBA
:105F38008046B4F904000DF00FFD014640460DF00F
:105F48005FFD014628460DF053FC80460DF01EFF0C
:105F58006D490546A06140460DF006FED9F80C30A3
:105F68008046284601930DF0F7FC4FF07C510DF068
:105F780047FD66490DF03AFC0546E389B4F90A0085
:105F880002930DF0E9FC29460DF03AFD29460DF083
:105F980037FD4FF058510DF033FD8146B4F9080034
:105FA800B4F810B0B4F80CA00DF0D6FC29460DF0EA
:105FB80027FD014648460DF01BFC4FF058510DF0E7
:105FC8001FFD4FF060510DF01BFD4FF07E510DF09D
:105FD8000FFC8146E0880DF0BBFC014648460DF0F9
:105FE8000FFD002181460DF09FFE00287BD1294638
:105FF80028460DF005FD03900FFA8BF00DF0ACFC70
:10600800039B014618460DF0FBFC4FF060510DF064
:10601800F7FC8346BDF908000DF09EFC01462846B2
:106028000DF0EEFC01460DF0E3FB014658460DF07D
:10603800DFFB4FF07A510DF0E3FC834601980DF039
:106048008BFC01464FF093400DF0D0FB05460FFA4C
:106058008AF00DF081FC4FF08F410DF0D1FC014624
:1060680058460DF0C5FB4FF066510DF0C9FC0146CE
:1060780028460DF0BBFB26490DF0C2FC49460DF041
:1060880073FD0546B4F916000DF066FC29460DF0BF
:10609800B7FC29460DF0B4FC4FF040510DF0B0FCB0
:1060A8008146B4F914000DF057FC014628460DF05E
:1060B800A7FC4FF060510DF0A3FC014648460DF0D7
:1060C80097FB8146B4F912000DF046FC014648469C
:1060D8000DF08EFB4FF076510DF092FC01462846EC
:1060E8000DF086FB00E0002017B10DF04FFE386080
:1060F8002EB140460DF04AFE64235843306005B087
:10610800BDE8F08F980200200000A04500007A4703
:106118000050C345C0100020704770472DE9F0417A
:10612800324C334D62892B8AB4F904809A1A238938
:10613800B4F902E05A43B4F91230D613B4F9142072
:10614800DB02324493FBF2F232440A26E261564300
:10615800A2F57A6202FB02F3B4F90EC002FB0EFE4E
:1061680002FB08F2B4F90C801B130CFB03FC03FBC5
:1061780008F31B1403EB62320232E388921002F533
:10618800004253434CF25032B4F920704FEAEE2EDD
:10619800B4F900400EEBEC2C0CEB8404BC406D69A8
:1061A8000234A5EBA4043A4162434FEAD3384EBF08
:1061B800B2FBF8F35400B4FBF8F340F6DE3448BF02
:1061C8005B001A12524362430A4C08365C4324149B
:1061D80004EB224202F6CF62361103EB221300B120
:1061E800036001B10E60BDE8F08100BF70020020BD
:1061F800C010002043E3FFFF074B1A6859694904A0
:1062080008D5520441BF4FF480425A61034B012222
:1062180048BF1A76704700BF00040140C010002034
:10622800024B4FF480521A80704700BF20000020B4
:10623800024B4FF480521A80704700BF20000020A4
:1062480070477720482101220BF04ABC772058215B
:1062580001220BF045BC7620F42131220BF040BC22
:10626800064B002193F82020054B92013432197611
:106278007720F42102F0FC020BF032BC70020020FF
:10628800C0100020034B00221A767720F4212E221A
:106298000BF026BCC010002007B5002101AB03227B
:1062A80077200BF0DDFB9DF805309DF804001B02FC
:1062B80043EA00439DF80600184303B05DF804FB69
:1062C80008B5FFF7E9FF014B586008BDC010002072
:1062D80008B5FFF7E1FF014B186008BDC0100020AA
:1062E80007B5F7216B46062276200BF0B9FB9DF81F
:1062F80000309DF801101B0343EA01139DF80210BA
:10630800094A43EA1113D3609DF803309DF804103D
:106318001B0343EA01139DF8051043EA1113936028
:1063280003B05DF804FB00BFC010002013B5104C8B
:10633800237E1BB9638B0133638316E0032201AB11
:106348007720F6210BF08CFB9DF805309DF8042092
:106358001B0243EA02439DF806201343054AB2F99B
:106368002020C2F10802D340636102B010BD00BF13
:10637800C01000207002002013B50B4C237E1BB9FF
:10638800638B013363830CE0022201AB7720F62193
:106398000BF066FB9DF804209DF8053043EA0223C4
:1063A800238202B010BD00BFC010002013B5062222
:1063B8000446432168206B460BF052FBA0B19DF8C0
:1063C80000209DF8013043EA022323809DF8022033
:1063D8009DF8033043EA022363809DF804209DF86A
:1063E800053043EA0223A38002B010BD13B506228C
:1063F80004463B2168206B460BF032FBA0B19DF8A8
:1064080000209DF8013043EA022323809DF80220F2
:106418009DF8033043EA022363809DF804209DF829
:10642800053043EA0223A38002B010BD13B5012250
:106438000DF107033A21044668200BF011FB0520F3
:1064480004F0DCF89DF8073003B10123237002B093
:1064580010BD104B13B51A7F1C46C2B90E4B1B68F2
:10646800ABB11A681AB10D49886902438A619A88E2
:106478009868ADF8042002228DF8072004220DEB5D
:1064880002018DF8062009F00FFE0123237702B0E0
:1064980010BD00BFC01000205402002000100240B0
:1064A80008B5FFF7D6FF6B21802268200BF018FB98
:1064B800642004F0AEF86B21032268200BF010FB77
:1064C8000F2004F0A6F8104B19211A7868200BF059
:1064D80007FB0F2004F09DF80C4B1A211A7868204E
:1064E8000BF0FEFA1B21182268200BF0F9FA1C2188
:1064F800102268200BF0F4FABDE808406820372124
:1065080002220BF0EDBA00BF580200200000002064
:1065180008B5FFF79EFF074B1B7813B1012B03D07B
:1065280008BD4FF4006201E04FF48052024B1A801C
:1065380008BD00BF5902002020000020F8B50F4612
:106548001646074C4FF48055656140F080000BF00B
:1065580023FF3846002132460BF044FF2561F8BD81
:10656800000C014013B501220DF107010446382043
:10657800FFF7E4FF052004F041F89DF8073003B168
:106588000123237002B010BD13B5044669464320A9
:106598000622FFF7D3FF9DF800209DF8013043EA5B
:1065A800022323809DF802209DF8033043EA02234A
:1065B80063809DF804209DF8053043EA0223A380F8
:1065C80002B010BD13B5044669463B200622FFF70A
:1065D800B5FF9DF800209DF8013043EA022323808F
:1065E8009DF802209DF8033043EA022363809DF85A
:1065F80004209DF8053043EA0223A38002B010BDB1
:1066080070B50E46054C4FF4805565610BF0C4FE1D
:1066180030460BF0C1FE256170BD00BF000C014083
:1066280008B580216B20FFF7EBFF642003F0F1FF32
:1066380000216B20FFF7E4FF642003F0EAFF6B20E2
:106648000121FFF7DDFF1B201821FFF7D9FF1C20D0
:106658001021FFF7D5FF054B1A201978FFF7D0FF57
:10666800BDE8084019200021CAE700BF010000204A
:10667800F8B50F461646074C4FF48055656140F053
:1066880080000BF089FE3846002132460BF0AAFE46
:106698002561F8BD000C014013B501220DF1070179
:1066A80004463A20FFF7E4FF052003F0A7FF9DF812
:1066B800073003B10123237002B010BD174A13B588
:1066C8001388044623F040031B041B0C1380138813
:1066D8003B2023F038031B041B0C138013886946E6
:1066E8009BB243F0400313800622FFF7C1FF9DF8D9
:1066F80000209DF8013043EA022323809DF8022000
:106708009DF8033043EA022363809DF804209DF836
:10671800053043EA0223A38002B010BD00380040D0
:10672800174A13B51388044623F040031B041B0CB7
:1067380013801388432023F038031B041B0C138099
:10674800138869469BB243F0400313800622FFF783
:106758008FFF9DF800209DF8013043EA0223238033
:106768009DF802209DF8033043EA022363809DF8D8
:1067780004209DF8053043EA0223A38002B010BD2F
:10678800003800400AF0F8BF0BF01EB90AF0F4BF59
:106798000BF01AB973B51D4C637F53BB1C4A1D4DD2
:1067A80093694FF4805643F00803936110238DF8E2
:1067B80006302846032301A98DF80730ADF8046098
:1067C80009F072FC144A2E61138823F040031B045D
:1067D8001B0C1380138823F038031B041B0C43F095
:1067E8000803138013889BB243F0400313800123EE
:1067F8006377752001A90122FFF7A0FE9DF8040028
:10680800A0F170035842584102B070BDC01000207A
:1068180000100240000C01400038004070B50E46E0
:10682800054C4FF4805565610BF0B6FD30460BF012
:10683800B3FD256170BD00BF000C0140284A08B5B2
:106848001388802123F040031B041B0C138013883A
:106858006B2023F038031B041B0C43F03003138018
:1068680013889BB243F040031380FFF7D7FF9620AD
:1068780003F0CFFE03216820FFF7D0FF962003F036
:10688800C8FE03216B20FFF7C9FF012003F0B6FE05
:1068980010216A20FFF7C2FF012003F0AFFE00219C
:1068A8006C20FFF7BBFF012003F0A8FE0021192090
:1068B800FFF7B4FF012003F0A1FE10211C20FFF711
:1068C800ADFF012003F09AFE1B201821FFF7A6FF59
:1068D800012003F093FE034B01221A7008BD00BF8C
:1068E800003800405A0200201F4A13B513886B2055
:1068F80023F040031B041B0C13801388802123F012
:1069080038031B041B0C43F0300313801388062440
:106918009BB243F040031380FFF780FF962003F0FB
:1069280078FE75200DF107010122FFF7A1FE9DF801
:106938000730682B04D0013C14F0FF04EED10EE0C0
:106948000C200DF107010122FFF792FE9DF8073098
:10695800142B04D3182B04D9543B062B01D900203F
:1069680000E0012002B010BD0038004007B5232028
:1069780003F04FFE6820752101220DF107030BF08B
:106988006FF828B19DF80700A0F1680358425841F4
:1069980003B05DF804FB00BF2DE9FF47CB4C074669
:1069A8002378CB4E002B00F0E78132686368D31A56
:1069B8007C2B40F2E181237A6260013323724FF02D
:1069C800000808F12400C14DC0B206F0D3FD05F15E
:1069D8000A0333F918000CF0BFFFBE4B8146188834
:1069E8000CF0BAFF014648460DF0BEF8BA490DF062
:1069F80007F80DF0CBF908F1010800B206F0A8FD80
:106A0800B8F1030FDDD1302006F0B4FDB5F9100060
:106A180006F09EFD06F0A6FD2B7A9A072CD141F2CE
:106A280088336A689A4218D9102006F0A3FD68696D
:106A38004FF0640890FBF8F000B206F089FD2120C1
:106A480006F098FD686990FBF8F308FB130000282E
:106A5800B8BF404200B206F07BFD142006F08AFD64
:106A6800B4F9180006F074FD1C2006F083FD002020
:106A780006F06EFD06F076FD237ADFF850825B079C
:106A880040F05781022006F075FDD8F81C006423F9
:106A9800323090FBF3F000B206F05AFDB8F92650F8
:106AA8004FF0050A95FBFAF5032006F063FD8B4BC2
:106AB800ADB21B78DFF8389213F0040F0DD008F54B
:106AC800D970394603F0BDFC28B9D9F8003013F065
:106AD800100F18BF002528B205E0D8F804389889A7
:106AE800B0FBFAF000B206F033FDD9F800309F078A
:106AF8006ED5DFF80092B4F8082899F800304FF006
:106B0800640808FB02325B00B2FBF3F3B4F80A78BE
:106B180006203F01BFB247EA0327BFB2C3F30323EE
:106B28001F4306F027FD38B206F012FDB4F80A3804
:106B380099F8001001339BB293FBF1F201FB123379
:106B4800A4F80A38D4F80C38604D9B7B012B05D18A
:106B5800392006F00FFDB5F908081AE0B5F808580D
:106B68006E235D43152795FBF7F53A20AFB206F083
:106B780001FDB7FBF8F528B208FB157506F0E8FC2F
:106B88003B2006F0F7FCA8B2451D0A2095FBF0F063
:106B980000B206F0DDFC282006F0ECFCD4F8103832
:106BA8000A2093FBF0F000B206F0D2FC042006F0B5
:106BB800E1FCD4F804389B8913B109F089F804E0A2
:106BC800424BD3F8140880F3100000B206F0C0FC62
:106BD800D4F818383D4F9D0640F1A08097F81C382E
:106BE80098071DD5112006F0C5FCB7F81E084FF40C
:106BF800F36568433A4B90FBF3F000B206F0A8FC4B
:106C0800192006F0B7FCB7F81E084543642095FB29
:106C1800F0F595FBF0F300FB135000B206F098FC7A
:106C280094F81C38B4F8205813F0020F08BF002558
:106C3800012006F09FFC28B206F08AFC092006F025
:106C480099FC002006F084FC264B94F822581A88F8
:106C5800B2F5967F0AD91D4B1B7A03F00F03072B59
:106C680004D842F20F75954228BF1546052006F054
:106C780081FCD4F80C385B7B0BB928B216E0A5F17F
:106C880020000CF069FE18490CF06EFF0021054643
:106C98000DF054F810B94FF07C5101E04FF03F412E
:106CA80028460CF0A5FD0DF071F800B206F050FC76
:106CB80094F81C28054B910703D493F82328012A3C
:106CC8001AD1012384F8233808482EE0E010002068
:106CD800782D00202000002000007A448231002016
:106CE800A0860100560000206666E63F04190020D1
:106CF800542D002054000020D3F80C58C04968686F
:106D08000CF07EFE0DF042F8BD490290A8680CF028
:106D180077FE0DF03BF8039002A806E0B94A02ABF3
:106D280092E8030083E80300184606F033FC06F0F7
:106D380019FC237A282B1FD1B34B00221A7233680F
:106D48004FF47A70B3FBF0F83C27172006F012FCDA
:106D5800B8FBF7F5B5FBF7F007FB1050000200B2DF
:106D680006F0F6FB182006F005FC07FB158000B2BC
:106D780006F0EEFB06F0F6FB94F82C38A24D002B3B
:106D880000F0618103F01EFCD5F830389F4AC31A21
:106D98009342074640F2C780002385F8363885F8C5
:106DA8003838B5F80838DAB21B0A85F8522885F859
:106DB800533885F8482885F84938D5F86028336865
:106DC8009A1AD5F86438D97B4FF47A734B439A42B0
:106DD8000ED38F4B1B68C5F8603895F86838013BAF
:106DE800012B9FBF102385F83638022385F83838E1
:106DF800D4F810280A20D4F8143892FBF0F293FB48
:106E0800F0F384F85028121284F8512884F8543882
:106E180094F81C281B1284F8553894F822389207E5
:106E2800794984F8833803D42D2381F8843878E0AD
:106E3800D4F824987748DFF8E8C199FBF0FA0CFBFE
:106E48000A924FF0060E042B0EFB02F28CBF33237E
:106E5800322381F88438704BD4F8286892FBF3F118
:106E680096FBF0F003FB1122642592FBF5F20CFB74
:106E7800006C0EFB0CFE84F87528121284F8762834
:106E88009EFBF3F203FB12E393FBF5F30AEB8A0A8A
:106E98004FFA81F80AEB8A0A08EB8A0189B284F86A
:106EA800731800EB8000090A84F8741800EB80005E
:106EB80051B201EB800292B284F87828120A84F861
:106EC800792884F87A38B4F81E281B1284F87B389D
:106ED8002423534393FBF5F5B4F896380A2284F833
:106EE8007C381B0A84F87D38B4F820384FEAD97901
:106EF800B3FBF2F303F5FA739BB284F87E381B0AEE
:106F080084F87F38B4F89838F60F84F87058C5F3C9
:106F1800072584F8729884F8776884F8715884F89B
:106F28008538C4F8307894F89A88374DB8F1000F4E
:106F38000DD1D5F8A00803F01BFC012807D90228B9
:106F4800364E00F05E8206F0F5FA0123B370D4F8ED
:106F5800A4282D4D002A76D095F89A683EB140F6BF
:106F6800B731D5F8AC38FB1A8B4219D86BE001233E
:106F7800D5F8A00885F89A3803F091F8D5F8B03814
:106F8800082193F9000002238DE8480032464FF4A7
:106F9800964303F097F885F8B468C5F8A00850E060
:106FA80095F8A868CEB9D5F8A008C5F8A46885F8FA
:106FB8009A6803F074F8D5F8B038082193F90000FE
:106FC80001238DE8480032464FF4964303F07AF8DF
:106FD800C5F8A00806F0AEFA33E0013EF6B285F82F
:106FE800A86895F8B41895F8B538DEB94A1C013385
:106FF80085F8B42885F8B538D5F8A0081FE000BF93
:107008008096184BE49C0108E01000203F0D030017
:10701800782D00208096980040420F002000002024
:10702800806967FF12F8016B01337018314685F8E3
:10703800B408D5F8A008C5F8A42885F8B53803F031
:107048009AFBC4F8AC7894F8B638A14DF3B1D5F8EA
:10705800B838DBB1D5F8BC38C3B1C5F8C0381B683F
:107068009C4AC5F8C438D5F8C8381344187AFDF7CF
:10707800E3FED5F8C03898790AF0B3FED5F8C838D9
:107088000133092B88BF0023C5F8C838924D94F8FE
:10709800CC282E688E4B002A00F0EE81D3F8D02839
:1070A800002A00F0E98193F8D438013B012B00F263
:1070B800E381D4F8D008864F03F05AFBE0B1D7F843
:1070C800D00803F052FB97F8D53880467E2BD5F8C8
:1070D80000900ED102231B2887F8D43809D1D7F89D
:1070E800D00803F045FB20B90123C7F8D89887F8E2
:1070F800DC3884F8D588DCE7D7F8D8282B689B1AC1
:1071080041F6583293421ED9032387F8D438B3E1A5
:10711800724A32F8130010B903464FF40360013382
:10712800B0F5C06FDBB279D01ED9B0F5006F7FD053
:1071380032D9B0F5036F3FD184F8DD38D4F8183868
:10714800634F99063FD494F8DC1894F8DD38002989
:1071580000F054812A68921B012AD9D984F8DD38B5
:10716800002384F8DC3887E1B0F5007F43D007D8E6
:10717800B0F5807F49D0B0F5887F00F08B80E6E7D6
:10718800B0F5806F00F0AE80B0F5826F00F0F3804C
:10719800B0F5047FDBD123E0B0F5E26F00F08B801F
:1071A800B0F5E46F00F08C80B0F5E06FCFD184F8D3
:1071B800DD38B4F90A1087E0B0F5046F74D0B0F583
:1071C800026FC4D103E197F81C389A07BBD5B7F80A
:1071D8001E1824234B436421123393FBF1F107E17A
:1071E80084F8DD383E4B3A4F1B689B07ABD5B7F8A0
:1071F80008380A21FBE084F8DD38394B344F1B6826
:107208001905A0D5D7F81018F2E084F8DD38D4F8BD
:1072180018382F4F5A0796D57969E9E084F8DD3890
:107228002F4B2B4F1B681B058DD5D7F81418DFE0A3
:10723800D4F81818264A8F0684F8DD3883D592F8D2
:107248001C1888077FF57FAFD90711D5D2F82838E1
:10725800192283EAE371A1EBE37101EB5101B1FB60
:10726800F2F1002BACBF41F0004141F040410EE08B
:10727800D2F82438192283EAE371A1EBE37101EB18
:107288005101B1FBF2F1002BB8BF41F080414FF43E
:1072980000608BE084F8DD38D4F818380C4F5B07B1
:1072A8007FF551AF3969A3E084F8DD38B4F91830B7
:1072B800642159437AE084F8DD38B4F90C1003E00E
:1072C800B4F90E1084F8DD382C2391FBF3F16DE04E
:1072D800E0100020E49C0108782D00208ABE0108F7
:1072E800542D002084F8DD3894F8DE38644A0133E0
:1072F800DBB2032B88BF012382F8DE3842F2107319
:1073080094F8DE1859435F4B1B78D80748BF013102
:107318009A0748BF02315F07B4F8E03848BF043124
:10732800D80748BF0A319A0748BF14311F0648BF1B
:107338002831D80548BF28315A0748BF64311F078C
:1073480048BFC831980548BF01F5C8719A0648BFBB
:1073580001F57A71DF0648BF01F5FA61580648BFA2
:1073680001F57A614FF4806000F0D2FD444B0022B1
:1073780083F8DC28E7E6D4F81818DFF8048111F060
:10738800200784F8DD3817D098F81C2812F0020F6F
:1073980014BF4FF47A71002112F0010F14BF4FF49B
:1073A800FA6300230B4494F82218194400F0B0FD46
:1073B800002384F8DC38C6E6334B1B6819067FF5D2
:1073C800C2AE394600F0A4FD88F8DC78BBE684F844
:1073D800DD38D4F818382A4F9A067FF5B4AE97F8F6
:1073E8001C389B077FF5AFAEB7F8203864215943A6
:1073F80000F08EFD002387F8DC38A4E684F8DD3839
:107408003AE0B37823B1C5F89C7886F802809EE507
:10741800D5F89C38FB1AB3F57A6FFFF498AD0123C1
:10742800D5F8A008B37003F0A0F90646D5F8A0086F
:1074380003F09BF976067FF48AAD8A2802D08E285D
:107448000DD084E5D5F8183898067FF580AD95F805
:107458009A38002B7FF47BAD05F6690306E095F8B2
:107468009A38002B7FF473AD05F63403C5F8A438B9
:107478002D2385F8A8386AE504B0BDE8F08700BF79
:10748800E010002082310020542D0020344B354A72
:107498001B68126810B51A60334A11685960516840
:1074A80092689960DA60314A116819615168926886
:1074B80059619A612E4A1168D961516892681962B6
:1074C8005A622C4A11881985518859859188D28821
:1074D8009985DA85284A11881986518859869288AB
:1074E8009A86264A1188D98651889288198719461A
:1074F80021F83A2F224A10780022824206DA214CDB
:1075080034F81240013221F8024FF6E71E4A128879
:10751800A3F864201D4A1288A3F866201C4A118823
:10752800A3F86C1051889288A3F86E10A3F8702005
:10753800184A3B2112689A66174A126892FBF1F2C0
:10754800B2F5967FC8BF4FF0FF325A67134A1288C8
:10755800A3F87820124A5289A3F85E2010BD00BF14
:10756800D82D0020603100206822002074220020DD
:1075780080220020001100201C100020EA100020AA
:10758800C81F00203C100020F42A0020DC0F002037
:1075980022100020F4100020040000205C100020BD
:1075A800281000202DE9F84305460E460D4B00240F
:1075B80093E88003B44213DA7B1933F9140008EB1B
:1075C800050333F9142009EB050333F914300134AA
:1075D8001344022293FBF2F3C01A0AF03CF8E9E7DD
:1075E800BDE8F883D82D002010B5134B014693F859
:1075F800D837012B19D1114B114C1878421CD2B233
:107608001A70120644BF00221A700E4A1B781278AC
:107618002154934236BFC2F180029B1A9B183F2B1C
:1076280009D9BDE8104005F099BE074BBDE81040E8
:10763800186803F0A0B810BD08110020642C0020C1
:10764800662C0020652C0020C02D002070B5472036
:10765800FFF7CAFF174B1B681B0307D5164B174AC2
:107668005B6810681B68C01A09F0E5FF144E154CDA
:10767800154D307809F0DFFF23682868C01A09F033
:10768800EAFF63686868C01A09F0E5FF0F4B1888BD
:1076980009F0D1FF0E4B188809F0CDFF0D4B188863
:1076A80009F0C9FF337823742B68A3606B68E36023
:1076B80070BD00BF5C2F0020D82D00206031002055
:1076C80002190020C42D00200419002000190020F0
:1076D800FE180020641000207FB5264C264E274D4A
:1076E8002749284A284B20B128480088B0F5805FF0
:1076F80031D2308891F820101278ADF8040028783B
:107708001C4D1B788DF806008DF807108DF80820A1
:1077180001A8294606228DF809300FF09BFC30B3EA
:107728000198BDF808302860AB805320FFF75CFF54
:10773800208809F080FFA07809F07DFFE37801A890
:107748000193237902936379039309F0D9FE0F4BD0
:1077580000221A800BE0308891F8201020801278DF
:1077680028781B78A070E17022716371DDE704B09E
:1077780070BD00BFC4190020C0190020FC180020EB
:10778800C42F00205B0E0020C00E00207C2F00209C
:107798000A4A138801331380094A136801331360B6
:1077A800084A138801339BB2202B01BF00231380A2
:1077B800054A138808BF0133138070477C2F0020C7
:1077C800642F0020682F00206A2F002038B5394B1D
:1077D80005461B780C46083B012B6AD84520FFF765
:1077E80003FF2846FFF700FF0C2D23D004D80A2DED
:1077F8000AD014D835B138BD0E2D4BD02ED3FF2D5D
:1078080050D038BD206849E02078FFF7EDFE627956
:107818006378002A14BF80200020184300E02078F5
:10782800FFF7E2FEA078FFF7DFFEE078FFF7DCFE67
:1078380020793BE0B4F9000009F0F2FEA078FFF7E8
:10784800D3FEE078FFF7D0FEB4F9040009F0E8FEB3
:10785800B4F90600BDE8384009F0E2BE6378207844
:107868008BB180F08000FFF7BFFEA468E0B2FFF79D
:10787800BBFEC4F30720FFF7B7FEC4F30740FFF7CA
:10788800B3FE200E12E0FFF7AFFE6068BDE8384097
:1078980009F0E1BE206809F0CEFE6068BDE8384016
:1078A80009F0C9BE044809F0DAFE0020BDE83840F6
:1078B8009AE638BDB42D0020AABE01082DE9F04F84
:1078C800BE4B8BB01A880193BD4F002A40F0A980A7
:1078D80042F20103B7F8D607BA4EC21A50425041D5
:1078E800FFF7FAFEFFF7D2FD346849202546FFF777
:1078F8007BFEB54B04F11C09186809F09CFE55F88D
:10790800040B09F098FE284607F066FD04F1100004
:1079180007F062FD4FF01008AC4D01232A6803FA06
:1079280008F3134203D0D9F8000009F094FE08F1D7
:107938000108B8F1130F09F10409EDD104F1280089
:1079480007F03AFDB7F84431B4F92E00C01A09F02F
:1079580072FE2B68DB0408D59D4BB4F864001B88C5
:10796800181AC0F30D0009F066FE2B68980403D5B9
:10797800B4F8660009F05FFE2B68590503D504F1D9
:107988006C0007F019FD2B681A0502D5A06E09F0E6
:1079980062FE2B685B0402D5606F09F05CFE2B6801
:1079A800180403D5B4F8780009F045FEA04604F1A0
:1079B800300007F001FD04F1360007F0FDFCB7F8D0
:1079C800443138F93C0F0127C01A09F034FE814BC5
:1079D8001B789F4208DA38F9020FB4F93C300137B6
:1079E800C01A09F038FEF2E72B68990505D5B4F9F5
:1079F8005E00A0F2DC5009F02EFE32687648726014
:107A0800B260121A9110754A4A43531C032293FB21
:107A1800F2F202EB42029A1A7C2303FB0203336060
:107A2800D6E16F4B6F4A1B6811688B4206D00AA9D2
:107A380041F8203D00201360FFF7C8FE019B97F82E
:107A4800D6171B8897F8D7070B44013BB3FBF0F216
:107A580000FB12338B4280F086815A4F0120FFF7DA
:107A68003BFEFFF713FD50203E687D68FFF7BCFD25
:107A7800BA683B6810681B687A680344106806F1A6
:107A88001C0BA3EB400009F0E6FD6A68736802A8C6
:107A98009B1A0293AA68B36805F11C089B1A039302
:107AA800EA68F36810249B1A049307F095FC2A6986
:107AB800336902A89B1A02936A6973699B1A039334
:107AC800B369AA699B1A049309F01AFD3F49012278
:107AD8000B68A2401A428A4606D0DBF80000D8F8A4
:107AE8000030C01A09F0B7FD0134132C0BF1040B58
:107AF80008F10408EAD106F1260005F12601002361
:107B080031F9024F30F9022F121B02AC44F823203E
:107B18000133042BF4D103214FF000094FEA890304
:107B28005FFA83F902AB53F821206AB102F1080029
:107B38000F2802D849F0010906E08032FF2A94BFD5
:107B480049F0020949F0030911F1FF31E6D248462C
:107B58000024FFF749FDA0460DF1080B09F00302C8
:107B6800022A16D0032A1DD0012A4ED1B8F1000FDF
:107B780005D1DBF8004090462401E4B245E0DBF88B
:107B880000004FF0000800F00F002043FFF72CFD25
:107B98003BE0B8F1000F0CD0DBF80000C0F3031095
:107BA80020432CE0B8F1000F1ED19BF80100FFF72D
:107BB8001BFD9BF80000FFF717FD26E0682F00204B
:107BC80008110020D82D0020642F00205C2F0020F1
:107BD800582F0020C81F0020E42D0020DF7BEFBDB8
:107BE800702F00206C2F0020DBF80000C0F303305A
:107BF8002043FFF7F9FCDBF80000C0F30710FFF79C
:107C0800F3FCDBF800402401E4B20BF1040B06ABF3
:107C18009B454FEA9909A1D1B8F1010F02D120463D
:107C2800FFF7E2FCDAF8003013F480541FBFB6F80F
:107C38006420B5F864100124521A18BF02929A04FD
:107C48000AD50AAA02EB8401B5F86600B6F86620E0
:107C58000134121A41F8202C580513D502AA02EB58
:107C6800840C06F16A0E05F16A0000223EF9021F33
:107C780030F9028FC8EB01014CF822100132032AB7
:107C8800F4D10334190508D50AAA02EB8400A96EB9
:107C9800B26E0134521A40F8202C5A0408D50AAAA8
:107CA80002EB8400696F726F0134521A40F8202C7D
:107CB80018040BD50AAB03EB8402B5F87810B6F8B4
:107CC800783001345B1A42F8203C00E0FCB1012C0A
:107CD80003D1029809F0BFFC19E0631E002002AA34
:107CE80052F823204000C0B20AB140F00100013B25
:107CF800F5D5FFF779FC4FF0000802AB53F82800E0
:107D080008B109F0A8FC08F10108A045F5DB30200E
:107D18000321FFF747FC36200321FFF743FC2F4BD5
:107D28003C201978FFF73EFCDAF80030990506D5B3
:107D3800B6F95E00B5F95E30C01A09F08CFC3A68F5
:107D480027487B687A60121A9110264ABB604A431A
:107D5800531C032293FBF2F202EB42029A1A7C2391
:107D680003FB02033B60204B1B681A0630D51F4CEF
:107D78001F4D22682B689A420BD162686B689A4241
:107D880007D1019B1B88102B11D11A4B1B885B064E
:107D98000DD14820FFF728FC206809F05CFC6068DA
:107DA80009F059FC23682B6063686B600EE0124A87
:107DB8000F4B11782A7C914208D1104A99681068B3
:107DC800884203D15268DB689A4201D0FFF73EFC33
:107DD80009F084FB0BB0BDE8F08F00BFC81F00207E
:107DE800E42D0020DF7BEFBD542D0020681000201B
:107DF800C42D00206A2F0020021900200419002039
:107E08002DE9F84F0C9EC2EB030B394C0B9B002954
:107E180014BF4FF0060A4FF0040AF61A63680546C5
:107E28000133904613D1236853455ED2314A032B60
:107E380098BF294652F823202F4809F07BFC636835
:107E48000022013363602D4B05469A7113E000252B
:107E580011E02B4A1278954240DA0B9BE3B109FBFB
:107E680006F2995C01228A40264909680A4213D120
:107E7800636801336360D4F804900A9B1C4F9945EA
:107E8800E7DB2BD10A20FFF7AFFB3B6801333B60F0
:107E98004FF0FF337B6021E0184A917921B12C2003
:107EA800FFF7A2FB013501E00121917109FB0BF3FA
:107EB800226808EB030752B958F8030009F0CFFB12
:107EC80097F9041005444B1CD2D00F4802E03A44FD
:107ED8000E48117909F02EFC0544C9E72068504581
:107EE8002CBF00200120BDE8F88F0020BDE8F88FE6
:107EF800742F0020F89C0108B5BE0108C4190020A1
:107F0800640000205C2F0020C4BE0108ECC10108F9
:107F180030B585B004AC002524F8025D0091ADF8B9
:107F280006002146102005F0E7FA9DF806002146D4
:107F380005F0E2FA9DF80700214605F0DDFA9DF804
:107F48000000214605F0D8FA9DF80100214605F009
:107F5800D3FA9DF80200214605F0CEFA9DF80300F9
:107F6800214605F0C9FA9DF80E002946C043C0B263
:107F780005F0C2FA05B030BD426A806A131A584249
:107F8800584170474171704743799B070AD5436A46
:107F98008269D154436A01690133B3FBF1F201FBF1
:107FA800123343627047437913F001031FBFC3685C
:107FB80003F1FF32C369006A1DBF181A1040C0B22E
:107FC80018467047437910B513F0010304460DD0E5
:107FD800FFF7E9FF58B1236A6269E168D05C0133B1
:107FE800B3FBF1F201FB1233236210BD184610BD3A
:107FF80090F83B3210B57BB990F83A3290F8394294
:10800800A34209D2B0F8401201229A400A43013330
:10801800A0F84022DBB2F3E710BD8379DB0748BF45
:10802800B1FA81F1D0F8343148BF49095A681B893F
:1080380009B1136170475361704710F80A3C013366
:10804800DBB20A2B84BF10F8131C054A00F80A3C5F
:1080580082BF002322F8113000F80A3C704700BFA5
:10806800A4300020334A70B5136C9068194440F668
:108078008C23081A98429160D060516013463BD90E
:10808800127893F9451010468A420BD1111F08291E
:1080980008D893F84610182901D8013103E083F86D
:1080A800442002E0002183F8461093F94440214916
:1080B800A24219D191F84740B4B10C31002494423E
:1080C80006DA51F8046F1C4D25F814600134F6E700
:1080D8000C2805D01849002421F810400130F7E792
:1080E800164801780131017083F8452000220121EA
:1080F8001A7083F8471070BD92F84710C9B140F262
:10810800DA51A0F2EF248C4208D811780B2905D84F
:108118000B1D0131117042F8230070BD002283F855
:108128004720074B03F13002002143F8041F934214
:10813800FAD170BD04010020A430002034060020CC
:1081480010010020024A136C01331944116470476E
:1081580004010020024B53F820301B681980704737
:10816800981F0020074BA1F57A7153F820301A6840
:108178001B8959434FF47A7391FBF3F189B211804B
:10818800704700BF981F00201FB50123ADF80830C5
:10819800ADF80410002301A9ADF80A30ADF80C3091
:1081A800ADF8062007F01FFB05B05DF804FB38B5F5
:1081B800A0F513746379A579DB0745D594F83832AF
:1081C80005F00105F3B1226B1068838DC3F34E03EC
:1081D800838494F83C3223B1B4F842320133A4F8D2
:1081E8004232917A6A00FFF7CFFF012384F83B32CD
:1081F800002384F8393284F83A3284F83832A4F803
:10820800403238BD94F83B322046012B04BF94F825
:10821800393284F83A32FFF7EBFE94F83B22236BAD
:108228003AB9012284F83B221868997A05FA02F2D1
:1082380007E0002284F83B2295421868997A08BF23
:108248000222BDE838409FE738BD10B5A0F512748A
:1082580094F83C22BAB9A36A616A994228D0591C99
:10826800A069A162C35C2069DBB25B0043F40073C0
:108278008142A4F83E324FF00A0384F83D3228BF09
:10828800A262012312E094F93D327BB1B4F83E12A8
:1082980020464B08A4F83E3201F00101FFF7BDFE6D
:1082A80094F83D32013B84F83D3201E084F83C32D9
:1082B80094F83832002B4ED194F839320133DBB2BE
:1082C800092B84F8393203D12046BDE810408FE6E7
:1082D8000A2B40D194F83B322BB9B4F8403243F022
:1082E8000103A4F840326379D9071CD5B4F84002D9
:1082F800820501D4C30705D4B4F844320133A4F885
:10830800443210E0E36AC0F347000BB198470AE033
:10831800E3696269D054E369E1680133B3FBF1F2C0
:1083280001FB1233E361012284F8382294F83B22DE
:108338000023012A84F839320DD1A27984F83B321E
:10834800236B12F0010F1868997A0CBF02220022E1
:10835800BDE8104018E710BDF0B5046D8279A38917
:10836800467923F4005312F0020F4FEA03434FEA11
:1083780013430CBF00214FF4005112F0040FA381E6
:1083880014BF4FF4806E4FF0000E16F0010F87688F
:10839800054614BF04200020B307238A48BF40F0D5
:1083A80008029BB223F4405343EA01032382A189C4
:1083B80048BF90B289B221F4B05121F00C014EEAC5
:1083C800010140EA0102A281A38A87B023F4407325
:1083D8001B041B0CA38201A807F0A4F9039B049EAD
:1083E800254A944218BF1E46A389192272431BB21C
:1083F800002BB4BF7E00BE00B2FBF6F66427B6FBC6
:10840800F7F00001010907FB1163A28912B2002AE3
:10841800B7BFD9001A013231B1FBF7F2A7BF323228
:10842800B2FBF7F302F007021043A8BF03F00F03F3
:10843800AA79A8BF184380B212F0010F20812B6DD2
:1084480006D00E498B4202BF042001F5484108615D
:1084580012F0080F9A8A0BBF22F0080292B2120497
:1084680042F0080208BF120C9A829A8992B242F42A
:1084780000529A8107B0F0BD003801400044004026
:108488002DE9F04F504C4FF4147685B08046914654
:108498001D4606FB0046274608B94C4B02E001285A
:1084A80004D14B4B33631033C6F834314FF4147393
:1084B80003FB08F3474AFC18FA500322627122466C
:1084C80003F59C733B44E162A36100214FF4807083
:1084D800D4F8343134324FF0010B62612162E1612A
:1084E800A162616284F83C1284F83912A4F842123D
:1084F800A4F84412C4F80890A571E060206184F8DB
:1085080038B284F8468258681B890222ADF80C30CC
:1085180003A910238DF80E308DF80F20019207F073
:10852800C3FD236B019A597B58681B898DF80E107F
:1085380003A9ADF80C308DF80F2007F0B5FD3046D3
:108548005946FFF76AFD322002F063F8224BD4F84F
:1085580034A11B681A46B2FBF9F1B1F5803F03D389
:10856800012AF8D95208F6E71C4A5046B3FBF2F242
:1085780089B2D2B205F072FE4FF4147000FB08F015
:10858800174B07EB000800F512703C180022C8F8DA
:1085980048325046214605F0A9FED8F8307015F04B
:1085A800010F0CBF022200223868B97AFFF7ECFDF0
:1085B8000C4B3846C8F84C32211D002205F096FEB7
:1085C800304605B0BDE8F08FCC19002070B901081D
:1085D80090B90108109D01086000002040420F007A
:1085E80053820008B781000803460A4690F84602FD
:1085F800D96A9B7944E71FB50123ADF808300023F9
:10860800ADF80C30ADF80A30084BADF804101B7803
:1086180001A9012B08BF0323ADF8062008BFADF858
:108628000C3007F0E0F805B05DF804FB000100200D
:1086380038B510F80E2C044650F8043C52B9012203
:1086480000F80E2C20F80C1C997A18680222BDE854
:108658003840D0E730F80C2C20F80A1C891A89B267
:1086680020F8081C074A10F80F0C002522F81010F3
:1086780004F80E5C1868997A2A46FFF7BCFF04F8DC
:10868800065C38BDA4300020044B53F820301BB1E1
:1086980007289CBF1B681980704700BF2C02002068
:1086A8002DE9F7438E460546DFF8A092114699F862
:1086B800A0440068164698467246631C89F8A034A0
:1086C80005F078FD2B8901A9ADF8043018238DF841
:1086D8000630686802238DF8073007F0E5FCAB7AAE
:1086E80009F2A447240127442A6849460C2B00F2C2
:1086F800F680DFE813F00D00F400F400F4005100F8
:10870800F400F400F4008A00F400F400F400C2005D
:10871800138CDFF83CC223F001031B041B0C1384E9
:10872800138CB2F804E0108B624520F073004FEA16
:1087380000404FEA10409BB21FFA8EFE40F07000D6
:1087480014D00CF5006C624510D00CF5406C6245F5
:108758000CD00CF5806C624508D00CF5806C624535
:1087680004D023F0020343F0030307E023F00E03D1
:108778002EF4407E43F003034EF4807EA2F804E01A
:108788001083A2F834801384138B23F008031B048E
:108798001B0C43F0080336E0138CDFF8B4C123F058
:1087A80010031B041B0C1384138CB2F804E0108B09
:1087B800624520F4E6404FEA00404FEA10409BB281
:1087C8001FFA8EFE40F4E04008D00CF5006C6245BC
:1087D80004D023F0200343F0300307E023F0E00344
:1087E8002EF4406E43F030034EF4806EA2F804E09D
:1087F8001083A2F838801384138B23F400631B04BE
:108808001B0C43F40063138369E0138CDFF840C149
:1088180023F480731B041B0C1384138CB2F804E03C
:10882800908B624520F073004FEA00404FEA1040F9
:108838009BB21FFA8EFE40F0700008D00CF5006C59
:10884800624504D023F4007343F4407307E023F433
:1088580060632EF4405E43F440734EF4805EA2F8E9
:1088680004E09083A2F83C801384938B23F00803E0
:108878001B041B0C43F0080330E0138CDFF8D0C056
:1088880023F480531B041B0C1384108CB2F804E0EF
:10889800938B20F4005023F4E6431B0400041B0CC4
:1088A800000C62451FFA8EFE43F4E04340F440504A
:1088B80003D00CF5006C624503D12EF4804E4EF4C3
:1088C800804EA2F804E09383A2F840801084938B32
:1088D80023F400631B041B0C43F4006393832B7B7A
:1088E80043B1B2F844306FEA43436FEA53439BB253
:1088F800A2F8443013889BB243F001031380AB7A8B
:108908000C2B19D8DFE803F0071818180B181818DB
:108918000F18181813000B1902F134000AE00B198C
:1089280002F1380006E00B1902F13C0002E00B19D5
:1089380002F14000C3F8A40438460C44A4F8AC641F
:10894800C4F8A82403B0BDE8F08300BFCC19002008
:10895800002C0140084A13689B020BD5074B0021E5
:1089680019704FF6FE730649086803400B604FF410
:1089780000135360704700BF00000240813100209F
:108988006C000240F0B50124B0FBF4F58D4201D330
:108998004C43F9E70026D4B1B0FBF4F504FB15000D
:1089A800B4FBF1F41EB9002D01DC002CF3D1092D24
:1089B80003F1010EEFB204DD002A14BF3725572555
:1089C80000E030253D441D7001367346E3E71C7016
:1089D800F0BDF0B50124B0FBF4F58D4201D34C4352
:1089E800F9E70026D4B1B0FBF4F504FB1500B4FB9D
:1089F800F1F41EB9002D01DC002CF3D1092D03F18F
:108A0800010EEFB204DD002A14BF3725572500E018
:108A180030253D441D7001367346E3E71C70F0BDF8
:108A280003685A1C0260197070472DE9F843089EC4
:108A3800002B074688461446334614BF4FF03009CA
:108A48004FF0200913F8012B0AB9254603E0002C42
:108A5800FBDD013CF6E7002D04DD38464946C047FA
:108A6800013DF8E7354624EAE474A01B284415F8CC
:108A7800011B11B13846C047F7E7BDE8F883024B40
:108A8800186801F078BE00BFE80F0020F8B5074667
:108A98000C464868002115461E460BF045F958B1AA
:108AA80028460AF059FF10490AF0AAFF01464FF07C
:108AB8007E500BF059F86060616830460AF098FE05
:108AC800014630460BF050F82568064629463846D8
:108AD8000AF08CFE014630460AF092FF014628460D
:108AE8000AF086FE2060F8BDDB0FC9402DE9F04191
:108AF80002780346202A00F10100F9D0092AF7D0AC
:108B08002D2A02D10346414D04E02B2A08BF034613
:108B18004FF07E551C460026234614F8012BA2F17F
:108B28003007F9B209290DD8394930460AF068FFEB
:108B3800064638460AF010FF014630460AF058FE4D
:108B48000646E9E72E2A17D1314F234614F8010BC0
:108B58003038C2B2092A0FD80AF0FEFE39460BF0A7
:108B680003F8014630460AF043FE294906463846CE
:108B78000AF046FF0746E8E71A7802F0DF02452ABE
:108B880039D15A782D2A02D10233012704E02B2A41
:108B980014BF013302330027013B002413F8012FCF
:108BA800303AD1B2092903D80A2101FB0424F5E798
:108BB800B4F59A7F28BF4FF49A74A0464FF07E53BD
:108BC800B8F1070F07D9184612490AF019FFA8F19A
:108BD80008080346F4E704F0070434B118460C49C2
:108BE8000AF00EFF013C0346F7E719462FB130465D
:108BF8000AF0BAFF04E04FF07E5130460AF000FF59
:108C0800014628460AF0FCFEBDE8F081000080BF5E
:108C18000000204120BCBE4C30B5054687B00C464C
:108C280003A800210C220EF030FA284600210BF090
:108C3800A3F820B1284628490AF0DAFD03E02846BF
:108C480025490AF0D3FD25490AF0DAFE0BF09EF813
:108C5800054680EAE0706946A0EBE57009F016FE6B
:108C6800002DACBF20232D2368468DF80C300EF064
:108C780050FA012807D130238DF80D308DF80E30C9
:108C88008DF80F300CE0022805D130238DF80D3017
:108C98008DF80E3004E0032804BF30238DF80D3022
:108CA800694603A80EF018FA03A80EF032FA033842
:108CB800C5B22A4603A920460EF056FA002363558A
:108CC800204607490EF008FA03AB204659190EF062
:108CD80003FA204607B030BD6F12033A00007A4409
:108CE800E8BE010870B50646B6FBF2F4084615461C
:108CF80014B12046FFF7F6FF05FB1464024B1B5D19
:108D080000F8013B70BD00BFEABE01082DE9F04F35
:108D180081468A4616461C4689B0002531780029C6
:108D280000F0DB80252902D00136484674E07278CD
:108D38004FF00008302A0CBFB278B71CA2F13003FC
:108D480012BF4FF0000BF71C4FF0010B092B19D87D
:108D5800A2F13003D9B2092905D80A2202FB083842
:108D680017F8012BF4E7A2F16103052B02D8A2F151
:108D7800570305E0A2F14103052B03D8A2F13703FD
:108D88000A2BEADD6C2A30D13A787E1C642A00F07E
:108D980083800BD8252A3DD003D8002A00F09D8077
:108DA800BCE7582A0CD0632A19D0B7E7732A22D017
:108DB80002D86E2A37D0B1E7752A5CD0782AADD1AF
:108DC800271D2068A2F1580462424FF01001624149
:108DD80055E02CD9582A32D0632A2AD13E46484633
:108DE8002178271DD04701350FE0642A63D00ED9BA
:108DF800732A14D13E46236848460093514642469A
:108E08000023FFF712FE271D05443C4686E7252A66
:108E1800DFD13E4648462521D04701357EE70AD8AE
:108E28006E2A06D13E46236804341D6076E7002A80
:108E380053D03E4672E7752A26D0782AF9D1A2F196
:108E4800580304F1040C5A422068CDF80CC04FF0C6
:108E580010015A4105ABFFF795FDDDF80CC03E4601
:108E6800644605AB00934846514642465B46FFF7C9
:108E7800DCFD054452E72068271D0A21002205ABC6
:108E8800FFF7A7FD3C46ECE704F1040CCDF80CC055
:108E980020680A210022DDE72068271D002808DA5B
:108EA8002D238DF8143040420DF115030A210022BC
:108EB800E6E705ABFAE7206804F1040C00280ADAB3
:108EC8002D238DF8143040420DF11503CDF80CC058
:108ED8000A210022BFE705ABF8E7284609B0BDE83C
:108EE800F08F0EB40FB505AB53F8042B019006496B
:108EF80001A80393FFF70AFF019B00221A7004B030
:108F08005DF804EB03B07047298A00080FB413B565
:108F18000B4904AB08680B4953F8042B0968019303
:108F2800FFF7F4FE0446084B186801F018FC002807
:108F3800F9D0204602B0BDE8104004B0704700BF29
:108F4800DC000020D8000020E80F002080EAE07351
:108F5800A3EBE0738B4206DB002801DD401A704763
:108F680002D0084470470020704770B504460AF0E4
:108F78000DFF2030402857D820462C490AF0FCFE27
:108F880028B120462A490AF031FC0446F4E7204675
:108F980028490AF0D3FE28B1204625490AF028FCC2
:108FA8000446F4E7204624490AF0E6FE30B1224997
:108FB80020460AF01BFC01461F480AE020461F49CC
:108FC8000AF0BCFE40B11C4920460AF011FC0146DB
:108FD8001A480AF00BFC0446214620460AF010FD08
:108FE8000546204629460AF00BFD1549064628463F
:108FF8000AF006FD13490AF0F9FB014628460AF073
:10900800FFFC11490AF0F4FB014628460AF0F8FC77
:109018000E490AF0EBFB014630460AF0F1FC014626
:1090280020460AF0E5FB70BD002070BDDB0F49400B
:10903800DB0FC940DB0F49C0DB0FC93FDB0FC9BFDE
:109048009A7C2E36FAAF4F393587083CA4AA2A3EB7
:1090580008B503490AF0CCFBBDE8084085E700BF26
:10906800DB0FC93F2DE9F04F056885B081462846DA
:109078000C46FFF7EDFF80462846FFF776FFD9F844
:10908800045006462846FFF7E3FF07462846FFF741
:109098006CFFD9F8089005464846FFF7D9FF824685
:1090A8004846FFF762FF4146814650460AF0A8FC51
:1090B8004146834648460AF0A3FC51460190304693
:1090C8000AF09EFC4946029030460AF099FC39465F
:1090D800039050460AF094FC4946206007F100408E
:1090E8000AF08EFC29466060A56002980AF088FCA8
:1090F800014601980AF07CFB2946E06003980AF0D3
:109108007FFC014658460AF071FB3946206106F19A
:1091180000400AF075FC2946606158460AF070FC68
:10912800014603980AF062FB2946A06101980AF0FB
:1091380067FC014602980AF05BFB4146E06138464D
:109148000AF05EFC206205B0BDE8F08F2DE9F04121
:1091580007688AB0466885680446084601A9FFF78B
:1091680081FF019938460AF04BFC04998046304645
:109178000AF046FC014640460AF03AFB0799804649
:1091880028460AF03DFC014640460AF031FB0299A8
:10919800206038460AF034FC0599804630460AF0CB
:1091A8002FFC014640460AF023FB089980462846D2
:1091B8000AF026FC014640460AF01AFB0399606053
:1091C80038460AF01DFC0699074630460AF018FC96
:1091D800014638460AF00CFB0999064628460AF06B
:1091E8000FFC014630460AF003FBA0600AB0BDE858
:1091F800F081074B10B51A881C4622EA00009042FD
:10920800188002D0012001F059FA208810BD00BF53
:10921800C0190020064B10B51A881C46104390420E
:10922800188002D0012001F049FA208810BD00BF43
:10923800C0190020024A936823EA00009060704732
:109248000811002008B5104B1A780023D9B29142B2
:1092580007D20E49002051F823100133096808800D
:10926800F4E7322001F0D5F9094B1B685A0309D5F8
:10927800084B9B685B0305D4BDE8084040F2DC500E
:1092880001F0C7B908BD00BFC81F0020981F002003
:10929800542D0020081100202DE9F7434E4F4F4A66
:1092A8004B233B706923137040F2DC735380BE2359
:1092B8001371EF2382F8D93700231946164682F82E
:1092C800DA37F25C0133514040F2DC729342F8D154
:1092D800424B434A83F8DA17424B4FF004085A606E
:1092E80002F188325A60002008F1FF3818F0FF08B0
:1092F8005FD03C4B3422DA60002454B100234FF491
:10930800005056F80490019306F05CFA0428EBD15B
:109318001DE04FF4302006F055FA0428E4D1314D11
:109328004FF430202B6943F002032B612E4B6B6105
:109338002B6943F040032B6106F044FA41F6FD73B4
:109348002A69042803EA02032B61D7D0CCE7254D0C
:109358001FFA89F22B694FF4005043F001032B6187
:1093680004F1006303F57E331A8006F02BFA042813
:1093780014D11E4B4FEA194923440193019B4FF422
:109388000050A3F8009006F01DFA41F6FE732A6912
:10939800042803EA02032B6106D0A5E741F6FE7311
:1093A8002A6913402B619FE740F2DC7304349C4226
:1093B800A3D10C4A0428136943F08003136102D136
:1093C80007F0F2FD10B90A2001F090F902233B7072
:1093D80003B0BDE8F08300BF350E0020081100205F
:1093E800230167450020024000F8030802F803083B
:1093F8002DE9F84307F0D8FD10B90A2001F076F9F5
:10940800BC4CBD4E4B23BD4940F2DC722046337044
:109418000DF030FE94F8B0374FF4CC71022B84BFB6
:10942800002384F8B03794F8B027B54D01FB02F358
:1094380003F53A7020442344286093F83C0301FB69
:109448000242022803F54E7384BF0020187192F877
:109458003C33AC4A13700C2202FB0343AA4A03F2C2
:10946800B273136046F20902A3681A401AB9A14AF6
:1094780043F400539360A368DF0703D54FF400500B
:10948800FFF7D8FEA368580409D50820FFF7D2FED5
:109498004FF40050FFF7CEFE0120FFF7CBFEA36884
:1094A800190706D54FF40050FFF7C4FE0120FFF757
:1094B800C1FEA3689A0413D54FF40040FFF7BAFE23
:1094C8008C4B93F88631012B03D14FF40060FFF7E2
:1094D800B1FE4FF48030FFF7ADFE4020FFF7AAFE43
:1094E800A3685B0603D54FF48030FFF7A3FE94F81A
:1094F800E021804B2AB193F8E42112B1002283F8CD
:10950800E4214FF00008C646804F814B1F6004EBF2
:109518000803B3F8F8C14FEA5C0101F077314FEA6C
:109528009C0303F03333C1EB0C00C11A4FEADC0390
:1095380003F01133CB1A03EB231303F00F32FF238D
:1095480092FBF3F31CF00109C3EB032318BF0EF1E0
:10955800010EA2EB030318BF5FFA8EFE012B0ADD92
:10956800022B40F0C480B9F1000F00F0C0801CF05D
:10957800BC0F00F0BC8008F10808B8F1200FC6D174
:109588000EF1FF3EBEF1010F00F2B18007F0E9FCD9
:10959800302200215F480DF078FDDFF8E8815E4B4E
:1095A800D5F80090C3F800805C4B002109F17900E0
:1095B800C3F8009000F034FF594B80F00100187098
:1095C800584B08F126021A60574B08F1D4021A606A
:1095D80099F8000001F0C2FE2868544B00F5C572E6
:1095E8001A6003F0EDFC524B94F8D81108F194027C
:1095F8001A6064224A434F4BC8325A6000229A606C
:10960800DA601A615A619A61DA6183F8202083F876
:109618002120494B2D6808F12C021A60474B05F2AE
:1096280019121A60464B05F289121A60454B08F167
:1096380008021A60444BDFF85091C3F80080434B8E
:1096480008F1A0021A6008F1AA03C9F80030404BDB
:10965800B4F866011F600AF07BF9C9F80800B4F88D
:1096680068010AF075F995F85C3009F1040289F887
:10967800043095F87830C9F80C0089F8053094F86A
:10968800E331286E89F81030324BC9F814501A604B
:10969800314B05F164021A6030490AF0B1F901460C
:1096A8004FF07C500AF060FAB5F816412C4B186060
:1096B80020460AF051F901462A480AF055FA2A4983
:1096C8000AF09EF9294A2A4B15602A4A186005F1C2
:1096D80068031360284A05F211151560274AC2F875
:1096E8000080274A136002233370BDE8F88305F031
:1096F800C1FE4BE708110020350E002000F80308D2
:1097080038100020002D0020601000209212002048
:109718004C310020EC0E0020200F0020240F0020E8
:109728000C0000200421002000060020300F00203B
:10973800E82F0020C42F0020602100208C29002061
:10974800640900206C200020702000207808002088
:109758003C09002094210020CC210020DB0F494047
:10976800C8210020000061444C3D0F4498070020A8
:10977800740800208C070020640800206C08002072
:10978800940600204C120020301F002008B5FFF777
:1097980083FDFFF72DFEBDE80840012000F08EBFD5
:1097A800F8B504460E4617460025204620210DF040
:1097B800A2FC0446D0B1013420460DF0FFFCB0F500
:1097C800617F05DB40F634039842A8BF184601E0E4
:1097D8004FF46170A0F56170192390FBF3F00DB997
:1097E800307000E070703B7801333B700DB9012593
:1097F800DBE72046F8BD30B505460C46134629463A
:109808002246BDE830400148FFF780BBE0BF0108B1
:109818007FB504780646E4B9354B1921186800EB82
:10982800840090F87B5090F879204D4305F56175D8
:1098380090F87A30009590F87C00414301F5617109
:1098480001912C4821460134FFF760FB142CE3D129
:109858004BE00DF0B3FC1328054641DC244B701C8B
:109868001C68202100238DF80F300DF044FC1E35B4
:10987800064670B1013630460DF0A0FC1A289FBF8D
:1098880004EB850358709DF80F30013398BF8DF8AD
:109898000F30304620210DF02EFC064670B10136FF
:1098A80030460DF08BFC0D289FBF04EB85039870A4
:1098B8009DF80F30013398BF8DF80F3004EB850405
:1098C8003046E11C0DF10F02FFF76AFF9DF80F30DB
:1098D800042B0AD0601C002104220DF0D6FB04E002
:1098E800054800211322FFF786FF04B070BD00BFB2
:1098F80038100020FFBF010814C00108014808F013
:1099080023BB00BF1AC001082DE9F04304788FB0CB
:109918000546002C59D17B4B0021142209A807AE1B
:10992800D3F800800DF0B1FB0722304600210DF07E
:10993800ACFB00231A46A70005A8059308EB07050A
:1099480083807149B5F802E031F813C01CEA0E0FA4
:109958000AD00E310DF1380C595C02F1010E624447
:1099680002F81C1C5FFA8EF20133072BE9D10021A3
:109978000B46664AB5F802E011F802C01CEA0E0F61
:109988000AD006320DF1380C8A5C03F1010E6344EB
:1099980003F8242C5FFA8EF301310629E9D118F86F
:1099A80007308DE841006A785949029209A81A09D6
:1099B80003F00F03FFF795FA2146564809AA013428
:1099C800FFF7A4FA202CA6D198E00DF0F7FB1F288A
:1099D800044600F3868028462021E4B20DF08BFB74
:1099E8001F2C02D9FFF78AFF88E0464B451C1B68ED
:1099F800002103EB8404204604220DF046FB0027D7
:109A0800454B09AE304600210A2217F803905FFA49
:109A180087F80DF03AFB002315F8012B32B10A2B19
:109A280004D04A4502D0F2540133F5E74A455ED1E5
:109A380008F1FF33032B09D8DFE803F01005023FD4
:109A48000DF1230134E00DF123011EE030460DF045
:109A5800B5FB2378C0B243EA001006E030460DF0AB
:109A6800ADFB237800F00F001843207031E001337C
:109A7800062B0AD0244800F11B069E5D9642F6D1BB
:109A880003445A7D63881343638011F8012F02B39E
:109A98000023EFE70133072B0AD01B4800F10E061D
:109AA8009E5D9642F6D130F8132063881343638095
:109AB80011F8012F6AB10023EFE730460DF07EFB65
:109AC8000F2804DC30460DF079FB607001E00023BC
:109AD80063700137052F93D1012406F06BFE6CB932
:109AE80080E70E4800211F22FFF785FE06E020468A
:109AF800002104220DF0C9FA0024EEE70FB0BDE8FA
:109B0800F08300BF481F0020289D01083D9D0108E3
:109B180028C0010837C00108499D010814C0010880
:109B2800F8B50478064674B9304D2146B5F8C62113
:109B3800B5F8C8312E480134FFF7E8F9042C05F1CF
:109B48000405F2D1F8BD2B490DF0A8FAA8B9274BA6
:109B58004FF47A714FF4FA62A3F8C611A3F8C8213A
:109B6800A3F8CA11A3F8CC21A3F8CE11A3F8D021E9
:109B7800A3F8D211A3F8D421F8BD30460DF01EFB8E
:109B8800032805462BD8304620210DF0B4FA0446A8
:109B980030B1013420460DF011FB0126074600E0E4
:109BA8000646204620210DF0A6FA10B9BDE8F84077
:109BB800A4E601300DF002FB012EF7D140F2DC5390
:109BC800A7F2EE229A42F1D8A0F2EE229A42EDD8FC
:109BD800064B703503EB8503DF801881F8BD064816
:109BE80000210322BDE8F84005E600BF0811002067
:109BF80043C0010856C00108D5CC01082DE9FF4132
:109C080004780546002C34D16D4808F09DF96D4D57
:109C1800686900210AF088F8002840F0CE802146C3
:109C28006948FFF773F968696946FEF7F5FF014669
:109C38006648FFF76BF9A8696946FEF7EDFF01462C
:109C48006248FFF763F9E8696946FEF7E5FF0146F0
:109C58005E48FFF75BF9286A6946FEF7DDFF0134C5
:109C680001465B48FFF752F90C2C05F11005CFD1DE
:109C7800A3E0584905220DF055FA38B9514B002296
:109C880003441030C0285A61F8D196E0284652495A
:109C980004220DF047FA04462846002C3FD1202123
:109CA8000DF029FA002800F08880451C28460DF0A0
:109CB80030FA0746494B53F824601EB9484808F063
:109CC80043F97AE028463146FAB20DF02BFA01340E
:109CD8000028EFD13B4B0021C2181030C028516139
:109CE8009E46F7D13F4B03EBC402D2F804C0984616
:109CF800BCF1000F04D131463B48FFF707F953E0A8
:109D0800002718F834309F42F5DA3B010EEB0305C3
:109D1800143563440FCB013785E80F00F1E70DF0E8
:109D28004DFA0B28064643DC284620210DF0E3F9BE
:109D3800054648B101352846FEF7D8FE214B0124D7
:109D480003EB0613586100E00446284620210DF075
:109D5800D2F9054640B101352846FEF7C7FE194B32
:109D6800013403EB06139861284620210DF0C3F94E
:109D7800054640B101352846FEF7B8FE114B0134BF
:109D880003EB0613D861284620210DF0B4F910B969
:109D9800FFF7B4FD11E00130FEF7A8FE094B032CD4
:109DA80003EB06163062F3D11048FFF727FF04E0F3
:109DB8000F4801210C22FFF71EFD04B0BDE8F08119
:109DC8005CC001080811002077C001087DC00108A7
:109DD800EFC9010856C0010881C0010868B8010828
:109DE80086C0010810BF010895C001086BBD0108B5
:109DF80014C00108F0B5047887B0064614BB514B6F
:109E080019201968062303FB041191F8CA5091F828
:109E1800CE20454305F5617591F8C930009591F854
:109E2800CB50C831684300F5617001900879029001
:109E380049794548039121460134FFF767F80C2C0E
:109E4800DDD17CE00DF0BAF90B28044672DC3D4BFD
:109E5800701C1D68202100238DF817300DF04BF978
:109E6800064680B1013630460DF0A8F903289FBF99
:109E7800062303FB045383F8CE009DF817309CBFDC
:109E880001338DF81730304620210DF034F907469C
:109E980080B1013738460DF091F90D289FBF062390
:109EA80003FB045383F8C9009DF817309CBF0133A6
:109EB8008DF8173006266643A9193846CA310DF1C0
:109EC8001702FFF76DFC20210DF015F9074670B158
:109ED800013738460DF072F914289FBF9DF81730E6
:109EE8007619013386F8CC0098BF8DF817303846BC
:109EF80020210DF000F978B101300DF05FF90D283F
:109F08009FBF062303FB045383F8CD009DF8173049
:109F18009CBF01338DF817309DF81730062B0ED0F3
:109F2800062202FB04500021C9300DF0AEF8FFF7FD
:109F3800E5FC04E0054800210B22FFF75CFC07B0B4
:109F4800F0BD00BF38100020A1C0010814C00108EE
:109F58002DE9F347047807464CB9204601A908F0D3
:109F680095FC0134FFF7F4FF122CF6D17FE00DF0D9
:109F780025F9C5B2112D75D83E4C05F1D00604EB74
:109F88004603781C202193F802800DF0B4F83A4F6C
:109F9800034630B9A8F10202D2F1000848EB0208E2
:109FA80048E007F1260800F1010A597840460DF00B
:109FB800A2F868B1032D8CBF03230023C8EB00006F
:109FC800C0B23B44184490F82A90B9F1030F02D16B
:109FD800FFF794FC4BE0A9F10203D3F100085046C7
:109FE8004FF0200148EB03080DF085F8D8B1B8F11F
:109FF800000FEDD001300DF0E1F840F2ED2380B212
:10A00800984205DD40F6CA039842A8BF184601E009
:10A0180040F2EE20A0F2EE20192290FBF2F004EBC1
:10A028004603D87002E0B8F1000FD1D104EB460323
:10A0380083F8029004EB4604A3781F4497F826207F
:10A04800B8F1000F09D0E17819234B430B48294692
:10A0580003F2EE23FEF75AFF09E029460848FEF707
:10A0680055FF04E0074800211122FFF7C4FB02B0A6
:10A07800BDE8F08708110020289D0108C1C001082B
:10A08800D3C00108D5CC010810B50446204600F01D
:10A0980066FB18B90A2000F0BCFAF7E710BD0022E9
:10A0A80007490C2303FB02135968814204D100229B
:10A0B800C2621A725A6070470132042AF0D170479E
:10A0C800802A00202DE9F743064689469DF8288016
:10A0D80011461A469DF82C3000250C2068431A4F6B
:10A0E800C419C057B04202D1207A20B126E0013508
:10A0F800042DF2D122E0012E0AD003DCF6B9009338
:10A10800124807E01E2E0AD01F2E17D1012006E0A4
:10A118000F480093434604F06DF9044605E0FEF746
:10A12800AFF94146044600F017FB4CB10C2303FB82
:10A138000575267185F808906C6001E0002000E044
:10A14800204603B0BDE8F083802A00200038014093
:10A158000044004010B5084B0022196801EBC20307
:10A1680093F90240844201D1981C10BD0132042A9F
:10A17800F4D1002010BD00BF7C2A0020F0B5027881
:10A1880087B08AB94A4C04F1200694F8F6210023D6
:10A19800484950B2595681426ED00C33302BF7D112
:10A1A8000834B442F1D181E0002204920592451CA2
:10A1B8000DF004F8C4B260B2FFF7CCFF074618B13F
:10A1C8008DF81040012400E00446284620210CF0B8
:10A1D80092FF054638B1013528460CF0EFFF0134EF
:10A1E800ADF81200E4B20026284620210CF083FFC7
:10A1F800B0B3451C28460CF0E1FF00222E495FFA57
:10A2080082FE51F82230834204D00132082AF5D167
:10A21800002300E0734651F82320824220D1022E09
:10A228000FD0032E12D05A1E012ED2B204D0042A07
:10A2380013D88DF814300EE0042A0ED88DF8153096
:10A2480009E0052B09D88DF8173004E09A1E052A75
:10A2580003D88DF816300134E4B20136042EC3D188
:10A26800052C04D807B0BDE8F040FFF747BB04ABA6
:10A2780003CB3860796019E094F8FB010E4B94F831
:10A28800FA5153F82000B4F8F821009094F8FD0131
:10A2980053F82000019094F8FC0153F8200053F87B
:10A2A800253002900548FEF731FE79E707B0F0BD8A
:10A2B80008110020802A002034A60108E2C0010805
:10A2C80038B1438811EA030003D08B420CBF012048
:10A2D8000220704730B50A4B0A491C680A79032ADC
:10A2E8000AD81346551C04EBC303EAB29D882842DA
:10A2F800F5D00A71981C30BD0A71002030BD00BF2E
:10A308007C2A0020481F0020014B00221A71E1E737
:10A31800481F00202DE9F047877890F803C0BBB2AA
:10A32800C7F1640E03EB83065C42C3F178001C4D51
:10A338005FFA8EFE7600CCF16408A4B280B2A3B2B4
:10A348000FFA83F9B9F1000F04DC002B14BF3B4668
:10A35800012300E0734609FB09F25B4302FB0CF2A0
:10A3680092FBF3F3434403FB09F30A2293FBF2F352
:10A3780033449BB225F8023FB1F800904A880A346A
:10A38800C9EB020A1AB202FB0AF24FF47A7392FB83
:10A39800F3F3A4B24B4484422B80D0D1BDE8F087BC
:10A3A8004C1F002010B544780078002240F6C411F4
:10A3B80002FB02F3193B634303F6C41353434343BD
:10A3C80093FBF1F3034921F812300132072AEDD14A
:10A3D80010BD00BF661F0020104B043033F9100079
:10A3E800B0F5617F05DB40F633039842A8BF1846F5
:10A3F80001E04FF461700A7819235A4302F283325C
:10A40800824208DA4A78534303F283338342B4BF63
:10A418000020012070470020704700BF902D0020C9
:10A4280010B500F1500302788A4203D18478C278CB
:10A43800944204D304309842F5D1002010BD012085
:10A4480010BD0B4B1B6813F4805F0A4BB3F9063041
:10A4580005D0C089421A934207DD084400E0008A0B
:10A468008342B4BF0020012070470120704700BF1D
:10A47800542D0020902D0020034B4FF4805208B13A
:10A488001A6170475A61704700080140034B4FF446
:10A49800805208B15A6170471A617047000801403C
:10A4A8002DE9F74F2F4C054627683846FEF7D0FDB3
:10A4B80006463846FEF759FD676881463846FEF776
:10A4C800C7FD01903846FEF750FDD5F804A00746B1
:10A4D8003146504609F094FAD5F808808346494633
:10A4E800404609F08DFA0146584609F07FF9019B6C
:10A4F80029688346184609F083FA494605465046B6
:10A5080009F07EFA394609F07BFA0146284609F037
:10A518006FF939460546404609F072FA314609F0A6
:10A528006FFA0146284609F063F9014658460DF0CE
:10A5380091F80D4909F064FA0C4909F015FBA16876
:10A5480009F056F90A4909F00FFB0CF0ABFF83B28A
:10A558001A0444BF00F5B47083B218B203B0BDE862
:10A56800F08F00BF741F00200000E144DB0F49405A
:10A57800000020411FB5084B1B681B0309D58DF847
:10A588000400039101230D2001A98DF80530FDF782
:10A598001DF905B05DF804FB542D00201FB5084BCC
:10A5A8001B681B0309D58DF80400029100230D20B8
:10A5B80001A98DF80530FDF709F905B05DF804FB30
:10A5C800542D002010B50A4A0A4B11689B6800BF39
:10A5D80012689142F7D1084A4FF47A70D46800FBA8
:10A5E80004F2D31AB3FBF4F300FB013010BD00BF33
:10A5F800782D002010E000E0741F002038B50446D4
:10A60800FFF7E0FF0546FFF7DDFF401BA042FAD346
:10A6180038BD10B504462CB14FF47A70FFF7EEFF41
:10A62800013CF8E710BD024A136801331360704714
:10A63800782D0020024B1B6903B11847704700BFF3
:10A64800741F0020014B1B68184700BF68310020A9
:10A6580010B50020FFF7F6FF054B00241C7009F029
:10A6680083F8044B1C759C619C831C6210BD00BF61
:10A6780050310020741F002010B510B9BDE81040FB
:10A68800E6E700230C225A430A4C1119125D824254
:10A6980003D00133102BF5D110BD074B186A18B140
:10A6A8004A784078824203D2002219629A839A61DA
:10A6B80010BD00BF0CAA0108741F002010B540008F
:10A6C8001428A8BF14200023074A022199540B44D8
:10A6D80099181424834201F8014CF5DBFF21D15469
:10A6E8000F20BDE81040C7E72C2D002038B540F2F8
:10A6F800DB156843134B10225A6108221A61851E24
:10A708000B24013C14F0FF0415D00E4B2846DA68E0
:10A7180082F01002DA60DA6882F00802DA60FFF785
:10A7280078FF0120FFF78EFF1920FFF772FF002046
:10A73800FFF788FFE5E7044A044B1A60044A054B13
:10A74800DA6038BD000C0140EFBEADDEF04F0020EE
:10A758000400FA0500ED00E003685B691847036828
:10A768001B6918470368DB68184703689B68184724
:10A7780003685B68184703681B681847B0F902301C
:10A788002DE9F74F93421CBF0023037090F800A0F7
:10A7980004460E469146BAF1000F40F0AB801046D1
:10A7A80009F0DAF8864909F02BF9864909F028F901
:10A7B8004FF07C5109F024F90CF0D4FE014605460F
:10A7C80009F01EF980498346284609F019F903461D
:10A7D80058461946019309F00BF84FF07E5109F0DD
:10A7E80007F801464FF07E5009F0BEF92946804629
:10A7F80009F006F9294609F003F9074601466060A1
:10A8080008F0F6FFE7604FF07E572946A060276101
:10A81800284608F0EDFF294609F0F2F84FF080418C
:10A8280008F0E4FF0146404609F0EAF8019B606140
:10A838001946584608F0DAFF394608F0D9FF0146AC
:10A84800404609F0DDF840F2DC53A046274655465D
:10A8580063651023A4F852301823A061A4F850307F
:10A868004FF09741D8F8100009F0CAF80021824645
:10A8780009F064FA28B150464FF07C5108F0B6FF51
:10A8880004E050464FF07C5108F0B2FF09F0E0FABE
:10A89800C7E90E014FF09741D8F8040009F0B0F865
:10A8A8000021824609F04AFA28B150464FF07C51FF
:10A8B80008F09CFF04E050464FF07C5108F098FFE8
:10A8C80009F0C6FA0135032DC7E9080108F10408A3
:10A8D80007F10807C4D1A6F2DC531B042367E3671A
:10A8E8006367C4F88030A367C4F884300123A4F8F0
:10A8F80002902370D4F85490B4F95280C9EB06063C
:10A90800636A06FA08F67343276A4FEAE67B206F04
:10A9180007FB0B332667A7FB0667E26F1F44636CD0
:10A92800D4F840C053434FEAE27B0CFB0B3ED4F80B
:10A938008010C4F88020ACFB02237344B61A67EB7E
:10A948000307E36AA26A43434FEAE07B02FB0B3E3C
:10A95800A2FB00237344B6185F41E36C656F4B4359
:10A968006067A06C4FEAE17B00FB0B33C4F88410EE
:10A97800A0FB01011944636B361A05FB03F3206B36
:10A988004FEAE57B00FB0B3367EB0107A0FB0501F2
:10A99800801919447941B4F95020A56708F014FFCB
:10A9A80008F1FF3201239340E067C01841EBE371DF
:10A9B800424608F009FF484403B0BDE8F08F00BFE5
:10A9C8006F12833ADB0F4940F404B53F2DE9F84391
:10A9D8000024244BE0B293F85460B0420CD203EB4D
:10A9E8008003214A5B6A32F810101BB10B2801D88A
:10A9F800DB6898470134ECE71C4B1B685B032ED5DA
:10AA080000242346E2B2B24229D2DFF858904FEA36
:10AA1800840809F1240757F8242055689D4216D068
:10AA2800284603F045FCEFF31283502282F3128884
:10AA38002821AA8C01FB009092B20132C267AA8A2F
:10AA4800DBB292B242F00102AA8283F3118857F86E
:10AA5800083000221B6801341A802B46D2E7BDE873
:10AA6800F88300BF741F00203C100020542D0020E4
:10AA780008B50E4B1B6813F4805F0D4B14BFD3F859
:10AA8800F820D3F8FC2093F8541092880023D8B209
:10AA9800884204D2074820F813200133F7E7FFF76C
:10AAA80095FFBDE808403220B3E500BF542D0020D3
:10AAB800741F00203C1000200A4B30B51A680A4B5E
:10AAC80002F48052D3F8F840D3F8FC5000230AB1BE
:10AAD800A18800E0A988054820F8131001330C2B41
:10AAE800F5D130BD542D0020741F0020022D002008
:10AAF80070B5124D0024214605F20110702285F828
:10AB080000410CF0C2FA2146D5F874310B4A0B44C7
:10AB180093F9020088B11E6802F201140E51081957
:10AB28009C88073184809B797029837192F8003161
:10AB380003F1010382F80031E6D170BD741F0020D3
:10AB4800094B1A680E2303FB0020437AFF2B07D01A
:10AB5800064A12789A4203D9054A32F8130000E0EF
:10AB6800808800B2704700BF8C290020742A00201A
:10AB7800902D00202DE9F04F9D4C91B0D4F87C31F8
:10AB880005469C4898479B489B4E014694F88C2163
:10AB980004F0E0FF3388002B00F08680D4F8903171
:10ABA80004F5CA771B7804F5D07A02934FF00008B1
:10ABB800B6F800904FEA4803B9F57A7F02BF002241
:10ABC8003A60CAF810208B4A019332F918003A68A3
:10ABD80002443A6008F0C0FEDAF810200132012A77
:10ABE800CAF8102007D10022CAF80400CAF80000E9
:10ABF800CAF808202EE0DAF80030059219460393C7
:10AC0800049008F0F3FD059A8346104608F0A4FE68
:10AC18000146584608F0A8FF039B0146184608F06D
:10AC2800E7FD0246DDF810C01146CAF80400604688
:10AC3800039208F0DBFD0146584608F0E1FEDAF819
:10AC4800081008F0D5FD039ACAF80C00CAF80020CD
:10AC5800CAF80800019B6749DFF8B8B10022B9F1CA
:10AC6800010F5A5223F80B202AD1DAF810000128D4
:10AC780008DD013808F070FE0146DAF80C0008F02B
:10AC880073FF00E000200CF071FE029B73B103908B
:10AC9800184608F061FE039A0146104609F06CF860
:10ACA80020B14FF47A73338000231CE03A684FF4E4
:10ACB8007A7102F5FA7292FBF1F2019B2BF80320EC
:10ACC80008F10108B8F1030F07F104070AF1140AA3
:10ACD8007FF46EAFB9F1010F02D14846FFF7CCFC03
:10ACE8003388013BDFE7424E424906F5EE7031F802
:10ACF800132030F81300121A21F813200133032B04
:10AD0800F1D13E4B1B6813F0020300F00B833C4B60
:10AD180006F5F1705B6898473A4B06F5F1701A78BA
:10AD2800014604F017FFB6F8E83106F5F177002B75
:10AD380042D0D6F8EC010023B4F8E8214FEA830C9E
:10AD4800B2F5C87F304A04BF002142F8231037F912
:10AD580013E052F80C10264E714442F80C100021F2
:10AD680027F8131020F813100133032BE4D1B6F899
:10AD7800E831012B1BD1D6F8F0314FF4C87E03F12E
:10AD8800C80292FBFEF20280D6F8F421C83292FB88
:10AD9800FEF24280D6F8F8311C4AC83393FBFEF322
:10ADA80012889B1A838029806980FEF7EFFCB4F82B
:10ADB800E831013BA4F8E831154B1B685A0740F10C
:10ADC8008C80B4F8FC210A4B322A25D1D3F8EC2127
:10ADD8001188A3F8FE1151889288A3F80012A3F8ED
:10ADE80002222A88A3F804226A88A3F8062215E01A
:10ADF800741F00201C1000207A310020F818002051
:10AE0800202D002083310020642100202000002014
:10AE1800542D002050210020002A3ED0D4F8EC0107
:10AE28000023B4F8FC214FEA830E322AC24A04BF39
:10AE3800002142F8231037F913C052F80E10BF4E04
:10AE4800614442F80E10002227F8132020F813203E
:10AE58000133032B1146E4D1B6F8FC31012B17D18D
:10AE68000C2086F8142286F81532FFF705FCD6F870
:10AE7800EC31B6F8FE211A80B6F800225A80B6F8EE
:10AE880002229A80B6F804322B80B6F806326B801C
:10AE9800B4F8FC31013BA4F8FC3194F81632A74A07
:10AEA800DBB1D2F80832322693FBF6F3D2F8EC0184
:10AEB800002182F816120380D2F80C3293FBF6F3C5
:10AEC8004380D2F810329E4A93FBF6F312889B1AFD
:10AED800838029806980FEF759FCD4F8EC21B4F806
:10AEE800E23111884FF000085B1AA4F8E23151886A
:10AEF800B4F8E4315B1AA4F8E4319288B4F8E63186
:10AF08009B1AA4F8E631FFF75DFBD4F818620546F2
:10AF1800831B1846019308F01BFDD4F81C120290FD
:10AF280008F06EFDC4F818524546D4F82072854ED4
:10AF380097F800B00390844A0DF11C0A32F9150005
:10AF480008F00AFD039908F05BFD4AF82500BBF1FB
:10AF5800000F2BD0584608F0FFFC01464FF07E50FA
:10AF680008F002FE0246DFF8089211464FF07E50C4
:10AF7800059208F03BFC59F8251008F041FDA9F1AD
:10AF88004201049031F9150008F0E6FC059A1146D3
:10AF980008F036FDDDF810C00146604608F028FCD0
:10AFA80049F8250008F0F2FE708003E0674A32F89D
:10AFB8001520728036F9022F0135032D02FB028815
:10AFC800B9D1642303FB08F85D4B61481B8807A9C6
:10AFD8005B4398FBF3F8A8F149081FFA88F8FEF7D5
:10AFE800B5F8B8F13B0F7D6810D9544BB3F93C0262
:10AFF800D3F8385208F0B0FC0146284608F0BCFEE9
:10B00800544B68B31A7842F008022CE04FF07E5196
:10B01800284608F0EDFB01464FF07E5008F0A4FDED
:10B0280081464FF00008DFF828B128465BF8281061
:10B0380008F0E6FC484A039032F9180008F08CFC46
:10B04800039B0146184608F0D3FB494608F0D8FC94
:10B058004BF8280008F10108B8F1030FE3D1C4E761
:10B068001A7822F008022946D4F834021A700CF033
:10B07800F1FA81462060D4F83002D4F838B200F1F1
:10B088000045D4F83402014608F0BAFC5946804617
:10B09800584608F0B5FC0146404608F0A9FB0CF0FC
:10B0A80065FC014628460CF0D5FA2C4980466060BC
:10B0B800484608F0A5FC0CF0F5F9294D27492880E9
:10B0C800404608F09DFC0CF0EDF9264B68801B68A3
:10B0D8001B074FD5244807A9FEF738F8BD684FF07D
:10B0E8007E51284608F084FB01464FF07E5008F058
:10B0F8003BFD82464FF0000B1B4B284653F82B10A4
:10B10800049308F07DFC1949039031F91B0008F0FD
:10B1180023FC039A0146104608F06AFB514608F0E2
:10B128006FFC049B43F82B000BF1010BBBF1030FE1
:10B13800E2D1184655E000BF7C210020741F002092
:10B1480020000020E81000201C10002056210020BC
:10B15800A4210020FC180020EA1000204C3D0F44D8
:10B168004C2D0020F8180020B421002022100020C7
:10B1780098210020704D51462846FDF7E7FF2868C2
:10B188006B680146039308F03BFC039B8246194613
:10B19800184608F035FC0146504608F029FBD5F85A
:10B1A80008B082465946584608F02AFC01465046DF
:10B1B80008F01EFB0CF0DAFB0021824608F0B4FD13
:10B1C80070B92868514608F0CFFC51462860686875
:10B1D80008F0CAFC51466860A86808F0C5FCA86079
:10B1E8005548FFF75DF9554B55491880029808F006
:10B1F80007FC524B08F10048054609F10049B3F92C
:10B208000000CDF82C80CDF8289008F0A5FB4D491A
:10B2180000F1004008F0F4FBDFF83C810C90B8F92D
:10B22800000008F099FB0D90B8F9020008F094FBB3
:10B238000E90B8F9040008F08FFB0AA90F900DA82A
:10B24800FDF784FF7B78012B1AD13F4B3F4F1B78CA
:10B2580013F0040F0ED1D7F84C02402390FBF3F300
:10B26800C01A08F079FB0F9908F0C2FA08F08EFDB1
:10B27800C7F84C02D7F84C02402390FBF3F001E0EA
:10B28800334B188808F068FB01460F9808F0AEFAAF
:10B29800D4F854120F90284608F0AAFA0146284616
:10B2A80008F062FCD4F85072054639460F9808F049
:10B2B8009DFA0146284608F0A3FB0146384608F0E7
:10B2C80097FA0746C4F850020D980CF0EBF8D4F83A
:10B2D80058522978FDF73AFED4F85C321844C4F87D
:10B2E8005C020E980CF0DEF82978FDF72FFED4F8F2
:10B2F80060321844C4F8600238460CF0D3F8697814
:10B30800FDF724FED4F86432124A184401991368F0
:10B31800C4F864021944D4F8683211600133C4F8DF
:10B32800683205E0A6F8E231A6F8E431A6F8E6317D
:10B3380011B0BDE8F08F00BF24000020F8100020F5
:10B34800BD37863535FA8E3C82310020741F0020C7
:10B358002000002064310020EA10002001380A4B48
:10B36800042804D8DFE800F00507090B0D00074A98
:10B3780008E0074A06E0074A04E0074A02E0074AED
:10B3880000E0074A1A60704758000020A12C010805
:10B3980069B90008BD2F0108CDBF000829BC000805
:10B3A800F9C2000808B508480BF0B3FEC0B2092876
:10B3B8000246054B04DC01302021C0B29954F6E75F
:10B3C80000221A5408BD00BF6D24002008B50748A4
:10B3D8000BF09FFEC0B21428044B04D8421C202155
:10B3E8001954D0B2F7E700221A5408BD6D24002082
:10B3F8002DE9F74FFFF7E6F8A64C80462668656802
:10B40800A768861BF643451BC71BED43FF43F60F92
:10B41800ED0FFF0F2EB93FB9002D00F08782B94616
:10B428002CE04FF0000929E0B14627E003EB8A0B36
:10B43800BBF802301A050ED413F4805F1DBF964A7C
:10B448009BF801101268954A954B14BF52F82120B9
:10B45800126843F82A20BBF80230D80516D499059B
:10B468000AD5904B1B7813F0040F0CBF8E4A8F4AF5
:10B478008B4B126843F82A2009F10109207B5FFAF7
:10B4880089FA8B4982450B68D0D326E0894A504611
:10B49800594605F01FF9884B1B885A0603D55046B4
:10B4A8005946864A16E0580703D550465946844AF5
:10B4B80010E0190703D550465946824A0AE09A0710
:10B4C80003D550465946804A04E0DB07D4D5504698
:10B4D80059467E4A05F0FEF8CEE7DFF808E2009309
:10B4E800BEF906307822A3F57A7353434FF47A7283
:10B4F80093FBF2F3F34603F22B13019300225FFA56
:10B5080082FE864517D2009B03EB820EBEF802E04E
:10B518001EF4806F0DD040F2671ADFF88491019B0A
:10B5280039F822E09E449EFBFAFC0AFB1CEE29F83F
:10B5380022E00132E3E74DB308F5C333A03363607B
:10B54800637B544A13BB9373614B1B6813F0020F60
:10B558000AD0DFF894E19EF800E0BEF1000F03D0B6
:10B568004FF0010E82F80EE0DA0506D5594BDB786C
:10B578001BB1A37B43F00203A3734A4B1B7813F060
:10B58800050F02BFA37B43F00403A37394F80EE0F6
:10B59800BEF1000F03D13F4B5B7B002B4FD094F8DB
:10B5A8000DC01CF0010FACF10C031DD1BCF1030F51
:10B5B80007D8DFF8E8901EF0040F3B4A08BF4A4658
:10B5C80000E0364AACF1040CBCF1070F05D8DFF8EF
:10B5D8001CC11EF0010F18BF6246DBB2032B0ED848
:10B5E8001EF0020F3C4B06E0DBB2032B06D82F4BB4
:10B5F8002A4A1EF0020F18BF1A4600E0274A4FF0E9
:10B60800000C5FFA8CF383420DD20B6803EB8C03BA
:10B618005B881B0642BFD2F80090214B43F82C9060
:10B628000CF1010CEDE785B1BEF1000F08D0637B8A
:10B63800184A0133DBB2142B06D1002304E025B1EC
:10B64800637B002BF3D100E05373002E52D0234AC2
:10B658003223B2F90250B2F90020002DB8BF6D4272
:10B66800002AB8BF524295FBF3F592FBF3F2EDB214
:10B67800D3B2AB4238BF2B46194A13B192FBF3F34E
:10B6880000E0134643442360E37B024A83BB012363
:10B698002FE000BFE02100208829002010BA01080F
:10B6A800AA0D002082310020F8A90108E8A90108A4
:10B6B800481F002018A20108C01900201EA2010876
:10B6C80024A201082AA2010830A2010836A2010812
:10B6D800542D0020C42F002000AA010800110020CA
:10B6E800400D0300902D00204819002008AA0108E9
:10B6F8000023D3738F4D904B2D78E27BADB9002F8B
:10B7080000F00F818D4B267B1A788D4B02F00402D6
:10B7180093F800C08B4BD2B2D3F800E00B6800213D
:10B72800894D03EB86060F46B5E01AB9874A1A61B8
:10B73800002508E0864AFAE70A68AB00D61876883A
:10B74800760604D40135EBB28342F5D3D7E7814EB0
:10B75800B6F90060192E25DD12F803E094F814C03C
:10B768000EF00F09E14526690CDCDFF8CCC19CF826
:10B7780015C0BCEB1E1FDEBFD6F800C0DFF8D8E14D
:10B7880043F80EC012F803E094F816C00EF00F0943
:10B79800E14533DBDFF8A0C19CF815C0BCEB1E1FE8
:10B7A8002CDC26E0193629DA12F803E094F814C0E4
:10B7B8000EF00F09E14526690CDCDFF87CC19CF826
:10B7C80017C0BCEB1E1FA2BFD6F800C0DFF888E187
:10B7D80043F80EC012F803E094F816C00EF00F09F3
:10B7E800E1450BDBDFF850C19CF817C0BCEB1E1F0E
:10B7F80004DBD6F800E0584E43F806E0554EB6F99B
:10B808000260192E1BDD12F803C094F814E00CF046
:10B818000F09F14526690CDCDFF81C9199F81590A1
:10B82800B9EB1C1FDEBFD6F80090DFF82CC143F837
:10B838000C90D25C02F00F0CF4451EDD82E719363D
:10B8480080DA12F803C094F816E00CF00F09F145FD
:10B8580026690CDBDFF8E09099F81590B9EB1C1F0E
:10B86800DEBFD6F80090DFF8F0C043F80C90D25C49
:10B8780002F00F0CF445FFF665AF94F817E0BEEB45
:10B88800121FA2BF3668344A9E505BE758880005ED
:10B8980004D404330435B342F8D122E04AB101EBB1
:10B8A8000C0A06209AFBF0F900FB19A001280DDC10
:10B8B80001E057B9012793F801900EEB89003EF893
:10B8C80029A090F80290C07803E01746002081462E
:10B8D8008246013125F802AC85F800906870C9B23B
:10B8E800D7E7174A1378013B13F0FF0308BF062375
:10B8F8001370124B1B785B0741BFBBF906304FF43E
:10B908007A72A3F57A7303EBC30348BF93FBF2F390
:10B91800124A46BF0133DBB2012392FBF3F34344DF
:10B92800A36003B0BDE8F04F04F0E0BA03B0BDE88F
:10B93800F08F00BF5B0E0020E02100208231002044
:10B948003000002088290020AC0D002004AA01083E
:10B9580010BA010800110020AA0D0020400D0300B4
:10B968002DE9F04F89B00593A04B80461B880492BF
:10B97800980737D540F2E632129B9D48DC89B0F92A
:10B9880000301B1B03F2F315954203D8002BB8BFF8
:10B998005B4201E04FF4FA73B0F9022040F2E6305E
:10B9A800121B02F2F314844203D8002AB8BF524291
:10B9B80001E04FF4FA729342B8BF13460522C3F56B
:10B9C800FA7393FBF2F30A22643B534398F81C2062
:10B9D800D2105343642293FBF2F3134423EAE37334
:10B9E800DBB200E06423C1460193CB1C039300241F
:10B9F800039B022C13F8016F7E4F03934FEA440A0E
:10BA080005D1B7F904301B365E4376114AE07A4B0C
:10BA180037F9142033F9143003EB4202049B5B42DC
:10BA28009A4203DB049B9342A8BF1346734A32F938
:10BA38000A50059A5B1B32F9145003EB050B07F00B
:10BA480019F988B16E4A5846155D07F085FF6D49AA
:10BA580008F08AF80146284606F0FAFC694907F01A
:10BA6800CFFF08F093F98346604A1288D10714D4AF
:10BA780037F90A501B366E4393074FEA261611D53D
:10BA880098F812509DF9042005FB0BF353436422E8
:10BA980093FBF2F306EB231604E098F8085005FB35
:10BAA8000BF52E11584B042533F90A30574F93FBE9
:10BAB800F5F5751B99F80160E35D6E435E430293EB
:10BAC800642396FBF3F698F851B0F611BBF1000F1A
:10BAD8001BD0022C30460CD107F03EFF5FEA5B0317
:10BAE80004D05B45A8BF5B461A4600E001224849DE
:10BAF80005E007F031FF5A46391D01EBC401FB6927
:10BB0800FCF7C4FF08F042F90646424B99F80B705F
:10BB180019883E4B01FB05F203F1200E5EF8240064
:10BB2800D21207FB02073C4AB7F5001FA8BF4FF423
:10BB38000017974203F12C00B8BF174650F824208D
:10BB480040F824504FF6FF700909B0FBF1F1AA1A2A
:10BB58004A4303F1380103F144054EF8247051F8C3
:10BB680024E055F8240045F824E098F85050921144
:10BB780070444FEA840C7F13104441F824208DB19F
:10BB8800CDF818C0079307F0E7FE079B2A4603F194
:10BB9800500101EBC401DB69FCF778FF08F0F6F807
:10BBA800DDF818C099F81530F2195843029B013492
:10BBB80043431846642390FBF3F0184B00120244E9
:10BBC80023F80A2003F108024CF80260032C03F161
:10BBD800140203F120034CF802704CF8030009F139
:10BBE80001097FF405AF09B0BDE8F08FC019002046
:10BBF800902D0020001100207C3100204C2D0020C9
:10BC08003CA20108000020411C100020F82100205F
:10BC18000C220020F80F00200000E0FF6022002026
:10BC28002DE9F04F8BB00793CA4B0592B3F9022068
:10BC3800002682EAE279A9EBE279B3F9002080468E
:10BC480082EAE273A3EBE2739945B8BF9946B4461A
:10BC58003446B9F5FA7F0691A8BF4FF4FA790290F5
:10BC680001960396BC4D2B88990755D0B94B6100B6
:10BC780033F91420B94B33F9143003EB4202059B16
:10BC88005B429A4203DB059B9342A8BF1346B44A22
:10BC98008F5E079ADB1B32F914001F1806F0EAFFC3
:10BCA80090B1B04B384613F804A007F055FEAE49E2
:10BCB80007F05AFF0146504606F0CAFBAA4907F0AA
:10BCC8009FFE08F063F8074698F8083064227B4323
:10BCD80093FBF2F398F81C206FF0040101FB02FCBF
:10BCE800634505DB02EB82029342A8BF13469C46DC
:10BCF80042F210729D4B53F8240038449042A8BF7A
:10BD080010469B4A9042B8BF104643F8240098F862
:10BD180012305843031303932D8805F00303012BB6
:10BD280038D08C4B934933F91430A6000193029B09
:10BD380051F8247093F801E08F4B33F9140080EA2E
:10BD4800E073A3EBE073B3F5206F16DC019A502380
:10BD58005A4392FBFEF3042290FBF2F0181A0744B0
:10BD6800B7F57A5F854BA8BF4FF47A579F42ACBFAF
:10BD780041F8247041F8243002E0002341F82430CF
:10BD88008B597D2693FBF6F6029BDB7A734340269C
:10BD980093FBF6F6AA0712D5019B09FB06F509FBEA
:10BDA80003F70398C9F5FA7202FB0C7702FB0052FD
:10BDB8004FF4FA7197FBF1F392FBF1F505E0EB070D
:10BDC80055BF35466346019B039D6B4A042732F9EC
:10BDD8001420DFF8ACB192FBF7F70BF19C02A25CE0
:10BDE8004FEA440A57436FF04F0297FBF2F798F86F
:10BDF80051201F449AB13846CDF810C0089207F078
:10BE0800ABFD0BF1040101EBC401089ADBF81C300F
:10BE1800FCF73CFE07F0BAFF0746DDF810C0564BAA
:10BE28004FEA840B3AF80300554B02B203F1A00124
:10BE38003AF901E02AF80100CEEB02024FF0040EB5
:10BE480092FBFEF203F1A40103F1AC0E04925EF83A
:10BE5800240051F824201044049A104451F8242056
:10BE68004EF82420049A41F8242098F8502092B1E2
:10BE7800CDF810C00993089207F06EFD099B089A47
:10BE880003F1500101EBC401DB69FCF7FFFD07F08A
:10BE98007DFFDDF810C03A4B03F1B402125D03F1E7
:10BEA80068015043202290FBF2F07A19121A2AF8FE
:10BEB800012003F170024BF8027003F17C024BF889
:10BEC8000250404203F188024BF80200029A013204
:10BED80002920CB90124C5E61E4A0420B2F90410E6
:10BEE800069A9C6A92790F3252004A4322495511A8
:10BEF800B1F9041085EAE57291FBF0F0A2EBE57266
:10BF0800322AA5EB000098F80D100BDC01FB00416C
:10BF18001C4A8A42A8BF0A461B498A42ACBF9A6299
:10BF2800996201E000229A6298F8031001FB00F27E
:10BF380016499211097803292BD9B8F84E10B1F592
:10BF4800FA7F26D24842824222DB8A42A8BF0A46AA
:10BF58001FE000BF00110020C01900207C31002024
:10BF68004C2D00203CA20108000020418C2200201A
:10BF7800F0D8FFFF182200201C10002080C1FFFF0E
:10BF8800F8210020FEFFFF0F020000F0C81F00206C
:10BF98000246996A6FF0FF0041F34F31B1F5807F97
:10BFA800A8BF4FF480718142B8BF01469A67501804
:10BFB8000022A3F86C00C3F88410C3F890200BB0DB
:10BFC800BDE8F08F2DE9F04F87B00393B94B814658
:10BFD8001D88029105F00205ADB2019295B1B64BEC
:10BFE800B3F90250B3F90030002DB8BF6D42002BF1
:10BFF800B8BF5B429D42B8BF1D46B5F5007FA8BFDC
:10C008004FF40075CB460026AB4BAC4933F91620EC
:10C01800AB4B4FEA460A33F91630520083EAE37411
:10C02800A4EBE374B4F5206F4FEA860851F82600B4
:10C0380011DC042493FBF4F3D31A0344B3F57A5FB9
:10C04800A048A8BF4FF47A538342ACBF41F82630CA
:10C0580041F8260002E0002341F8263051F8087024
:10C068009BF80B30FF119BF801405F43914B544301
:10C078001B88BF119B074FEAA41456D0924B3AF97C
:10C0880003301A44019B5B429A4203DB019B9342B3
:10C09800A8BF13468D4A3AF902209B1A039A32F92F
:10C0A80016201A44049206F0E5FD049A98B1884BCC
:10C0B80010469B5D049307F04FFC864907F054FD3A
:10C0C800049B0146184606F0C3F9824907F098FC1C
:10C0D80007F05CFE024642F210707F4958F80130C2
:10C0E80013448342A8BF03467C488342B8BF034633
:10C0F80048F8013099F8081099F81C004A4300EBF9
:10C108008000D21141428A4203DB8242A8BF024624
:10C11800114699F81220641A53431B13FF1A6F43F0
:10C128006C4303EB672701EB6424654B04223AF95F
:10C13800033093FBF2F16A4B03F19C02925D4A4390
:10C14800A4EBA21499F851207AB1204605930492E1
:10C1580007F002FC059B049A191D01EBC601DB6977
:10C16800FCF794FC07F012FE0446554B3AF803001E
:10C178005B4B02B203F1B8013AF901E02AF8010079
:10C18800CEEB02024FF0040E92FBFEF203F1BC016B
:10C1980003F1C40E58F801C058F80E0048F8012001
:10C1A8006044104499F8502048F80EC072B10593C5
:10C1B800049207F0D1FB059B049A03F1500101EBAF
:10C1C800C601DB69FCF762FC07F0E0FD444B0BF1AC
:10C1D800010B03F1B402925D03F168015043E219C7
:10C1E8004011121A2AF8012003F1700248F802409F
:10C1F80003F17C0248F80270404203F1880248F8D3
:10C2080002000EB90126FFE62B4A0420B2F90410F9
:10C21800029A9C6A92790F3252004A432849521175
:10C22800B1F90410002A91FBF0F0A2EB0000B8BFAE
:10C238005242322A99F80D100BDC01FB0041294AC1
:10C248008A42A8BF0A4628498A42ACBF9A629962C4
:10C2580001E000229A6299F8031001FB00F22349D9
:10C268009211097803290CD9B9F84E10B1F5FA7F63
:10C2780007D24842824203DB8A42A8BF0A4600E04E
:10C288000246996A6FF0FF0041F34F31B1F5807FA4
:10C29800A8BF4FF480718142B8BF01469A67501811
:10C2A8000022A3F86C00C3F88410C3F8902007B0EC
:10C2B800BDE8F08FC01900200011002018220020CE
:10C2C8001C10002080C1FFFF7C3100204C2D002075
:10C2D8003CA20108000020418C220020F0D8FFFF7A
:10C2E800F8210020FEFFFF0F020000F0C81F002009
:10C2F8002DE9F04F054690F850008DB00891059251
:10C30800099318B13228A8BF322000E0012007F0B5
:10C3180023FB0146AA4807F027FCAA4B04461888C5
:10C32800002808BF012007F017FBA749069007F06F
:10C3380067FB01900199204607F05AFA01460198D7
:10C3480007F012FCA14B07901B889A0724D5A04937
:10C35800B1F90030B1F9020083EAE37280EAE071D2
:10C36800A2EBE372A1EBE07191420C46B8BF144610
:10C37800B4F5E17F12DA914203DD0028D8BF4042CC
:10C3880003E0002BCCBF1846584207F0E5FA914964
:10C3980007F0EAFB064603E0002601E04FF07E5670
:10C3A8004FF00009CA4603950024630004938A4BA2
:10C3B80033F9140007F0D0FA884907F021FB07F099
:10C3C800E5FC07F0C9FA864907F01AFB804B029092
:10C3D80033F9140007F0C0FA7C4B07461B889B070B
:10C3E8007ED0014607F004FA7E4B804633F91400EC
:10C3F80007F0B2FA0146404607F0FAF907F0C6FC22
:10C40800059B5B42984203DB059B8342A8BF03461A
:10C41800754A0499885E099A1B1A32F9140018445F
:10C4280007F09AFA804606F025FC70B16F4B40463B
:10C438006F4914F8039007F097FB0146484606F049
:10C4480007F86B4907F0DCFA8046287F07F080FA86
:10C45800684907F0D5FA8246287A07F079FA014642
:10C46800404607F0CDFA644907F0CAFA07F08EFC97
:10C4780081460AF1004007F089FC814505DB5046FA
:10C4880007F084FC4845A8BF484607F065FADFF87E
:10C498008C9101998246404607F0B2FA59F8241067
:10C4A80007F0A6F955494FEA840B804607F046FC89
:10C4B80038B94046524907F05FFC20B1DFF84081A7
:10C4C80001E0DFF8388149F80B80A87C07F040FAD2
:10C4D8000146404607F094FA4A4907F091FA814626
:10C4E8003A4BB3F800B01BF0010F40F099803A4B7B
:10C4F800049ADFF82081D35E002BB8BF5B42B3F506
:10C50800206F4FEA84030A9303DD002348F82430A0
:10C518002AE03D49384607F073FA039B0B90587898
:10C5280007F016FA0B9A0146104607F01DFB029910
:10C5380007F05CF9019907F063FA58F8241007F03E
:10C5480057F93249804607F0F9FB38B94046304977
:10C5580007F012FC20B1DFF8B88001E0DFF8AC800A
:10C568002C4A0A9B42F80380039BD87A07F0F0F91B
:10C57800284B53F8241007F043FA274907F040FAEC
:10C588001BF0020F80464DD03846514607F02EF971
:10C598000146304607F034FA0146504607F028F9BC
:10C5A80049460746404607F021F90146304607F05C
:10C5B80027FA0146484607F01BF9804632E000BFDB
:10C5C80083F9223EF80F0020BD378635C0190020B8
:10C5D800001100200000E1431C1000200000A03ED4
:10C5E800CDCC4C407C3100204C2D00203CA20108D1
:10C5F800000020410000A0406F12033C0000F0C181
:10C608000000F0410AD7A33D0000A043000040C34A
:10C6180000004043CC2200200AD7233CC42200203B
:10C62800C8465746DFF83CB20BF19C03185D07F08B
:10C6380093F90146029807F0E3F9894907F0E0F910
:10C648000146384607F0D2F895F85120034642B122
:10C658000BF10401DBF81C3001EBC401FCF716FAFE
:10C668000346804F029807F1E00B5BF824100A9309
:10C6780007F0BCF8019907F077FA029B07F1E80286
:10C688004BF8243052F824B00292594607F0AEF81D
:10C698000146079807F0B4F90146584607F0A8F88C
:10C6A800029A834642F8240007F1B402105D07F0AD
:10C6B80053F90146584607F0A3F96B4907F0A0F96A
:10C6C80083460A9B4146184607F092F8594607F0F8
:10C6D8008DF80AF0E7FE049B07F16802D0520A9B26
:10C6E80007F170021846029207F050FB029A07F110
:10C6F8007C0342F824004046029307F047FB029B64
:10C7080007F1880843F824000BF1004007F03EFBCE
:10C71800039B48F82400013303930CB9012444E631
:10C72800089A524B9479B3F90430640028345C4376
:10C738004F4B6411B3F9040007F00EF94FF07A512A
:10C7480007F05EF90AF0AEFE201A07F005F9002C92
:10C75800B8BF6442322C064602DD0023BB6224E0E7
:10C76800069807F013FB20F0030007F0F5F8804661
:10C77800687B07F0EDF80146304607F041F93D497E
:10C788000446404607F0F0F90146204607F038F91C
:10C7980007F0FCFABB6A1844374B9842A8BF184602
:10C7A800364B9842ACBFB862BB62BB6A6FF0FF0001
:10C7B8005B13B3F5807FA8BF4FF480739842B8BF6E
:10C7C800184607F0C9F88046304607F0DFFAEB78DC
:10C7D8005843801107F0C0F8294B04461B78032BF7
:10C7E80011D9B5F84E60B6F5FA7F0CD207F0CEFA3B
:10C7F8007342984203DBB0420346A8BF334618464B
:10C8080007F0AAF8044695F8512062B1530803D0FE
:10C818009A42A8BF1A4600E0012220461949FB693E
:10C82800FCF734F904464146204606F0E1FF07F0DC
:10C83800ADFA00B207F090F80AF034FEA7F86C00E1
:10C84800204607F0A3FAB867404607F09FFA00238E
:10C85800C7F88400C7F890300DB0BDE8F08F00BF6E
:10C86800A69B443BF8210020F7CC92380011002009
:10C878001C10002000803B45FEFFFF0F020000F067
:10C88800C81F00200C22002010B507F065F8002111
:10C89800044607F071FA08B1204601E004F10040AF
:10C8A800054907F061F9054907F0AAF8FCF7D0FB3C
:10C8B800034B186010BD00BF8096184B35FA8E3CAC
:10C8C8004C000020F8B59C4B04461B68187818B13A
:10C8D800012800F06A819AE2242C984D0CD006D8E1
:10C8E8000A2C00F0D9800D2C00F0D68048E12A2CC3
:10C8F80006D02C2C04D043E128706870A87050E151
:10C908008F4B69782F7800208C4A58542FBB1978A0
:10C91800D770472921D1597850291ED199784729AC
:10C9280007D1D978472904D11979412901D10121A1
:10C93800D1709978824A522903D1D1784D2900F0D3
:10C94800688299787E4A472907D1D178532904D13A
:10C958001279562A04BF0322EA70EA78774E022A2F
:10C9680039D0032A4CD0012A40F08580BA1E072A04
:10C9780000F28180DFE802F004080F131A257F2AED
:10C9880005F0D8FE686076E01B78532B73D16B688E
:10C998005B426B606FE005F0CDFEA8606BE01B7832
:10C9A800572B68D1AB685B42AB6064E01B78302BD7
:10C9B800644B1A788CBF42F0020222F002021A700D
:10C9C80059E0002005F016FF287354E0002005F018
:10C9D80011FFE8814FE0072F06D0082F4BD1012027
:10C9E80005F008FF708246E0012005F003FF41F2E0
:10C9F800184358434FF47A73B0FBF3F030823AE0AF
:10CA0800022F07D0032F0AD1002005F0F3FE4E4B6A
:10CA1800187030E0002005F0EDFE30752BE02AD9C3
:10CA28003A1F9210337D0132D2B2013B02EB8303ED
:10CA3800DBB2102B1FD8F91EC2F1010201EB8202F2
:10CA4800D2B2012A0BD0042A11D100205E1E05F0B3
:10CA5800D1FE3E4B002298553D4B9A5507E03D4A82
:10CA68005E1E0020935505F0C5FE3B4B98553B4A8A
:10CA7800136801331360314B2A2C18BF9A7807F1D9
:10CA880001074FF000000CBF012254402F7068705E
:10CA98000CBF5A759C7084E0687D002848D0304BE4
:10CAA80013F8012D2F495A708B42F9D1244A234C8F
:10CAB80013785278402B85BF373B1B011B01DBB233
:10CAC80098BF03F0F003402A8CBF373A303AD2B20D
:10CAD8001344AA78DBB29A4227D121230B7022494A
:10CAE800E0780B68012803F101031E4A0B600AD0A5
:10CAF80002281CD172231370228A1C4B1A80628A66
:10CB08001B4B1A8013E0672313700E4B1B789F078B
:10CB18000ED5184B62681A60A2685A60227B164BC1
:10CB28001A70E289154B1A8002E03F230B7000202F
:10CB380000236B7535E000BFC4070020E822002001
:10CB4800802D0020FC1800207C100020AD10002053
:10CB58009D1000207D1000208D10002084240020CE
:10CB6800D4020020C002002090240020FE180020DB
:10CB78006410002004190020021900200019002068
:10CB88006B78687D0E2B9FBFA54A591C5170A54A2A
:10CB980098BFD454A24A18B993785C40947000E0C6
:10CBA8000020003018BF0120F8BD9D4B0022997D60
:10CBB800082900F22C81DFE801F0050B0F15202B66
:10CBC800475D6700B52C40F02281DA75012239E013
:10CBD800622C08BF022235E003229A751C765C7627
:10CBE8009C7614E104229A755A7E997E2244D2B228
:10CBF8005A760A449A76DC7609E105229A755A7EB5
:10CC0800997E2244D2B25A760A449A769C83FEE0F0
:10CC180006229A755A7E997E2244D2B25A760A44DE
:10CC28009A769A8B02EB0424A4B2B4F5AC7F82BF47
:10CC38007B4A0121D17500229C83DA83002C40F0C5
:10CC4800E68007229A75E2E05A7E997E2244D2B2A3
:10CC58005A760A449A76DA8BB2F5AC7F3EBF7049B1
:10CC6800891881F820400132998B92B29142DA8377
:10CC7800E7D9CCE008229A755B7EA34200F0C78012
:10CC8800674B0122DA750DE0674D9A7515F8012D8D
:10CC98006A70664A9542F9D1997E614AA14206D0E6
:10CCA8003F232B70624A536801335360AFE06148F9
:10CCB800016801310160D07D10B13E232B70A6E0E0
:10CCC80021212970D17E062941D004D8022907D014
:10CCD800032923D0F8BD122959D0302967D0F8BDCF
:10CCE8005021546A297054494C60946A0C60116B45
:10CCF8004FF47A7491FBF4F1504C218092F878113A
:10CD08004F4A19B1117841F0020102E0117821F07F
:10CD180002011170012283F8792169E053212970F9
:10CD280092F82510CE0705D592F82420D51E6A4220
:10CD38006A4100E0024602F0010183F87811002AF6
:10CD480056D13F490A7822F002020A7050E04F217A
:10CD5800297092F82B10CC0705D592F82A20D11EFD
:10CD68004A424A4100E0024602F0010183F8781184
:10CD780022B933490A7822F002020A7093F84F1058
:10CD8800304A1170B3F84C102F4A118030E0562108
:10CD9800546B29702D490C8042F21074916B91FBF1
:10CDA800F4F12B4C2180012182F87A1120E04921ED
:10CDB800297092F82410274A102988BF1021117071
:10CDC800254914780022A2420ED20E7A234D5655D8
:10CDD8004E7A234D5655CE7A224D565511F80C6F82
:10CDE800214D56550132EEE720490A6801320A60A2
:10CDF80093F879310A4A002B3AD092F87A31BBB3CA
:10CE0800002182F8791182F87A111846F8BD0020BD
:10CE1800F8BD1279432A7FF494AD0222EA7090E5B6
:10CE2800E8220020802D0020D4020020C00200202B
:10CE3800A4070020902400200419002000190020D5
:10CE4800FC1800200219002056000020FE180020BF
:10CE5800641000207C100020082300207D10002092
:10CE68008D1000209D100020AD100020842400208B
:10CE7800F8BD0449044B0968002218705A61996189
:10CE88001A777047782D0020A4070020F8B5101AEB
:10CE98000D461F4606F060FD0446781B06F05CFD53
:10CEA800174B079E196806F0ABFD2146054620463C
:10CEB80006F0A6FD29460746284606F0A1FD0146CC
:10CEC800384606F095FC0AF051FD0E4906F098FD2B
:10CED80006F082FF069B2946186004F100400AF01C
:10CEE800B9FB094906F08CFD084906F081FC06F0FB
:10CEF8004DFF0028BCBF00F50C40A0303060F8BDE5
:10CF08004C0000202C7D8E3FA00CB34500A00C46A1
:10CF180044F25063984203DDA0F50C40A0387047F6
:10CF2800034B9842BCBF00F50C40A030704700BFCF
:10CF3800B0B9FFFFF7B50368174C184D23600B68AD
:10CF4800174E63600068FFF79FFC95E80300154BD8
:10CF58000196009394E80C00FFF798FF3668124B8F
:10CF680060681E606B68114FC01A06F0F5FC104B24
:10CF7800196806F045FD06F009FF2A6823687860FD
:10CF88009B1A3B600B4B1E600B4B1B68DA880B4BE4
:10CF98001A8003B0F0BD00BF042C00200419002043
:10CFA800102C00200C2C00204C2C0020142C0020CD
:10CFB8004C000020442C0020300F0020402C002082
:10CFC80070B50446407906F0C3FC1E4906F0CCFD56
:10CFD8001D4D1E4E2860E07B06F0BAFC194906F08C
:10CFE800C3FDEE606860A07906F0B2FC184906F04F
:10CFF800BBFD184D2860207C06F0AAFC114906F0FC
:10D00800B3FD6860A07E06F0A3FC134906F0ACFDF2
:10D01800EE60A860E07906F09BFC0D4906F0A4FDDF
:10D028000E4D2860607C06F093FC064906F09CFDD6
:10D038006860E07E06F08CFC074906F095FDEE601E
:10D04800A86070BD0000C8421C2C00200000FA44F3
:10D05800000020412C2C002000007A44502C002095
:10D0680010B50C4C23789B0713D50B4B1B78042B5E
:10D078000FD90A4A0A4B1068526818605A60FFF7BD
:10D0880003FC084B1A88084B1A80237843F00103E5
:10D09800237010BDFC18002002190020041900207C
:10D0A80068100020F8100020602C0020164B13B5E3
:10D0B8001B681B0325D5154B154C1B7815498DF896
:10D0C8000030154B20681B788DF8013006F098FC6D
:10D0D80006F082FE11498DF80200606806F090FCA7
:10D0E80006F07AFE8DF80300A06806F075FE0C4B7A
:10D0F8008DF804001B780A2069468DF80530FAF788
:10D1080065FB02B010BD00BF542D0020462D002045
:10D11800682D002000002041642D002000007A4482
:10D128004A2D0020054A137883F001031370044A3E
:10D1380000231360034A1360B8E700BF4A2D00209C
:10D14800602D00205C2D0020094A137818441346EE
:10D15800C0B210F0800F18BF80381070054A1978D7
:10D168001378994201BF00231370014A1370704766
:10D17800652C0020642C002010B50A4B0A4A1B7845
:10D1880042609C18094A046012789A4225BFD31A53
:10D198000B60C3F1800300232EBF4B600B604A6015
:10D1A80010BD00BF652C0020662C0020642C0020D8
:10D1B8001FB5684602A9FFF7DFFF044B02981B68FA
:10D1C80003440398184405B05DF804FB24060020C6
:10D1D8002DE9F04F89B001930023824699460291C8
:10D1E8000392039A934205DA029A52F823200133F4
:10D1F8009144F6E7019B4D46002B56D103F056F8B3
:10D20800002852D101987DE00222404E8DF81C2062
:10D218001A0C4FF480578DF81D2006201A0A8DF835
:10D228001E208DF81F3003F065F87761062005F0A1
:10D23800B3F8374B01223761D0461A70776126461A
:10D24800002007A9042205F0CDF8029F4FF0000B3B
:10D25800039B9B451EDABC4657F8042B4FEA8B0309
:10D26800002A48D0B24236D332465AF8031000207A
:10D27800CDF814C0049305F0B5F8049BDDF814C08C
:10D288005AF8032032444AF80320DCF800309E1B89
:10D29800CCF800601D4B4FF480521A611D4A2D1BBB
:10D2A80013681C44019B146053B34DB3194B1B689E
:10D2B800DCB22A19B2F5807F174A88BFC4F580749A
:10D2C800D26898BF2C4693429ED3144A0023137009
:10D2D800134A137014E00020D8F8001005F082F803
:10D2E80057F8043CD8F80020F61A1344C8F8003060
:10D2F800002347F8043C0BF1010B08F10408A7E7E9
:10D30800C5EB090009B0BDE8F08F00BF000C014073
:10D31800210600202406002010000020642C002094
:10D32800652C002030B50B4C0B4D22782B7885B03E
:10D338009A420CD0684602A9FFF71EFF01236846EF
:10D3480002A90222FFF744FF00232B70237005B0C7
:10D3580030BD00BF652C0020642C002030B50E4D78
:10D368000E4C2A78237885B09A4211D0684602A9D3
:10D37800FFF702FF002302A902226846FFF728FFF1
:10D38800FFF7E2FE20782B781B1A5842584100E03C
:10D39800012005B030BD00BF652C0020642C0020A2
:10D3A80038B50E4C4FF4805545F2082002F0A2FF24
:10D3B8006561062004F0F0FF094B01222561C720B2
:10D3C8001A70656104F0E8FF064A002325611370AE
:10D3D800054A1370054A136038BD00BF000C0140B0
:10D3E80021060020642C0020652C00202406002043
:10D3F8000148024900F09ABE00080040442000207D
:10D408000148024900F092BE000400401C200020A0
:10D418004FF08040014900F089BE00BFF41F002092
:10D428000148024900F082BE002C0140CC1F0020B8
:10D438000148024900F07ABE002C0140CC1F0020B0
:10D448000028114AB8BF404290FBF2F330B50F4CA8
:10D458003C2504FB030068430D4D90FBF2F22D6858
:10D468002D7B25B903EB830303EB830301E0C3EBB7
:10D47800031302EB830304FB02020B804FF47A735D
:10D4880092FBF3F24A8030BD80969800806967FF6E
:10D49800EC180020022803D0431E58425841704718
:10D4A800064B1B681B7823B1054B1868C0F3C040B6
:10D4B8007047044B1878C0F38000704700060020BE
:10D4C800FC0F00208231002010B50A4C5E2801466E
:10D4D800206805D15D21FDF74EF920683E2105E061
:10D4E8005D2903D1FDF747F920683D21BDE81040CB
:10D4F800FDF741B964240020A0F17D03012B70B52C
:10D5080004460D460A4E05D830687D21FDF733F9EB
:10D5180084F0200430682146FDF72DF935B12B88B9
:10D528001C4404EB142404F0FF042C8070BD00BFDD
:10D53800B019002010B5054C2068FDF719F918B18D
:10D548002068FDF712F9F6E710BD00BF801900202A
:10D5580010B50446C0B2FFF7B7FFC4F30720BDE813
:10D568001040B1E7024B5E211868FDF704B900BF0F
:10D578006424002038B50546054C5E212068FDF777
:10D58800FAF820682946BDE83840FDF7F4B800BF2E
:10D598006424002013B5044601A90068FFF750FF72
:10D5A8001320FFF7E7FFBDF90400FFF7D1FF1B20A9
:10D5B800FFF7E0FFBDF90600FFF7CAFF2320FFF7DA
:10D5C800D9FF2368002BB4BF53204E20FFF7C0FFBC
:10D5D80001A96068FFF734FF1220FFF7CBFFBDF900
:10D5E8000400FFF7B5FF1A20FFF7C4FFBDF90600D6
:10D5F800FFF7AEFF2220FFF7BDFF6368002BB4BF23
:10D6080057204520FFF7A4FF02B010BD674B73B544
:10D618001878FFF73FFF664D04462B78834220D0E9
:10D62800C8B1644B1B68E3B193F90000022300936F
:10D63800614B04211B6800225B78003318BF01236B
:10D6480001934FF41653FCF73DFD5C4B186040B155
:10D6580001232B7005E0594E3068FCF720FD34603B
:10D668002C70574B574D1878FFF714FF2B7804464A
:10D67800834218D088B1544B1B68A3B100220124FF
:10D6880093F9000008214FF4964300940192FCF7A7
:10D6980019FD4E4B186028B905E04C4E3068FCF770
:10D6A800FEFC34602C704A4B4A4D1878FFF7F2FEA6
:10D6B8002B78044683422E4643D0002838D0464B68
:10D6C8001A68002A3DD0D37992F90000002B4FF058
:10D6D8000202424C08BF02230092002254F8233071
:10D6E80001921021FCF7EEFC3D4B0546186040B353
:10D6F8003C4C94F84A30022B0BD094F89620022A1E
:10D7080001D14C3405E023B1002A04F14C0418BFC0
:10D718000024354B1C6044B1204600214C2209F0FE
:10D72800B4FC0223256084F84A300123337008E0F2
:10D738002B4E306804F018FB3068FCF7B0FC3460FE
:10D748002C702A4B2A4D1878FFF7A4FE2B78044634
:10D75800834229D000B3274B1B682BB3264A93F981
:10D7680000001268032352782021002A0CBF0822E7
:10D778000922009301924FF461430022FCF7A2FCB6
:10D788001E4B186080B11E4A012313702B701D4B6D
:10D798001A681D4B1A6007E0184E3068FCF77FFCCA
:10D7A800174B34601C702C7002B070BD0806002046
:10D7B800E010002004060020EC180020642400205B
:10D7C800090600200C19002090190020801900205B
:10D7D80014060020961900201006002034A601081F
:10D7E80098190020D82900209C1900202006002024
:10D7F800AC1900201C06002018060020B0190020D3
:10D80800B4190020782D0020B8190020642928BFF9
:10D818006421F8B501FB00F5642495FBF4F4064691
:10D82800E4B20027FBB2A34204D29F2002F09DFD80
:10D838000137F7E7B4420BD2142195FBF1F5C4EB9D
:10D848008410663DC4EB80002844C0B202F08DFD10
:10D858000134E4B2B44201D29A20F7E7F8BD2DE9C9
:10D86800F743FCF7AFFE924C6368C31A002BC0F273
:10D87800688300F5433303F5A07363608D4B1D780F
:10D88800237AC5F38005EB1A18BF012325724DB121
:10D89800002B00F05683884B5A789A7001225A70F0
:10D8A8001A702BE0844A2BB1D37843F00203D3706B
:10D8B80093785370D67806F0020101F0FF0339B966
:10D8C8007D498968411A002903DB06F0010300E05D
:10D8D800012303F00107784917707BB1F2070DD5D2
:10D8E8000A7905230132D2B2B2FBF3F303EB8303C7
:10D8F800D31A724ADBB20B71D35C4B706E4EDFF8F1
:10D90800088233787BB3F37823F00203F3706C4B0F
:10D918000344AE20B36002F04CFD08B102F04EFDA6
:10D9280088F80000002800F00C83B02002F041FDC8
:10D93800402002F03EFD002002F03BFD102002F0E6
:10D9480038FD4FF48067013F0020BFB202F008FDA8
:10D95800002FF8D1384602F0A0FD7278594B53F8E1
:10D96800220002F01DFD98F80030002B00F0E9823B
:10D978007378062B00F2B282DFE813F00700B002DA
:10D98800180078006A018701EC014F494F4A504B53
:10D998005048FBF7A6FA012002F07FFD4D4802F03F
:10D9A800FFFC022002F079FD4B48ACE14B4F3B688D
:10D9B8009B0735D5DFF854810A23B8F80010DFF843
:10D9C8005091B1FBF3F203FB121399F8001092B2D5
:10D9D8009BB200913F484249FBF783FAFDF7F6FCFA
:10D9E800012002F05AFD3B4802F0DAFC3D4B99F861
:10D9F80000201868B8F80030067902FB1631642355
:10DA08004B43C17802208E1B5643B3FBF6F6F6B2A1
:10DA180002F043FD31461520FFF7F8FE032600E02B
:10DA280001263B681F0540F159822F4B2F491F687B
:10DA3800642397FBF3F2096803FB127300912548EE
:10DA48002B49FBF74EFAFDF7C1FC304602F025FDE5
:10DA5800204802F0A5FC02F03BF90746701C02F0D2
:10DA68001CFD15203946FFF7D1FE37E20120214F72
:10DA780002F013FD204802F093FC3B68980749D553
:10DA88001E4A1448B2F90210B2F900300091B2F9F6
:10DA980004201B4901921B4AFBF723FAFDF796FC69
:10DAA800022002F0FAFC0B4802F07AFC032632E06E
:10DAB80064240020823100204829002001C1010887
:10DAC800404B4C0040A2010806C101080FC10108E3
:10DAD80049BA01086D24002016C10108542D002000
:10DAE8001FC10108E4180020F0180020F4180020D5
:10DAF80037C10108F81800204CC10108EA100020BD
:10DB080062C1010871C101084D020020E818002017
:10DB18005400002002263B68D9071AD57B4A7C4866
:10DB2800B2F90210B2F900300091B2F90420794933
:10DB38000192794AFBF7D5F906F10108FDF746FC91
:10DB4800304602F0AAFC5FFA88F8714802F028FC17
:10DB580046463B681A0718D5704A6D48B2F9021054
:10DB6800B2F900300091B2F904206A4901926C4A76
:10DB7800FBF7B7F9771CFDF729FC304602F08DFC5E
:10DB8800FFB2634802F00CFC3E46664A6149B2F9AE
:10DB98000030B2F902205E480092634ADFF8B09183
:10DBA800B2F90020771C0192604AFBF79AF9FDF759
:10DBB8000DFC304602F071FC554802F0F1FB544967
:10DBC800D9F80000FBF728F8514809F0A2FAFFB28B
:10DBD800C1B2092909D84B1CDBB2214420224A7260
:10DBE8000021E21891721946F3E7DFF82481D9F889
:10DBF80004004144FBF710F8FDF7E8FB384602F053
:10DC08004CFC404602F0CCFB4146D9F80800FBF733
:10DC180003F8404609F07DFA0236F6B2C7B2092F7A
:10DC280009D87B1CDBB2274420227A720021E21833
:10DC380091721F46F3E73E4BB3F9000005F08CFEE6
:10DC480008EB0701FAF7E8FFFDF7C0FB304657E09D
:10DC58000026384F3B78B34240F240810E2E00F048
:10DC68003D817008013002F018FC304604F0E8FDF0
:10DC78003B78B34206D9202002F077FB701CC0B273
:10DC880004F0DEFD0236F6B2E3E72B4E2B4996F898
:10DC9800B0271F48FBF725F9012002F0FEFB1C48BE
:10DCA80002F07EFB264B27491F7819483A46FBF7B6
:10DCB80018F9022002F0F1FB154802F071FB0C2361
:10DCC80003FB0766204996F8B32796F8B237104841
:10DCD800FBF707F9FDF77AFB032002F0DEFB0C489F
:10DCE80002F05EFB96F8B81796F8B62796F8B7379D
:10DCF800074800911549FBF7F4F8FDF767FB042086
:10DD080002F0CBFB024802F04BFBE7E01C100020BE
:10DD18006D24002062C1010875C10108221000208D
:10DD2800F4D501084C2D0020F810002079C1010815
:10DD3800B0210020742A0020081100207DC10108AC
:10DD4800002D002089C101089AC10108ABC1010852
:10DD5800A42100207C4B1B681B0640F1BB80236A72
:10DD6800616A7A4A8B421CBF536292F828304FF09E
:10DD780001011CBF013303F003034FF0000018BF7B
:10DD880082F8283002F095FB94F82830704A002673
:10DD9800D05C02F0EAFA0220012102F08AFB6D4B06
:10DDA8003620F35C0136C3EBC30393FBF0F0C0B23B
:10DDB800062828BF06206038C0B202F0D6FA102E16
:10DDC800EDD1654B65491B78654813F0020F654B2B
:10DDD8001A7814BF59234E23FBF783F8FDF7F6FA98
:10DDE800022002F05AFB5E4802F0DAFA5E495F4B05
:10DDF8004E680A685A4892FBF3F25D4996FBF3F3C2
:10DE0800FBF76FF8FDF7E2FA032002F046FB5448EF
:10DE180002F0C6FA574B58491A885148FBF761F87F
:10DE2800FDF7C0FA042002F038FB4D4802F0B8FABA
:10DE3800524B53491A884A48FBF753F8FDF7B2FA90
:10DE480004210A2002F035FB454802F0A9FA4D49A1
:10DE5800E26A4348FBF745F84B4EFDF7A3FA052065
:10DE680002F01BFB3E4802F09BFA7268B368474910
:10DE78003B48FBF736F8FDF795FA05210A2002F032
:10DE880018FB374802F08CFA3369F2684049D21A15
:10DE98003348FBF726F8FDF785FA062002F0FDFA6D
:10DEA8002F4802F07DFAB2683A492D48FBF719F875
:10DEB800FDF778FA06210A2002F0FBFA284802F05A
:10DEC8006FFA35491522264809F04EF9FDF76AFA26
:10DED800072015E7F37843F00203F370002D30D1E3
:10DEE8002E4B002193F820301220052B97BF2C4A87
:10DEF8003F259B181D7F02F0DCFA284602F035FA10
:10DF08001320002102F0D5FA264B1B78002B264B54
:10DF180018BF72201B7808BF2120002B18BF522081
:10DF280002F023FA1420002102F0C3FA94F83050CA
:10DF3800074B585D013505F0030502F016FA84F821
:10DF4800305003B0BDE8F083542D00206424002035
:10DF5800BDC10108AD100020FC180020C2C1010895
:10DF68006D240020021900200419002080969800D2
:10DF7800D3C10108FE180020E0C101086410002088
:10DF8800E8C10108EFC10108A4070020F6C1010893
:10DF9800FFC1010806C20108C0020020C42F0020EA
:10DFA80040A201085B0E0020C00E0020026D70B573
:10DFB80015880446ADB2A90613D5036B8BB9C36A9D
:10DFC8001BB1908880B298470BE0E169928840695C
:10DFD8004E1CD2B2E6614254E169E268914228BF20
:10DFE800E3612B0613D5636AA26A9A42236D0AD0AD
:10DFF800511CA069A162825C9A802369994206D368
:10E008000023A36270BDDA6822F08002DA6070BD76
:10E01800026B0346C16810B5406942B11A6C8C1A8C
:10E02800013A08BF0A46005D1A64C0B210BD1A6AF8
:10E03800805C01328A4228BF0022C0B21A6210BD39
:10E04800436B13B190F844007047836A406A1B1A07
:10E05800584258417047036B13B15B68016C01E08B
:10E06800C369016A8B423CBFC2689B18581AC0B288
:10E078007047836A8169426B1944D160416A994249
:10E0880097BF0169CB1ACB1A536096BF0023536020
:10E0980083624FF0000380F84430136888BF8162C0
:10E0A80043F0010313607047436A8269D154436A9D
:10E0B80002690133934228BF00234362436B1BB1BB
:10E0C8001B68DB0705D4D4E7026DD36843F08003EF
:10E0D800D360704738B50D4B0D4D99680D4B1A68D4
:10E0E8001C465288114203D0FCF76CFA286007E0FE
:10E0F800FCF768FA2B68984282BFC01A064B186072
:10E1080023685A68054B5A6138BD00BF000C0140AE
:10E1180098240020A00700200400002000040140EB
:10E128004171FAF719B98160FAF716B92DE9F0418A
:10E1380005460E46078A83899BB21F40002F37D0B9
:10E14800B7FA87F24FF00043D340DB4399B21F4040
:10E15800A2F11B032982042BF0D8DFE803F0221F69
:10E168001C190300746A24B1013C0023A4B2736231
:10E1780001E0AC8DA4B2D6F82080B8F1000FDDD054
:10E18800D8F80030404621469847D8F80480F4E78C
:10E198003068A98E08E07068298F05E0B068A98FFB
:10E1A80002E0F068B5F84010036889B29847C5E7FF
:10E1B800BDE8F081254B10B55A43254B254C1B680B
:10E1C8000139B3FBF2F20388013AA04289B292B254
:10E1D8009BB212D004F50064A0420ED0B0F1804F7B
:10E1E8000BD0A4F59834A04207D004F58064A0426F
:10E1F80003D004F58064A04202D123F070039BB2DF
:10E20800154CA04206D004F58064A0421CBF23F43C
:10E2180040739BB203800F4B8185984202850FD0D3
:10E2280003F5006398420BD003F54063984207D08A
:10E2380003F58063984203D003F58063984201D1C7
:10E24800002303860123838210BD00BF40420F00D4
:10E2580060000020002C01400010004073B5054606
:10E268000068FFF7A7FF2A680124138800269BB2DD
:10E2780043F001031380EB7A01A88DF804308DF880
:10E2880005408DF806608DF8074004F067F8EB7AD2
:10E298001B2B0BD1192301A88DF804308DF80540EC
:10E2A8008DF806608DF8074004F058F802B070BD8C
:10E2B8000C4B800A98420CD004D8B0F5801F0CD1C2
:10E2C80001207047084B984205D04933984206D040
:10E2D80003E00220704703207047FE2070470020AB
:10E2E800704700BF01001000020010002DE9F8433C
:10E2F80004680746204688469146FFF7D9FF032859
:10E308004BD8BA7A9108B8F1000F06D1A589AEB2F8
:10E3180002258D4026EA0505A5810A2303FB001383
:10E328001F4A42F82380043342F82390B8F1000FC3
:10E3380007D0BD7AA189AD080223AB400B439BB23D
:10E34800A3812823434303F120011144EFF31286EC
:10E35800502585F3128803F10C051C33154413442A
:10E3680055F8047F17B10F60296804319D42F7D131
:10E3780000230B60F3B283F31188282303FB0020EA
:10E38800036A23B1A3899BB243F0010304E0A38984
:10E3980023F001031B041B0CA381BDE8F88300BF15
:10E3A800CC1F002096E695E694E60148FEE500BFFE
:10E3B8009C2400200048F9E5F02400200B4B4FF482
:10E3C80000525A604FF6FE730948D0F88C20116845
:10E3D8000B401360C26FD0F880309A4201D0583099
:10E3E80047E6012380F89C30704700BF00000240D8
:10E3F800982400202DE9F0431E46984B8DB0984292
:10E40800894690469DF8507057D1954B954A964944
:10E418009A6503F1AC02DA6603F5D6721A674FF40F
:10E4280080725A669A66914AC3F86080C3F8882059
:10E43800A2F54842543AC3F8A420C3F8A020C3F870
:10E44800A800C3F88C108A4B9A6942F480429A61FA
:10E458005A6942F001025A6102238DF803303A07E3
:10E468004FF40073ADF8003001D51C230FE0B3075B
:10E4780006D518237F4869468DF8023001F014FE4E
:10E48800F5070AD54FF48063ADF800304823794882
:10E4980069468DF8023001F007FE0E238DF804302E
:10E4A8000022012301A88DF805308DF806208DF88B
:10E4B8000730714C03F052FF4FE0704B984240F028
:10E4C800C880674B674AC3F80C805A604FF4807263
:10E4D8005A611A6103F52B729A6103F56B72DA615E
:10E4E800674A5865DA641A65614B3C07DA6942F491
:10E4F8000032DA615A6942F001025A614FF00203B0
:10E508008DF803304FF00403ADF8003001D51C231B
:10E518000EE0B00706D51823564869468DF8023034
:10E5280001F0C2FDF10709D50823ADF800304823F2
:10E53800504869468DF8023001F0B6FD26238DF863
:10E5480004300022012301A88DF805308DF806203B
:10E558008DF8073003F002FF4A4C002501232046BE
:10E5680084F844302562E561A5626562C4F82C90A0
:10E578006671C4F80880A771F9F7EEFEF20731D585
:10E58800206B002826D0E36C039501934FF4805349
:10E598000A9380230693E36805950493202309933F
:10E5A80063690795029308950B9501F043F801A953
:10E5B800206B01F021F8226B216D136843F00103F1
:10E5C80013608B8A9BB243F040038B8253689BB2E3
:10E5D800236407E04FF6DF72236D1A80DA6842F091
:10E5E8002002DA60B3072CD5606B28B3A36C002532
:10E5F80001934FF480530A9380230693236902956D
:10E6080004931023039305950795089509950B9591
:10E6180001F010F8606B01A900F0EEFF636B1A6857
:10E6280042F002021A60226D5D605D60938A9BB2BF
:10E6380043F08003938204E0226DD36843F08003A3
:10E64800D360226D204693899BB243F40053938193
:10E6580000E000200DB0BDE8F08300BF00380140A5
:10E668009824002064A20108440002405800024097
:10E678000010024000080140F0240020004400403F
:10E68800044400409C24002038B500240B4D6059F8
:10E69800254403F059FC696811B10948FAF736FCBA
:10E6A800A96811B10748FAF731FC0748103403F09C
:10E6B8004BFCB4F5E87FE9D138BD00BF7CA2010866
:10E6C8003FC2010845C20108ADCA0108F0B585B0CE
:10E6D800044608F01EFD082826D1621EE01D1F49C9
:10E6E80012F8013F09681944497801F00301022929
:10E6F80008BF203B82421370F1D1254604F1080778
:10E7080015F8016B1648314608F0F5FC20B128468B
:10E71800314608F0F0FC10B1FBF7F0F81CE0BD4200
:10E72800EED1204600F0D0FE0E4803F00DFC002389
:10E738000D4A04A91A4492F88A210A440849595CE6
:10E748000133082B02F80C1CF2D10023074801A959
:10E758008DF80C30FAF7DAFB05B0F0BD6800002040
:10E76800F8D501084BC2010808110020EFC90108BB
:10E778002A4B2B4C1E6880B52068FBF785FC304679
:10E78800FBF782FC206841798D0703D441F0020130
:10E79800FBF7E2FF234B08221A61234D10221A616E
:10E7A8002B689A0341BF06236371E37923F00103C1
:10E7B80044BF43F00203E3712068FBF7D9FF90B12F
:10E7C800184F08237B61164B1868FBF7CEFF80466D
:10E7D800FEF778F808B102F047F830464146FBF7F3
:10E7E800CAFF08233B613046FBF7C2FF78B10D4FE3
:10E7F8004FF01008C7F814803046D4F80090FBF7A3
:10E80800B4FF01464846FBF7B6FFC7F810802B68EF
:10E818009B03D1D5FFF723F8CEE700BF1C2D0020BE
:10E8280044290020000C0140542D00202DE9F04718
:10E83800054608F06EFC2F4E0446D6F8088090B9BD
:10E848002D4803F081FB2D4B53F8241049B10123C7
:10E85800A34013EA080F02D02948FAF757FB0134FE
:10E86800F1E7284822E028462749224608F05AFCC2
:10E8780058B9264803F068FB254C54F8041F0029B2
:10E88800EFD01F48FAF742FBF7E72B784FF0000963
:10E898002D2B03BF013504F1FF344FF0010A4FF06F
:10E8A800000A164B53F8297027B91A48BDE8F047F3
:10E8B80003F04ABB28463946224608F033FCA8B97B
:10E8C800012000FA09F0BAF1000F03D0FAF7B2FC00
:10E8D800114803E040EA0800B060104803F034FB38
:10E8E8003946BDE8F0470E48FAF710BB09F10109AF
:10E8F800D7E700BF0811002051C201084CA4010845
:10E908005BC20108ADCA01085FC2010864C2010800
:10E9180048A4010886C0010870C2010879C201082C
:10E92800EEC9010810B5084803F00EFB074B002498
:10E938001C741C64064B1C70FCF7BEF803F0DCFC6E
:10E94800044B1C6010BD00BF81C20108442900208F
:10E95800843100201C2D002070B5064600240B4B86
:10E96800E518AA8816420AD0E1580948FAF7CEFAFB
:10E978002846002103F079FA064803F0E5FA40F644
:10E98800BC4314349C42EAD170BD00BFACAB010853
:10E99800ADC20108ADCA010808B50848FAF7B6FAC9
:10E9A800FEF7FEFC01F082FC18B96420FBF731FE8B
:10E9B800F8E70348BDE80840FAF7A8BAB7C2010863
:10E9C800C4C201082DE9FF410A48068885684488C1
:10E9D800B0F80480C768FEF7EBFBCDF80080029022
:10E9E800019731462A4623460348FAF78FFA04B0BE
:10E9F800BDE8F08110000020CCC20108F0B5047811
:10EA08008BB005460CB1002436E04B4B19680E2339
:10EA180003FB0411B1F91D51B1F91921B1F91B31E9
:10EA2800009591F8205101F58C70019591F82151CC
:10EA380001F59071029590F90700039091F9021081
:10EA48003E48049121460134FAF760FA082CDCD1DB
:10EA580070E02D2B14D1072C1BDC284608F0AEFBE8
:10EA68000AAB661C03EB440424F8100C15F8013FAC
:10EA7800303B092BFAD934462B78002BE9D104E036
:10EA8800A3F13002092A09D8E5E7082CBDF81820B7
:10EA980009D00BB0BDE8F040FAF730BF202BF8D111
:10EAA80001352646E7E7072AF3D840F2DC55BDF8DA
:10EAB8001A00214BA0F2EE2189B2A9421B68E8D8BE
:10EAC800BDF81C10A1F2EE24A4B2AC42E1D8BDF806
:10EAD8001E6004B237B2A742DBDB0DB2AF42D8DC0E
:10EAE800A542D6DBBDF8247007F16404A4B2C82C93
:10EAF800CFD8BDF826E00FFA8EF4112CC9DCBDF88A
:10EB08002050B42DC5D8BDF82240B42CC1D812B2BB
:10EB18004FF00E0C0CFB0233A3F81901A3F81B11DC
:10EB2800A3F81D6183F8205183F8214183F81F71F0
:10EB380083F822E10BB0F0BD3810002029C301088A
:10EB4800F0B504468FB0204608F0E3FAC5B21DBB05
:10EB5800AB4803F0F9F9AB4C94F8D61009B9AA48B8
:10EB680053E049B294F8D42094F8D530009194F841
:10EB7800D710A648019194F9D8100734029194F956
:10EB8800D210039194F8D310049129460135FAF76D
:10EB9800BDF9102DE0D1E2E720469D49052208F095
:10EBA800C1FA0546B8B929469A48702208F06DFAA4
:10EBB8002846994B19680E2303FB001301300022E5
:10EBC800082883F8232183F8242183F8252183F852
:10EBD8002621F0D112E120469049042208F0A2FA39
:10EBE80005462046002D4AD1202108F084FA002845
:10EBF80000F00481461C304608F08BFA2C46074684
:10EC0800874B53F824502DB986480FB0BDE8F04023
:10EC1800FAF77CB930462946FAB208F083FA01348B
:10EC28000028EDD1774A164602F17001002382F8D8
:10EC3800DA3082F8D63082F8D53082F8D43007320C
:10EC48008A42F3D1784901EBC40191F82822934212
:10EC580010DAD1F82C72C3EBC302B0183A44176823
:10EC680000F1D401C0F8D47090880133888092797B
:10EC78008A71E7E729466D48FAF748F98FE06C4949
:10EC8800072208F04FFA05462046002D49D12021D9
:10EC980008F031FA064608F03CFAC4B26CBB654885
:10ECA800FAF734F9214664480134FAF72FF90E2CA3
:10ECB800F8D15548FAF72AF9002460482146FAF7AE
:10ECC80025F90025544A012311680E2202FB04127B
:10ECD800D2F82321AB401342594B5A495A4808BF2E
:10ECE80019460135FAF712F90E2DEBD146480134D1
:10ECF800FAF70CF9082CE0D180E03046534908F0C7
:10ED080061FA2C4600284CD0022C4FD008F056FA55
:10ED180006AB43F824004D49002008F053FA0134AB
:10ED2800F0E74A4908F04EFA002460B1082C38D0C0
:10ED380008F044FA06AB43F824004449002008F0E0
:10ED480041FA0134F1E7082C2BD1069B0F2B28D868
:10ED5800DDF81CE0BEF1070F23D8089F0D2F20D83F
:10ED6800099E06F16402C82A1BD80A9DFF2D18D8EF
:10ED78000B98642815D80C99642912D8884210DA9F
:10ED88000D9C032C0DD8324AC3EBC303134483F8FC
:10ED980004E05F719E71DD71187259729C722D4C7E
:10EDA800D1E60FB0BDE8F040FAF7A8BD069B072BE7
:10EDB80020D807990D291DD80278722A0DD06E2AFD
:10EDC80018D1154A0E20126800FB032301228A403D
:10EDD800D3F8231121EA020209E00F4A0E20126833
:10EDE80000FB032301228A40D3F823110A43C3F806
:10EDF800232101E0FAF782FD0D4CA4E60FB0F0BD27
:10EE080051C3010808110020ADCA01087CC30108DC
:10EE180056C00108DC1100203810002081C001080C
:10EE280068B8010886C001087CA2010895C00108DD
:10EE380049C3010849C2010898C30108ECC1010887
:10EE4800C2CE010808CE01089DC30108A1C301086C
:10EE5800D81100206BBD01082DE9F7430478054659
:10EE68008CB9324D95F8AB12B5F8A82295F8AA32AC
:10EE78002F48009121460134FAF748F8102C05F183
:10EE88000405EFD14EE008F099F90F28044636DC66
:10EE98002846202108F02FF9264EE4B2D6F84480FF
:10EEA800451CA4000027284608F088F95FFA87F96E
:10EEB800B9F1010F83B208D0B9F1020F0BD0B3F545
:10EEC800B47F24D2726C13530AE0FF2B1FD8736CE3
:10EED8002344987004E0FF2B19D8736C2344D8702E
:10EEE80028462C2108F007F9054608B1013502E04B
:10EEF800B9F1020F0BD10137032FD4D112E00E481C
:10EF080000210F2203B0BDE8F043FAF774BC08EB08
:10EF180004000021042208F0B8F803B0BDE8F0436B
:10EF2800FAF7ECBC03B0BDE8F08300BF081100207D
:10EF3800A3C301084429002014C001082DE9F04F9B
:10EF4800AB498BB0044608F0A9F8AA490028204626
:10EF58000CBF0125072508F0A1F8A749002820467D
:10EF680008BF022508F09AF8002808BF0425E90719
:10EF780040F1E680A14802F0E7FF002002F0F4FD2E
:10EF88009F4CA04802F0E0FF9F4802F0DDFF637944
:10EF98009E4A013B52F823109D48F9F7B7FF9D4858
:10EFA800F9F7B4FF26460027D6F81480002140461A
:10EFB80004F0BAFE20B19848F9F7A8FF002669E0E6
:10EFC80039469648D6F818B0D6F81CA0D6F820903E
:10EFD800F9F79CFF4046002104F0B0FE10B1202054
:10EFE80002F0AAFF06A94046F9F716FE01468C482A
:10EFF800F9F78CFF5846002104F0A0FE10B120203C
:10F0080002F09AFF06A95846F9F706FE0146844819
:10F01800F9F77CFF5046002104F090FE10B1202043
:10F0280002F08AFF06A95046F9F7F6FD01467C482A
:10F03800F9F76CFF4846002104F080FE10B120204B
:10F0480002F07AFF06A94846F9F7E6FD01370146BE
:10F058007448F9F75BFF0C2F06F11006A4D1AAE754
:10F0680049B294F8D42094F8D530009194F8D71088
:10F078006D48019194F9D8100734029194F9D2108F
:10F08800039194F8D310049131460136F9F73EFF05
:10F09800102E03D094F8D6100029E1D1634802F06D
:10F0A80053FF574B624C9F6854F8041F19B16148CD
:10F0B800F9F72CFFF8E70E465F4B53F826404CB1A2
:10F0C8000123B3403B4203D05C482146F9F71EFFB9
:10F0D8000136F1E75A4802F037FF2146484B0AAAA1
:10F0E8000B4493F88A311344564A8A5C0131082943
:10F0F80003F8102CF2D1002306A953488DF82030CC
:10F10800F9F704FF514802F01FFF5148FBF736F8A2
:10F11800504802F019FF4E48FAF7F6FB4E4802F045
:10F1280013FF4B48FFF798FE4C48F9F7EFFE4020D5
:10F13800FFF712FC4A4802F007FF4548FAF708FFB4
:10F14800AA0739D5474802F0FFFE474802F0FCFEFF
:10F158003F4802F049FD454802F0F6FE3C48FAF700
:10F1680057FB434802F0F0FE3948FAF743FE41489E
:10F17800F9F7CCFE3648FAF7D3FC3F4802F0E4FE34
:10F188003348FFF73BFC00260E27774300243B4A11
:10F198000123926CA3403A44D2F80A2013421ED1AC
:10F1A80001340E2CF3D10136082EEDD12B48F9F796
:10F1B800ADFE8020FFF7D0FB6B0716D5304802F074
:10F1C800C3FE304802F0C0FE214802F0E7FC2348A5
:10F1D800F9F79CFE4FF48070FFF7BEFB05E031465F
:10F1E80022462948F9F792FEDAE70BB0BDE8F08F1E
:10F1F800B7C3010800C80108BEC30108C4C3010899
:10F2080008110020D2C30108E4C3010868B8010846
:10F21800F0C30108FBC3010808C4010815C40108AC
:10F2280048C20108EFC901082DC401081DC401081E
:10F2380048A401084CC401084CA401085AC4010898
:10F2480067C40108F8D5010873C401087CC4010823
:10F258006BBD01088BC4010897C40108ADCA010839
:10F26800A5C40108B2C40108C5C40108D3C4010873
:10F27800DDC40108ECC40108FAC4010844290020CF
:10F2880006C5010817C5010829C50108084BDA6831
:10F29800D10709D4DA68520708D4DB6813F0100FD5
:10F2A80014BF0320042070470120704702207047D4
:10F2B8000020024070477047704703788B4286BF32
:10F2C800024B33F811000020704700BF902900203E
:10F2D8000021062207F0D9BE0021062207F0D5BE7C
:10F2E80070B50546FBF76EF9324CA369A061C31AE5
:10F2F800B3F5FA5FE36182BF002384F8203084F815
:10F30800213094F820302BB9A12D02BF294A0121C0
:10F3180082F8211094F82110264A31B1D118EDB2A3
:10F32800013381F8225082F8203094F8205094F864
:10F338004330AB423CD11F4B93F84430052B02D0ED
:10F34800062B03D02FE0002004F08CF994F823302A
:10F358001E2B28D100200246C1B26B1E99421ADA30
:10F36800214491F822300821DBB283EA0206F6072D
:10F3780044BF83F01803C3F3460301F1FF3154BFC0
:10F388005B0843F0800311F0FF01C2F34702ECD1A0
:10F3980001301A46E0E7234493F822309A4202D11A
:10F3A800032004F05FF9002384F8213084F820302A
:10F3B80070BD00BF9029002010B50446B0F90000C8
:10F3C80002F049F9B4F9020002F045F9B4F9040071
:10F3D800BDE8104002F03FB910B50446006802F0DD
:10F3E8003AF9606802F037F9A068BDE8104002F009
:10F3F80032B92DE9F74F0120FAF786FF002488B3C8
:10F40800012C2FD84FF04C0909FB04FA174E06EBD4
:10F418000A0808F19007BD7815B10134E4B2EEE7A7
:10F4280090F9003090F804E01846114B03228DE85B
:10F43800240001212A4653F82E30FAF743FE83466A
:10F4480060B106F14800504429464A4607F01DFEBF
:10F4580001231C44C8F848B0BB70E4B20120FAF795
:10F4680039FFCCE703B0BDE8F08F00BF902900203A
:10F4780034A601080021222210B5104807F005FE25
:10F488000F4B002219460F480424105C013283F800
:10F49800F60183F8FB4105200024042A83F8FA01C9
:10F4A80083F8FD4183F8FC0103F10803EBD1012344
:10F4B800A1F8F831522381F8F43110BDFC12002074
:10F4C8000811002071C9010870B50646441E14F8D9
:10F4D800011F89B1094D284607F00DFE0028F6D016
:10F4E80005F1080398423FBF054B401BC018A31BFA
:10F4F80038BF80F88A31EAE770BD00BFF8D5010847
:10F508000811002007B51C4B03F1E402C3F8E02002
:10F518001A4A92F892215AB1012A14D1032183F888
:10F52800E610072183F8E82083F8E7100C2208E0AA
:10F53800022183F8E610032183F8E82083F8E71016
:10F54800072283F8E4200E4A0E4B40201A60FAF78F
:10F55800DBFE70B10122002390F9000040218DE804
:10F568000C00094A4FF4E133FAF7ACFD003018BF3C
:10F57800012003B05DF804FB902900200811002049
:10F588002934010834000020D93401080120002161
:10F5980002F038BC174AF0B5164692F8E930D2F8AE
:10F5A800ECE0032B10D85C1C0EEBC3039D1CE4B2EB
:10F5B80008D09A88D10705D5104203D008E0013158
:10F5C800042907D12346ECE786F8E9300020F0BD8E
:10F5D8009F7800210C2202FB01F3064D05F1F00C87
:10F5E8001CF803209742EAD12B4485F8E940D3F868
:10F5F800F400F0BD902900208A6810B50C6A0368F1
:10F6080014430A6923F4FF4314434A6923F070033F
:10F6180014438A691443CA6914434A6A14438A6AB8
:10F62800224313430360CB6843600B6883604B68D5
:10F63800C36010BD4FF6FE730268134003600023D9
:10F64800036043608360C360284B984201D1284A15
:10F6580027E0284B984201D1254A2AE0264B9842B8
:10F6680001D1234A2DE0254B984201D1204A30E0B0
:10F67800234B984201D11E4A33E0224B984204D1D1
:10F688001B4A536843F470032EE01F4B984204D181
:10F69800174A536843F0706326E01C4B984204D124
:10F6A8001B4A536843F00F031EE01A4B984204D1DB
:10F6B800174A536843F0F00316E0174B984204D1F9
:10F6C800134A536843F470630EE0144B984204D114
:10F6D8000F4A536843F4704306E0114B984204D133
:10F6E8000B4A536843F47023536070470800024084
:10F6F800000002401C00024030000240440002406A
:10F70800580002406C000240800002400804024099
:10F71800000402401C040240300402404404024039
:10F7280058040240224A10B5536803F00C03042B16
:10F7380003D0082B04D01F4B14E01F4B5B6811E06B
:10F7480053685168C3F38343C90303F1020301D427
:10F758001A4906E0516811F4003F1749496818BF73
:10F7680049084B4303605368154CC3F30313234400
:10F7780093F820100368CB4043605168C1F302211D
:10F78800214491F8201023FA01F181605168C1F3F6
:10F79800C221214491F82010CB40C3605268C2F3C3
:10F7A8008132224492F83020B3FBF2F3036110BD9A
:10F7B8000010024000127A003400002000093D00C9
:10F7C80034A6010810B50446FFF760FD012806D1EC
:10F7D8001CB1FFF75BFD013CF8E7052010BD002CCC
:10F7E80008BF052010BD0A88F0B54B888E88B1F88F
:10F7F80008E0CC88002A3AD1028C43F0010322F0B9
:10F8080001021204120C0284058B078CADB225F09C
:10F81800F30545EA0E1189B241EA06027A49BFB2F8
:10F82800884212D001F5006188420ED0B0F1804FB5
:10F838000BD0A1F59831884207D001F58061884244
:10F8480003D001F58061884202D127F0020701E068
:10F8580027F00A071F4302830784038B23F00C0356
:10F868001B041B0C0383038B9BB21C4344E0042A38
:10F8780044D1028C22F010021204120C0284018B73
:10F88800058C21F440721205120D42EA0E325E49CF
:10F8980092B242EA06228842ADB292B212D001F583
:10F8A800006188420ED0B0F1804F0BD0A1F598319D
:10F8B800884207D001F58061884203D001F5806154
:10F8C800884207D125F0200141EA03139BB243F097
:10F8D800100304E025F0A00143F010030B4302835A
:10F8E8000384038B23F440631B041B0C0383038BE7
:10F8F8009BB243EA0424A4B20483F0BD082A028C14
:10F908003ED122F480721204120C0284828B3E4D86
:10F9180092B222F0F307018C47EA0E1292B2A84283
:10F9280089B242EA060212D005F50065A8420ED057
:10F93800B0F1804F0BD0A5F59835A84207D005F552
:10F948008065A84203D005F58065A84207D121F457
:10F95800007141EA03239BB243F4807304E021F46D
:10F96800206143F480730B4382830384838B23F0E9
:10F978000C031B041B0C8383838B9BB21C4341E049
:10F9880022F480521204120C0284858B018C25F417
:10F9980040752D052D0D45EA062545EA0E321A4D0E
:10F9A80089B2A84292B212D005F50065A8420ED0DD
:10F9B800B0F1804F0BD0A5F59835A84207D005F5D2
:10F9C8008065A84203D005F58065A84207D121F4D7
:10F9D800005141EA03339BB243F4805305E047F6F4
:10F9E800FF5543F480530D402B4382830384838B5C
:10F9F80023F440631B041B0C8383838B9BB243EA71
:10FA08000424A4B28483F0BD002C0140016830B501
:10FA1800CD43154B1C682C401C605A682A405A601C
:10FA2800027902F1804202F58232146821431160A2
:10FA380002689C68D5432C409C60D9682940D960ED
:10FA48004179102909BF996801F1804311439960F0
:10FA580015BF03F58233D96819680A4316BF0A43EC
:10FA6800DA601A6030BD00BF00040140CA78F0B502
:10FA7800D40648BF8C780D8802F00F0348BF234393
:10FA880015F0FF0F1DD0016800240126A64006EAE4
:10FA98000507B74211D14FEA840E0F2606FA0EF673
:10FAA80021EA0601282A03FA0EF641EA060101D1E5
:10FAB800476102E0482A08BF07610134082CE4D1F5
:10FAC8000160FF2D1FD94168002404F108070126B1
:10FAD800BE4006EA0507B74211D14FEA840E0F2649
:10FAE80006FA0EF621EA0601282A03FA0EF641EA7A
:10FAF800060101D1476102E0482A08BF07610134C5
:10FB0800082CE2D14160F0BD0F4B1A6842F00102A7
:10FB18001A6059680D4A0A405A601A6822F08472BD
:10FB280022F480321A601A6822F480221A605A6815
:10FB380022F4FE025A604FF41F029A60044B4FF001
:10FB480000629A60704700BF001002400000FFF892
:10FB580000ED00E02DE9F8435B4C0368013AC4F876
:10FB6800203183880D46A4F82431072A42D8DFE8DB
:10FB780002F0040A101822292F35B4F820310B801E
:10FB8800B4F8223113E0B4F822310B80B4F82031F4
:10FB980005E0B4F820315B420B80B4F822315B42B7
:10FBA80005E0B4F822315B420B80B4F820316B8059
:10FBB800B4F824311DE0B4F820315B420B80B4F86E
:10FBC800223112E0B4F822310B80B4F820310CE075
:10FBD800B4F820310B80B4F8223105E0B4F82231B2
:10FBE8005B420B80B4F820315B426B80B4F824315F
:10FBF8005B42AB80354B1B7A002B62D1B5F9000014
:10FC080003F0AAFE8046B5F9020003F0A5FE0746F8
:10FC1800B5F9040003F0A0FED4F8281106464046C2
:10FC280003F0EEFED4F834118146384603F0E8FEBE
:10FC38000146484603F0DCFDD4F8401181463046C1
:10FC480003F0DEFE0146484603F0D2FD07F02AFC29
:10FC5800D4F82C112880404603F0D2FED4F838118D
:10FC68008146384603F0CCFE0146484603F0C0FD05
:10FC7800D4F844118146304603F0C2FE0146484696
:10FC880003F0B6FD07F00EFCD4F83011688040464A
:10FC980003F0B6FED4F83C118046384603F0B0FEB7
:10FCA8000146404603F0A4FDD4F848110746304603
:10FCB80003F0A6FE0146384603F09AFD07F0F2FB72
:10FCC800A880BDE8F88300BF9029002034000020F8
:10FCD80038B50F4B1B689C890E4B186880F31000D1
:10FCE800201A03F039FE0C4903F08AFE0546204627
:10FCF80003F032FE0146284603F036FF04F046F8CA
:10FD08006428A8BF642020EAE070C0B238BD00BFF4
:10FD1800E4180020F41800200000C84244F6FB71E3
:10FD2800084B1A68137803EB431300FB031350784E
:10FD3800C0EB0030B3FBF0F39078B3FBF0F080B287
:10FD4800704700BFE418002008B50A480A2290F856
:10FD58004D3100EB4303B3F85C1100F5B47089B280
:10FD680020F8041CFAF70AFD80B2FFF7D7FF024B10
:10FD7800188008BD90290020E818002037B5062211
:10FD8800044603216B461E2001F06AFE9DF80130EF
:10FD98009DF80000154D43EA002000B203F0DCFD99
:10FDA800296803F02DFE03F0F1FF9DF80330208051
:10FDB8009DF8020043EA002000B203F0CDFDA968D7
:10FDC80003F01EFE03F0E2FF9DF80530A0809DF8C9
:10FDD800040043EA002000B203F0BEFD696803F0A6
:10FDE8000FFE03F0D3FF608003B030BD4000002059
:10FDF8001FB5044602210C2001220DF1070301F072
:10FE08002FFEC8B39DF80730DB0735D5032106223E
:10FE180002AB0C2001F024FE0C20092101220DF177
:10FE2800070301F01DFE38B39DF8073013F00C0FDF
:10FE380022D19DF809209DF808300C2043EA0223BE
:10FE4800C3EB83339B009DF80B2023809DF80A3079
:10FE58000A2143EA0223C3EB83339B009DF80D205C
:10FE680063809DF80C3043EA0223C3EB83339B0085
:10FE7800A380012201F034FE04B010BD07B50A21A9
:10FE880000220C2001F02CFE1420FAF7C2FB0A21F4
:10FE98000F220C2001F024FE0A20FAF7BAFB01AB6E
:10FEA800102103220C2001F0DBFD0A20FAF7B1FB38
:10FEB8000A2100220C2001F013FE0A20FAF7A9FB00
:10FEC8000DF10303022101220C2001F0C9FD0DF1FF
:10FED8000303092101220C2001F0C2FD0A2101229D
:10FEE8000C2001F0FDFD03B05DF804FB2DE9F0479F
:10FEF800664D2B686649581C0A788E4602F0FF0644
:10FF08000AB10346F6E737462B60687BAB6895F87D
:10FF18000C80AA7B39B2202900F09C80DFF880C1D0
:10FF28000CEB8103DC789B783CF82110C3F1FF03CC
:10FF38009BB2002B65D04FF03C0CB1FBFCF9C3F130
:10FF4800FF0363431B12B9F1050F5DD8DFE809F021
:10FF5800030B1A293A4AE01A4143B1FBFCF0DAB222
:10FF68001044C0B251E0B1FBFCF00CFB101189B297
:10FF7800DAB2C1F13C01E31A4B43B3FBFCFC204667
:10FF880094442CE0B1FBFCF00CFB1011E21A89B28E
:10FF98004A43B2FBFCF25FFA83F84244D2B22046ED
:10FFA80032E0B1FBFCF90CFB191189B2E01AC1F17E
:10FFB8003C014843B0FBFCF05FFA83F84044C0B210
:10FFC800224621E0B1FBFCF80CFB1811D8B289B22B
:10FFD800E31A01FB03F2B2FBFCFC224684445FFAFD
:10FFE8008CF412E0B1FBFCF80CFB181189B2D8B202
:08FFF800C1F13C01E31A4B4387
:020000040801F1
:10000000B3FBFCF20244D2B203E02246204600E0F9
:1000100044464FEA042C4CEA004C4CEA020C1723ED
:100020004FF0010808FA03F806F1170118EA0C0F5F
:10003000A1EB0301DFF8748014BF4FF011094FF0FA
:10004000090989B213F1FF3308F80190E8D2183694
:100050000137B6B2BFB2114BA0465FE7AB600123D8
:100060008EF8003040F22A33AA730D4AE9800D4918
:1000700085F80C806873AE80536000238B840B88F6
:100080009BB243F001030B80136843F0010313603C
:10009000BDE8F087802B0020813100208C2B0020D0
:1000A0006C00024000040040AA0D0020D502002090
:1000B000F0B5B1F800E000234EFA03F2D50725D5DC
:1000C0008E784FEAD30CF40648BFCC7806F00F02C6
:1000D00003F0070748BF2243BF0050F82C500F24FD
:1000E000BC4025EA0404BA402243282E40F82C20C4
:1000F00005D1C46801229A4024EA020205E0482E94
:1001000004D1C46801229A402243C2600133102BFB
:10011000D2D1F0BD2DE9FF41604B1B689BB11A683D
:100120001AB15F49886902438A619A889868ADF874
:10013000042002228DF8072004220DEB02018DF825
:100140000620FFF7B5FF3220FAF767FA00211122E7
:100150001E2001F0C9FC012160221E2001F0C4FC18
:100160006420FAF75AFA002402A8FFF70BFE27468C
:1001700026460A25022101221E2001F0B5FC32206C
:10018000FAF74BFA02A8FFF7FDFDBDF90820BDF90B
:100190000A1014448A42A8BF0A46BDF90C300F4425
:1001A00093421E44A8BF134613F5805F09DD3D4A04
:1001B000013DD36883F01003D360DBD14FF0010819
:1001C00001E04FF000081E200021122201F08CFCFB
:1001D0000A25022101221E2001F086FC3220FAF7B6
:1001E0001CFA02A8FFF7CEFDBDF90820BDF90A10E0
:1001F000A41A8A42A8BF0A46BDF90C307F1A93425E
:10020000A6EB0306A8BF134613F5805F07DD254A5A
:10021000013DD36883F01003D360DAD101E04FF0E1
:100220000008204603F09CFB01461F4803F0A0FC99
:100230001E4D20F000402860384603F091FB014637
:10024000194803F095FC20F000406860304603F048
:1002500087FB0146164803F08BFC20F00040A860A5
:10026000002170221E2001F03FFC012120221E20CF
:1002700001F03AFC1E200221002201F035FC64202E
:10028000FAF7CBF9B8F1000F04D14FF07E532B6091
:100290006B60AB6004B0BDE8F08100BFB402002029
:1002A00000100240000C014000406F46400000205A
:1002B00001C05E460F4B73B518781C4698B10523F4
:1002C0000D4D8DF800304FF4805600238DF801302D
:1002D00001A86E616946022202F088F82E619DF83D
:1002E000050000F0010000F00100207080F0010026
:1002F00002B070BD21060020000C0140064B70B515
:1003000006461C461D68FFF7D5FF18B923685B1B1E
:10031000B342F8D970BD00BF782D0020F7B5032394
:100320008DF80430030C8DF805308DF80700030AB2
:1003300006200F4614468DF80630FFF7DFFF78B130
:10034000084D4FF4805601A904226E61002002F08E
:100350004DF838460021224602F048F820462E612A
:1003600003B0F0BD000C0140024640213C2001F0EA
:10037000BBBB70B500EB8000094CA0F1A1059C3817
:1003800025440444074B15F8010F1E787040FFF711
:10039000EBFFA542F6D13046BDE87040E4E700BF70
:1003A00068A601088531002010B5441E14F8010F1D
:1003B00010B1FFF7DEFFF9E710BD024680213C20B7
:1003C00001F092BB10B5D420FFF7F7FF8020FFF7B4
:1003D000F4FFA820FFF7F1FF3F20FFF7EEFFD32047
:1003E000FFF7EBFF0020FFF7E8FF4020FFF7E5FFF6
:1003F0008D20FFF7E2FF1420FFF7DFFFA120FFF7BA
:10040000DCFFC820FFF7D9FFDA20FFF7D6FF122064
:10041000FFF7D3FF8120FFF7D0FFCF20FFF7CDFFFD
:10042000D920FFF7CAFFF120FFF7C7FFDB20FFF756
:10043000C4FF4020FFF7C1FFA420FFF7BEFFA620A6
:10044000FFF7BBFFAF20FFF7B8FFA620FFF7B5FF10
:10045000AE20FFF7B2FF2020FFF7AFFF0020FFF72D
:10046000ACFFB020FFF7A9FF4020FFF7A6FF002058
:10047000FFF7A3FF1020FFF7A0FF4FF48064013CBB
:100480000020A4B2FFF770FF002CF8D18120FFF705
:1004900094FFC820FFF791FFAF20FFF78EFF0120E8
:1004A00010BD08B55038C0B2FFF787FF0020FFF736
:1004B00084FFBDE8084010207FE710B5044650399E
:1004C000C8B2FFF77AFF04EB4400400000F00E00D2
:1004D000FFF773FF06206043BDE81040C0F3031030
:1004E00010306AE7012828BF01202DE9F04F0646A9
:1004F000734F142000FB0671724BD1F8A4421E7595
:100500001C61714BD1F8B422DD69B1F8AC822A4389
:10051000DA61A288B1F8AEA222F44072D1F8A852F2
:10052000120489B0120C4AEA0809A28003A9C5F88E
:10053000109002228DF80E0028460193ADF80C9021
:100540008DF80F20FFF7B4FD019B00971F464FF079
:10055000080BAA6818EA020F03D10A20FAF752F82A
:10056000F7E70A20C5F81480FAF74CF8C5F81080B0
:100570000A20FAF747F8BBF1010BEAD1C5F814A03D
:100580000A20FAF73FF8C5F814800A20FAF73AF87B
:10059000C5F810800A20FAF735F80222C5F810A035
:1005A000284603A98DF80F201C228DF80E20ADF8E7
:1005B0000C90FFF77DFD454A03A894423A690BBFB2
:1005C00042F4001242F480023A613A610BBF3A6988
:1005D0003A6922F4001222F480023A61A38823F4DB
:1005E00040731B041B0CA38023889BB243F00103C0
:1005F0002380A588FFF79AF80599354B25F03F052C
:10060000B1FBF3F32D042D0C1D43ADB2A580228860
:10061000002522F001021204120C22802D4A03A8A8
:10062000B1FBF2F100298AB208BF012242F4004175
:100630004FF4967253434FF47A7293FBF2F3013303
:100640009BB22384A1832388009A9BB243F00103C9
:100650002380238823F4816323F002031B041B0CF3
:1006600023804FF480432381142303FB062696F84E
:10067000B13201248DF80C308DF80D508DF80E50EC
:100680008DF80F4001F06EFE96F8B0329DF80F2005
:100690008DF80C308DF80D508DF80E501AB103A85E
:1006A00001F060FE08E05A0903F01F039C4002F1CC
:1006B0002003094A42F8234009B0BDE8F08F00BF8B
:1006C00068A60108802B0020001002400054004062
:1006D00040420F00804F120000E100E010B54B884F
:1006E000DC0641BF2F4B14791B6853F8244044BFEC
:1006F0002D4B43F820404B889B0641BF294B547932
:100700001B6853F8244044BF274B43F820404B88D4
:100710001C070ED5254B0C781B78B3EB141FA1BF1B
:10072000204BD4781B6853F82440A4BF1E4B43F8D9
:1007300020404B889B070ED51D4B0C781B78B3EBE4
:10074000141FDFBF174B54781B6853F82440DCBFDD
:10075000154B43F820404B88DC070FD5154C0B7820
:10076000247803F00F03A342DFBF0E4B14781B68FD
:1007700053F82440DCBF0C4B43F820404B885B0708
:100780000FD50B780C4903F00F0309788B42A1BFFA
:10079000044B92781B6853F82220A4BF024B43F805
:1007A000202010BD88290020AA0D0020F72100205C
:1007B000F5210020F4210020F6210020254A002305
:1007C000F0B515681C461A462348244903700B707F
:1007D0002E1976884EB92F5D3FB9037000230A7039
:1007E0004B7007781C461A460CE0360548BF0132AC
:1007F00004F1040403F1010348BFD2B2802CDBB240
:10080000E6D1EAE7E0B2B8420CD215F82400013490
:1008100006099E4200F00F00A8BF731C9042A8BFBB
:10082000421CEFE78A704B70C2F3470102F00102ED
:100830000A444C1E0A490B480A70C3F3470203F0EE
:100840000103134404700849501E084A08701370CD
:10085000F0BD00BF481F0020EC210020982B002095
:10086000F6210020F4210020F7210020F5210020AE
:10087000924B2DE9F04FDA68914D1A612A6891B0D8
:10088000DA60904A0295136843F0200313608E4BA0
:100890001A78012A0CBF002201221A708B4B1A7899
:1008A000910740F14D838A490978042940F2488331
:1008B0008849097801F0040101F0FF0011B922F024
:1008C00001021A701B78DB0702D408B1FCF7CCFBDD
:1008D0008149CA78531C052293FBF2F202EB820293
:1008E0009A1A7E4BCA701F7892000023DFF810829C
:1008F000DFF8109258F82310794C91FBF9FE04F1BF
:10090000080040F823E0774844F8231000FB0E115C
:1009100042F2107091FBF0F004F1100680B226F85C
:1009200013004FF0140C04F114060CFB036C04F1DB
:100930003C0A5AF823605CF802504CF80210761B0F
:10094000314405264AF8231091FBF6F109FB0E11FC
:100950004434012F44F823104FEA830B444605D159
:100960000238B0F5797F98BF4BF808100BB9012316
:10097000BCE7594E029BB2461868336DC01A02F0AC
:10098000EBFF594903F0F4F8029B4FF07E511B68CE
:100990000746336503F0D6F908B94FF07E574B4B45
:1009A000CAF854701B78514E13F00103504D12D009
:1009B0000DAA00924F4B0EAA01920CCB94E80300B3
:1009C000FCF768FA0D9A6421B2FBF1F20E9B3280BB
:1009D00093FBF1F300E033802B809AF858303E4DC2
:1009E000002B35D0696D4FF07E5003F0C1F80746FB
:1009F000EB6D2068C01A02F0B3FF394603F004F82B
:100A000003F0C8F92B6E86B2606836B2C01A02F0E5
:100A1000A7FF394B196802F0F7FF394602F0F4FFDF
:100A200003F0B8F9B5F9662000B28118B5F9642071
:100A30000220B31891FBF0F193FBF0F389B29BB263
:100A4000A5F86A10A5F86830A5F86610A5F8643016
:100A500001238AF85830294B61681B88206803F00D
:100A600030031D4E264DCAF86010CAF85C00002BFA
:100A700000F0668206F17403009306F17803019397
:100A8000F26E336FFCF706FA6B68306FC01A02F033
:100A900067FF194B196802F0B7FF03F07BF9F36E9B
:100AA0002A68C6F880009B1AF3670C4B1B78012B51
:100AB0002AD0022B00F0E68042E200BFA40700200B
:100AC000782D0020F818002066100020FC18002067
:100AD0000219002082310020982B00202C0F0020CA
:100AE0009C2B0020806967FF00007A447619002063
:100AF00078190020681000204C000020C019002048
:100B00000419002080969800D6F88430D6F8A040CA
:100B10000293D6F8943004F100400393D6F898304D
:100B2000776D059303F036F98146204603F032F9DC
:100B3000D6F89C30BB4C0493BB4B06901B684FF01F
:100B4000000B0793B94E4FEA4B0356F82B80A6F1E2
:100B50001402404632F81B50089302F001FF02993C
:100B600002F052FF03F016F9401B1FFA80FA2836F4
:100B700026F81BA00FFA8AFA504602F0F1FE0399FC
:100B800002F042FF03F006F986B20AEB080002F019
:100B9000E7FE059902F038FF394602F035FF21687B
:100BA00002F02AFE03F0F6F8484504DB069B984263
:100BB000A8BF184600E0484602F0D2FE206003F0CD
:100BC000E9F8079B304486B2987802F0C5FE984950
:100BD00002F01AFF01464FF07E5002F0C9FF39467D
:100BE00002F00AFE0146384602F0C2FF0990606832
:100BF000D4F808A0C0EB080002F0B2FE394602F0BB
:100C0000B7FF514602F0F6FD099A0146104602F080
:100C1000FBFE0146504602F0EFFD3135ADB2622DCC
:100C200001462061C4F80480A0600ED9049802F047
:100C3000EBFE03F0AFF87F4AB0F5FA6FA8BF4FF4B0
:100C4000FA609042B8BF104600E0002040F6B8328B
:100C5000064436B29642A8BF1646774A089B96428B
:100C6000B8BF1646754A54F8140B9E52142202FB64
:100C70000BF273495050BBF1000F40F061814FF00F
:100C8000010B5FE7684BB6F8A8401F68736F3D899A
:100C900002935B089D4228BF1D4623B29D4202DCA1
:100CA0001FFA85F90AE06749706D02F0ADFE03F0A6
:100CB00071F820441FFA80F9A6F8A890DAF8786055
:100CC000DAF8AC40341B2046FCF726F941F29313C6
:100CD0000028D8BF40429842CCBF0020012078B302
:100CE000204602F03DFE584902F08EFEF8F741F929
:100CF0000446029802F030FE0146204602F084FECF
:100D000003F048F840F6B83380B2AAF8B00000B259
:100D10009842A8BF1846484B9842ACBF3018F0180C
:100D200048F6A043984203DDA0F50C40A03804E04B
:100D30000028BCBF00F50C40A030CAF8B40001E0A8
:100D4000CAF8B460DAF8B4300026C3F50C50283085
:100D5000039302F005FE3C4902F056FE0446F8F704
:100D60007BF90F902046F8F704F9DAF8B830DAF892
:100D7000C4400593DAF8BC300E9004F100400893AB
:100D800003F008F80490204603F004F8DAF8C030C5
:100D9000DAF854802A4C09900793730048460A9366
:100DA00002F0DEFD0EAB53F8261002F02DFEDFF848
:100DB000A0A005463AF9160002F0D2FD01462846E9
:100DC00002F018FD02F0E6FF05B2204BB5F57A7F80
:100DD000A8BF4FF47A759D42B8BF1D460AF13C0A80
:100DE000A8B22AF8160000B202F0BAFD05998246B0
:100DF00002F00AFE02F0CEFF089983B25046069335
:100E000002F002FE414602F0FFFD216802F0F4FC10
:100E100002F0C0FF049B98421CDB099B9842A8BFCC
:100E2000184618E0680F0020300F0020142C002016
:100E3000DB0FC94030F8FFFF48F4FFFF3A0F0020F6
:100E4000900F00200000C842D302373918FCFFFF82
:100E5000002C0020049802F083FD20608346B878BF
:100E600002F07AFD384902F0CFFD01464FF07E5086
:100E700002F07EFE414602F0BFFC0146404602F011
:100E800077FE0B906068D4F808A0281A02F068FD7D
:100E9000414602F06DFE514602F0ACFCDDF82CC07C
:100EA0000146604602F0B0FD0146504602F0A4FC47
:100EB000656001462061A060079802F0A5FD02F080
:100EC00069FF069B1434034458469A4602F062FFB9
:100ED00040F6B832504400B29042A8BF10461B4AB8
:100EE0000A9B9042B8BF1046194A1A4998521422D8
:100EF000724342F801B00EB901264EE73B792BB19F
:100F0000039A642392FBF3F3134A13803B88029AFB
:100F1000124C9A420DD9D4F8AC30A06FC01AFBF72E
:100F2000FBFF42F2107380EAE072A2EBE0729A4299
:100F300006DD0B4B01221A70B4F8C820064B1A804C
:100F400011B0BDE8F08F00BFDB0FC94048F4FFFFD0
:100F50003A0F0020680F0020280F0020982B002057
:100F60002C0F00200846F6F743BB10B50D4C206847
:100F7000F9F71CFA20680022047A02FB02F3193BFD
:100F8000634303F6C4135343192193FBF1F306495A
:100F900021F812300132072AEFD1BDE81040034991
:100FA000F9F7BCB960100020B80F00204C120020E7
:100FB0000E4B1A78692A16D140F2DC725988914298
:100FC00011D11A79BE2A0ED193F8D9270020EF2A21
:100FD0000BD113F8012B5040054A9342F9D1B0FAD6
:100FE00080F04009704700207047704700F8030800
:100FF000DCFF03082DE9F74FE84C002140F2DC72DA
:10100000204606F046F8E64B04F53A721A60E54BC6
:1010100000221A70E44B04F2B27119606923237044
:10102000032363714FF48073A3604FF41673A4F825
:101030006631FA23A4F86831BC23A4F864314FF474
:10104000FA73A4F86E31012384F8623184F87E319A
:1010500084F88631052384F8273240F2DC53A4F863
:10106000983140F24C43A4F89A3140F26C73A4F8E2
:101070009C3140F27533A4F89E3140F64303A4F846
:10108000A0312346202184F86A116E2184F87C1156
:101090000A2184F87D112B2184F87F11212184F805
:1010A0008011232184F881114FF4C871A4F88211B2
:1010B000032ACCBF0121002102F1010283F8A21111
:1010C00014BF1E217521122A83F8A31103F1020314
:1010D000EED140F27E41A4F8441140F23A71A4F8F6
:1010E000461140F27E51A4F84C1140F2EA5140F210
:1010F000DC50A4F84E1140F2B4514FF4FA63A4F856
:10110000C831A4F8CC31A4F8D031A4F8D4310523E7
:1011100084F8E231C82301264FF47A784FF0320B7D
:10112000A4F8E631DFF878924FF4C8734FF01E0A46
:101130001922A4F8EA31A4F84A01A4F85011A4F83D
:10114000C681A4F8CA81A4F8CE81A4F8D28184F81B
:10115000E46184F8E56184F8E861A4F84881A4F8C2
:1011600052B184F895A184F8E32100920190A4F88B
:10117000543184F8E16184F8EE61A4F856B184F842
:10118000F161FEF77BF9D9F80030009A00254FF0A5
:101190000F0E2674E673A573A58183F805E0DA7156
:1011A0004FF0220E2122172183F806E05A744FF0E7
:1011B0000E0E53225975997583F810E0DA76552191
:1011C0000A224FF0350E2827D97083F81AE02D2116
:1011D0004FF05A0E9A7400924FF0780C642283F804
:1011E0000BA083F80CA0597383F808E01A771D70E0
:1011F0005F709F70DD7583F804B09D731D76DD739D
:101200005D765F7283F80AC019754FF4FA71A3F81E
:101210004E10082183F850106449DFF8ACC199637F
:10122000D9636349C3F82CC0C3F830C09962DFF8B2
:101230009CC14FF07E5159634FF07F5A5D49019830
:10124000C3F820A0C3F824A0C3F848C04FF0000A98
:101250004FF04B0C59649E7783F8525083F85170CD
:10126000C3F840A083F84CC084F8B2E7A4F8BC07E8
:101270004FF0410E042084F8B3E784F8B4B784F843
:10128000B55784F8B95784F8BA5784F8B65784F834
:10129000B75784F8B85783F85C00A3F85850A3F800
:1012A0005A50A3F856501966152183F86810424920
:1012B0004248D966424983F864701967414983F806
:1012C0006570596783F87860FEF702F9D9F8003045
:1012D000009A18464FF4487183F8115183F812515F
:1012E00083F8137183F8146183F81851A3F8161169
:1012F00084F8D821C82284F8D9216422A4F8DA819C
:1013000084F8DC51A4F8DE210E2202FB05326FF0D6
:10131000170482F81941032482F81A416FF02F0450
:1013200082F81B41072482F81C416FF0230482F8E5
:101330001D41052482F81E4101355A2480F82041C0
:1013400080F821416422FF24082D80F81F2180F8B5
:1013500022414FF0000100F10E00D5D1C820A3F8C2
:101360008A01142083F88C01A3F890211E204FF4E9
:10137000967283F88D01A3F892210120282283F828
:10138000891183F88E01A3F894210B46034D5A1955
:101390001033C02BC2F814A0F8D119E008110020B6
:1013A00038100020002D0020601000208FC2F53C76
:1013B000000060400000A0409A99193F75C90108DB
:1013C000F6287C3F3D0A773FCDCCCC3E0000404024
:1013D00005F52A700021402205F05BFE0023264E11
:1013E000EA18995904330868382B244CC2F8A8022B
:1013F000F5D104F50A700021802205F04AFE06F1BD
:101400003801702204F50A7005F038FEFFF7D6F9AE
:10141000D9F8006000230125314604F590604FF4AF
:10142000CC7284F8D83784F8D65784F8D75705F0AB
:1014300025FE04F5C36031464FF4CC7205F01EFE64
:101440000F4B1B681A68C4F8BE275A68C4F8C22735
:101450009A68C4F8C6271A68C4F8CA275A68C4F834
:10146000CE279A680223C4F8D22784F8D45484F88B
:101470006C3603B0BDE8F08F34A9010808110020D4
:1014800060100020074B93F8D837012B08D1064A8B
:10149000064BD0681B68834234BF00200120704790
:1014A00000207047081100201000002024060020B2
:1014B00038B5094B93F8D85765B9084C2068F8F748
:1014C000F2FD074B25601B78022B03D1BDE83840A5
:1014D000FDF793BF38BD00BF08110020C02D0020CC
:1014E000BC2D0020064B93F8D8371BB1012B05D13A
:1014F000FBF738BF034B1868F9F735B90020704780
:1015000008110020C02D0020F8B5011F0646002359
:10151000083051F8042F02F120043F2C3BD802F18F
:1015200008040F2C06D80232032A04D9002B08BF66
:10153000012300E002238142EBD1012B30680ED061
:10154000022B1AD0736800F0030003F003039B0022
:1015500043EA0010B36803F00303184317E000F0F8
:101560000F0040F04000F6F743F8B068736800F0F1
:101570000F0040EA0310C0B209E000F03F0040F065
:101580008000F6F735F83079F6F732F8307ABDE8B2
:10159000F840F6F72DB806F10C0734463A46002518
:1015A00052F8043DAD0003F18001FF2910D903F585
:1015B0000041B1F5803F02D245F0010508E003F596
:1015C0000003B3F1807F34BF45F0020545F0030509
:1015D000B242E5D165F03F00C0B2F6F709F805F078
:1015E0000303022B207807D0032B0CD0012B13D13F
:1015F000F5F7FEFF60780FE0F5F7FAFF6078F5F792
:10160000F7FFA07808E0F5F7F3FF6078F5F7F0FF53
:10161000A078F5F7EDFFE0780434F5F7E9FFBC4278
:101620004FEAA505DBD1F8BD10B50446C0B2F5F709
:10163000DFFFC4F30720BDE81040F5F7D9BF10B5B0
:1016400004467F2C06D964F07F00C0B2F5F7D0FFC6
:10165000E409F6E7E0B2BDE81040F5F7C9BF430082
:1016600083EAE070EBE72DE9F047314B86B093F861
:10167000D8370746012B01D004464AE005F04DFD5E
:101680000546064603A96846FBF77AFD039B049AC4
:10169000029713442B443F2B059519D90023684624
:1016A00003A90322FBF798FD039B3BB9049B2BB9CD
:1016B000204A13705370059BABB301E0FBF748FD64
:1016C000039B049A059E134433447F2B2BD8029F1F
:1016D000DFF860903946CA461AF8024BC4F1800818
:1016E000B04528BFB0460AEB04004444E4B2424689
:1016F00005F0C4FC802C89F8004014D1C8EB060624
:10170000504607EB0801324605F0B8FC89F8006046
:1017100009E0254614F8011B21B1074B1868F9F7B9
:101720002EF8F6E7ED1B284606B0BDE8F08700BFAF
:1017300008110020642C0020C02D00200FB407B534
:1017400004AB53F8042B054900200193F7F7E2FAA4
:1017500003B05DF804EB04B0704700BF650F0108EB
:10176000054A08B5138801339BB21380034B1878E0
:10177000FEF7B8FE002008BDFA0F0020942B0020D1
:101780009148F0B50368914A9C8AA4B2E1B211F085
:10179000010F2ED0198821F400610904090C198069
:1017A000198889B241F48061198000211170517843
:1017B00099B1917811B9D178FF290ED10121917099
:1017C0001179022901BF198889B241F40061198099
:1017D000517941F001011982E1E0517901F0FE01F6
:1017E0001982D378FF2B00F0DA80784BFF21197033
:1017F000D5E08E073AD5BFF35F8F1479E4B2012CA0
:1018000013D1517889B1917879B1198821F4806127
:101810000904090C1980BFF35F8F198B1988947123
:1018200089B241F4007119801BE0198BBFF35F8FFF
:1018300014796649022C0AD14C7844B1897831B1C7
:10184000198821F480610904090C1980A1E0147938
:101850005E49032C05D14C781CB18978002940F0F1
:101860009880998889B241F4806197E04D0756D5F8
:10187000012191715178002937D09178002934D015
:1018800011791C88022911781DD924F4806424045C
:10189000240C1C801E8A9568CCB2F6B249B26E54F4
:1018A000198889B241F4007119800168A31C137072
:1018B0000B8A0134DBB264B22B558B889BB243F4A4
:1018C00080638B8026E0A4B244F400741C801D8ADF
:1018D0009668CCB2EDB249B275541B8A611C49B20C
:1018E000DBB203347354147014E09178374C09B9A7
:1018F000217B41B1198889B241F4007119801378B4
:101900000133137006E0198889B241F4807119809F
:101910000123A37001680B88DB05FCD43FE001F0D4
:10192000400101F0FF05E1B114781F8A9668E5B225
:10193000691C64B2FFB23755C9B21679117049B249
:10194000CC1CA64201BF9C8824F480642404240C8F
:1019500008BF9C8013798B4221D11C4B02351D702E
:101960001DE027061BD511784CB2661C0AD01569FC
:1019700001312C5DC9B21C821479117049B28C42BC
:101980000DD106E0D17815701982517809B9117915
:1019900029B9998821F480610904090C9980137987
:1019A00092F9004001339C4208490CD100238B700E
:1019B0008B7933B101688B8823F440731B041B0CB3
:1019C0008B8000231375F0BD902B0020E82C0020A5
:1019D00010B5224C2368998A89B211F4706F1EBF2A
:1019E0001F4A0120507511F4E06F2BD01A8B9A8892
:1019F000890522F480624FEA02424FEA12429A803D
:101A000020D41A8892051DD41A88D0050FD51A88BB
:101A1000D105FCD41A8892B242F400721A801A8856
:101A20009205FCD40F4B1878FEF75CFD0AE01A888B
:101A300092B242F400721A809A8822F44072120420
:101A4000120C9A802268938A23F470631B041B0C87
:101A50009382034B00221A7510BD00BF902B00200B
:101A6000E82C0020942B002010B51D4C4000C0B283
:101A7000A36023611B4B6071E17001200021217381
:101A80006070227120751868617538B383889B0572
:101A900015D40388D9050DD447F230530288920536
:101AA00002D5013BFAD112E08BB103889BB243F41B
:101AB0008073038083889BB243F44073838047F232
:101AC0003053227D12B1013BFBD100E013B9BDE8D8
:101AD000104045E6024B587D80F0010010BD00BF6C
:101AE000E82C0020902B002013B51F4B400002ACC7
:101AF000C0B2587104F8012DD970012200211A7367
:101B000059701A711A75194A1C6110689C605975D0
:101B100038B38288920515D40288D4050DD447F2D3
:101B200030520188890502D5013AFAD112E08AB112
:101B3000028892B242F480720280828892B242F4A9
:101B40004072828047F23052197D11B1013AFBD1C7
:101B500000E012B9FFF704FE03E0034B587D80F06C
:101B6000010002B010BD00BFE82C0020902B002027
:101B700007B5064B06490093064B074A01930748F1
:101B8000074BF7F7C7F903B05DF804FB74BA010817
:101B900016C1010849BA01080FC101087EC9010830
:101BA00068BA010808B5037833B90C4B0C481978AA
:101BB000BDE80840F7F7AEB905F004FB02280CD8E1
:101BC000064B0C221870074B02FB0030064B02300C
:101BD0001860FFF7CAF90548E5E708BD002D0020A9
:101BE0009EC90108B8180020601000206BBD0108D4
:101BF00008B503783BB90B4B0B4893F8B017BDE819
